:020000040800F2
:100000000000012095760008EF330008F133000866
:10001000F3330008F5330008F73300080000000050
:10002000000000000000000000000000F93300089C
:10003000FB33000800000000FD330008FF33000818
:10004000E5760008E576000801340008E57600084A
:10005000E5760008E57600080D3400081D34000838
:10006000E57600082D340008E576000835340008F0
:10007000413400084D340008E5760008E5760008B4
:10008000593400085D340008E5760008E57600087C
:1000900000000000E576000869340008E5760008F5
:1000A000E5760008E5760008E5760008E5760008C4
:1000B000E5760008E5760008E5760008E5760008B4
:1000C000E5760008E57600086D340008E57600085E
:1000D000E576000879340008E5760008E576000842
:1000E000E5760008E576000885340008E576000826
:1000F000E57600080000000000000000E57600083A
:10010000E5760008E576000891340008E5760008F9
:10011000E5760008E5760008E5760008E576000853
:10012000E5760008E5760008E5760008E576000843
:08013000E5760008E576000801
:1001400010B5054C237833B9044B13B10448AFF311
:1001500000800123237010BD48080020000000002B
:10016000042C030808B5034B1BB103490348AFF344
:10017000008008BD000000004C080020042C03088B
:1001800014214160704714207047406A7047000096
:1001900081010008870100088B010008A101000807
:1001A00010B5044604F1100000F05CFCC4F8F8003F
:1001B0000148C4F87C0110BD90010008F8B5E6B014
:1001C00004460D4616461F460A4906A800F0CAFE18
:1001D00070996F9A05910492009733466E996D9AC3
:1001E000039102922A466C990191214600F060F831
:1001F00067B0F0BD9C010008F8B5E6B004460D46B6
:1002000016461F46094906A800F0ACFE6F996E9A83
:100210000491039200976D996C9A02910192334672
:100220002A46214600F087F867B0F0BD9C0100081F
:1002300038B500281CBF01680029184A23D1184B83
:100240001C684FF6F0710C404CF24025AC421FBFC9
:100250001B6819404CF27024A14212D1114D29683B
:1002600079B911490B68C3F30B03B3F58A6F1FBF4C
:100270000968C1F30B0140F28343994204BF012195
:10028000117028B905E0094B994204BF0121117092
:100290004068BDE8324002F073BC00BF6408002033
:1002A00000ED00E0002004E00010005C0000374892
:1002B0002DE9F04104460D46216816464A681F465E
:1002C00090478046B8F5403F2ED122680A9993683E
:1002D000204698478046B8F5403F25D12368089AC4
:1002E0000799D3F80CC02046E0478046B8F5403F58
:1002F0001AD12368069A39461F692046B8478046B6
:10030000B8F5403F10D1236829465D693246204642
:10031000A8478046B8F5403F06D123680B9A099953
:100320009D692046A847804621680A682046904774
:100330004046BDE8F0812DE9F04104460D462168B4
:1003400016464A681F4690478046B8F5403F2ED172
:1003500022680A999368204698478046B8F5403F3E
:1003600025D12368089A0799D3F80CC02046E047A6
:100370008046B8F5403F1AD12368069A39461F696E
:100380002046B8478046B8F5403F10D1236829463B
:100390005D6932462046A8478046B8F5403F06D101
:1003A00023680999DD6900222046A8478046216814
:1003B0000A68204690474046BDE8F0814FF440303F
:1003C00070470000F0B50C4685B0114600281A466B
:1003D0001CBF0568002D0B4B11D082B104B971B957
:1003E0000D9860B10F9E0E9F0A9B02900496039792
:1003F0000B980C9E009001962046A847034618468D
:1004000005B0F0BD020003002DE9F04F0646D0B064
:100410000868F56DD6F860E0726EB76EF36E00BADC
:1004200000906C46486800BA60600DF1400888682A
:1004300000BAA060C86800BAE060086900BA20612C
:10044000486900BA6061886900BAA061C86900BAE9
:10045000E061086A00BA2062486A00BA6062886A8D
:1004600000BAA062C86A00BAE062086B00BA2063F2
:10047000486B00BA6063886B00BAA063C86B00BAAF
:10048000E063402058F80C1C58F820CC58F838ACE1
:100490008CEA010158F840CC8AEA01018CEA010992
:1004A0004FEAF979401E48F8049BEBD187EA020035
:1004B00000EA0E00784010EBF5610098DFF824C4E4
:1004C00041186144C81882EABE032B404FEAF0612C
:1004D00053405918636859186144CF194FEAB5035E
:1004E00083EABE01014081EABE0111EBF765A16814
:1004F0004D196544A91883EAB0023A404FEAF16504
:100500005A405519E26855194FEAB70282EAB00716
:1005100065440F4005EBBE0E97EAB00717EBFE658A
:1005200027697D194FEAB10782EA0701654401EAAC
:100530000E01EB18514011EBF36561694D194FEA5B
:10054000BE0187EA010E65440EEA030E15EBB0000A
:100550008EEA070E0EEBF065D4F818E0754465449A
:10056000AA1881EAB30505404FEAF26E4D40AE4449
:10057000E569AE44E64477444FEAB00080EAB30E42
:100580000EEA020E8EEAB30E0EEBF765D4F820E009
:1005900075446544691880EAB2053D404FEAF16E42
:1005A0004540AE44656AAE44E6440EEBB3034FEA01
:1005B000B70787EAB20E0EEA010E8EEAB20E0EEB14
:1005C000F365D4F828E075446544281887EAB10536
:1005D0001D404FEAF06E7D40AE44E56AAE44E6440D
:1005E0000EEBB2024FEAB30383EAB10E0EEA000E3D
:1005F0008EEAB10E0EEBF265D4F830E07544654436
:10060000EF1983EAB00515404FEAF76E5D40AE443E
:10061000656BAE44E6440EEBB1014FEAB20282EAEA
:10062000B00E0EEA070E8EEAB00E0EEBF165D4F8AE
:1006300038E075446544EB1882EAB7050D404FEA8F
:10064000F36E5540AE44E56BAE44E6440EEBB000AD
:100650004FEAB10181EAB70E0EEA030E8EEAB70E39
:100660000EEBF065D4F840E07544654481EAB30EC2
:10067000AA180EEA000E4FEAF2658EEA010E7544E2
:10068000DDF844E04FEAB000754480EAB30E6544FB
:100690000EEA020E15EBB7078EEAB30E0EEBF76506
:1006A000DDF848E04FEAB202754480EA020E654484
:1006B0000EEA070E69188EEA000E0EEBF165DDF802
:1006C0004CE07544654405EBB3034FEAB70E1427BD
:1006D0000DF1500CDFF810528EEA010B82EA0B0B81
:1006E0000BEBF36A5CF804BBDA44AA44504483EA97
:1006F000B10B4FEAF06A8EEA0B0BDA445CF804BBEC
:10070000DA44AA44524480EAB30B4FEAF26A8BEA15
:10071000B10BDA445CF804BBDA444FEAB000AA44F7
:1007200080EA020BD6448BEAB30B0BEBFE6A5CF853
:1007300004BBDA444FEAB202AA4482EA0E0B0AEB87
:10074000B10180EA0B0B0BEBF16A5CF804BBDA44F5
:100750007F1DAA44282F0AEBB3034FEABE0EBBD37A
:100760003C2F61D3502F4DD204EB870CC7F15407B7
:100770005E4CA7FB04A504465D4FA8088EEA010A5B
:1007800082EA0A0A5CF804BB0AEBF3655D447D1952
:100790002C1983EAB10A4FEAF4658EEA0A0A554435
:1007A0005CF804AB5CF804BB55447D19AA1884EAD4
:1007B000B30A4FEAF2658AEAB10A55445D444FEA4A
:1007C000B4047D1984EA020AAE448AEAB30A0AEB49
:1007D000FE655CF804AB55444FEAB2027D1982EA2B
:1007E0000E0A15EBB10184EA0A0A5CF804BB0AEBB5
:1007F000F1655D447D1915EBB303401E4FEABE0E53
:10080000BCD12046F46D1B19F365336EC9183166EF
:10081000716E71447166B36ED218B266F16E401893
:10082000F06650B0BDE8F08F4EEA010B0EEA010A07
:100830000BEA020B4BEA0A0A0AEBF36554F827A00D
:10084000DFF8B0C0554443EAB10B654403EAB10A8E
:100850000BEA0E0B28184BEA0A0A7F1C0AEBF0651C
:1008600054F827A0554440EAB30B654400EAB30AA4
:100870000BEAB10BAA184BEA0A0A7F1C0AEBF265D5
:1008800054F827A055444FEAB00040EA020B6544F3
:1008900000EA020A0BEAB30BAE444BEA0A0A7F1CD9
:1008A0000AEBFE6554F827A055444FEAB20242EA2B
:1008B0000E0B654402EA0E0A0BEA000B15EBB101C0
:1008C0004BEA0A0A7F1C0AEBF16554F827A055444D
:1008D0007F1C65443C2F05EBB3034FEABE0EA3D348
:1008E00040E700BF9979825AA1EBD96ECDCCCCCC30
:1008F000D6C162CADCBC1B8F00B581B00168074A53
:10090000914200D110B9064801B000BD7C212EF003
:1009100028FF4FF4003001B000BD00BF040A0008FA
:10092000030002002DE9F0410B4A92E8F85188B02B
:10093000694681E8F8510268084B9A4200D118B91B
:10094000074808B0BDE8F0811422083000F04FFBE2
:1009500008B0BDE8F08100BFE4090008040A0008FF
:1009600003000200152904D20268044B9A4200D108
:1009700008B903487047083000F048BB040A000873
:100980000300020010B481B013460268074CA24273
:1009900000D118B901B010BC0548704701B000F192
:1009A000240210BC083000F035BB00BF040A000868
:1009B0000300020010B481B013460268074CA24243
:1009C00000D118B901B010BC054870470A4601B003
:1009D00000F1240110BC083000F070BB040A0008CC
:1009E000030002000123456789ABCDEFFEDCBA9816
:1009F00076543210F0E1D2C3000000000000000085
:100A000000000000F9080008250900086509000831
:100A100085090008B509000809040008810F0008CD
:100A2000CD0F0008890F0008F0B5A3B004460B48AD
:100A300002900D4616461F46094B0822402104A885
:100A400000F0D1FA28980190009733462A462146B3
:100A500002A800F01BF823B0F0BD00BF040A000894
:100A6000180A000810B5040008BF002408D0054883
:100A7000054B20600822402104F1080000F0B3FA81
:100A8000204610BD040A0008180A00082DE9F041AC
:100A900004460E46216817464A681D469047804620
:100AA000B8F5003F19D12268069993682046984707
:100AB0008046B8F5003F10D123683146DE683A46DB
:100AC0002046B0478046B8F5003F06D12368079A14
:100AD00029461D692046A847804621680A682046A5
:100AE00090474046BDE8F08110B500F033FA4FF46E
:100AF000403400280EBF034C4FF4C0712EF031FE7D
:100B0000204610BD0200030010B5044600F022FA92
:100B100008B9054810BD0021A160D0F87C211168FA
:100B200088474FF4403010BD0200030070B5044602
:100B30000D4600F00FFA064E40B1D0F87C01416836
:100B40008847A84224BF65604FF44036304670BDE8
:100B5000020003002DE9FF4715000C4600D02CB120
:100B6000064600F0F7F95FEA000801D16448C3E0E7
:100B7000D8F8F80001684A689047B0F5003F17D1EF
:100B8000D8F87C118A68404690478146B9F1810FB8
:100B900080F09E80A94508F1FC0A17D2D8F8F80029
:100BA0000368D3F80CC02A462146E047B0F5003F61
:100BB00040F08E80D8F8F8000368D3F810C06A4679
:100BC0005146E047B0F5003F76D10AE0002004E04E
:100BD000215C0AF800100098401C00900098A84280
:100BE000F6D34FF0000C4749474A484B01AC0098F8
:100BF000844558D2D3E9007001ADC5E90070107882
:100C000000281ABF042086464FF0000E085854F8FA
:100C10000E5028443E4D05600127D0F800E0876063
:100C2000019D4F681AF80C007D408EEA050585F09D
:100C3000040E65680F687D4085F0FC05754485F0FD
:100C4000A30568400AF80C000CF1010CCFE7D3E9CA
:100C5000004501A8C0E9004510782E4D002814BFBA
:100C60004FF0040E4FF0000E01A8744651F80EE04C
:100C70000459A6440127CEF80050DEF80040CEF813
:100C800008704D68019F40687D406C400D68684069
:100C900084F0040480F0FC00041984F057040AF87E
:100CA0000C400CF1010CCC45D1D3D8F8F800016808
:100CB0004A689047B0F5003F0AD1D8F8F8000368B9
:100CC000D3F80C804A465146C047B0F5003F01D0EA
:100CD000114811E0002006E05AF8201081F06A3136
:100CE0004AF82010401CB0EB990FF5D3B06840F0E3
:100CF0000100B0604FF4403004B0BDE8F08700BFA1
:100D0000020003004C6D0308640800202C0F00084B
:100D1000ADBE4ED70DBE75A10100030038B50C461F
:100D2000017A1546CA0702D500F014F908B9084837
:100D300032BDD0F8F80003682146DC682A46A04797
:100D4000B0F5003F01D0034832BD4FF4403032BD12
:100D500002000300010003002DE9F84191B00546AF
:100D60000E461746402101A82EF0FBFC297AC80741
:100D700004D5284600F0EEF8040002D1DFF8A48084
:100D80004BE0D4F8F800DFF8A0800368D3F810C077
:100D90006A4601A9E047B0F5003F3ED1D4F8F8001B
:100DA00001684A689047B0F5003F36D1D4F87C110D
:100DB0008A6820469047D4F8F830024618461B68E7
:100DC000D3F80CC004F1FC01E047B0F5003F24D19A
:100DD000D4F87C0141688847D4F8F83002461846B8
:100DE0001B68D3F80CC001A9E047B0F5003F14D14F
:100DF000D4F8F8000268696893689847B0F5003F36
:100E00000BD1D4F8F80003681C693A463146A04774
:100E1000B0F5003F08BF4FF44038404612B0BDE87F
:100E2000F08100BF02000300010003002DE9F8413A
:100E3000A5B0074688461646402115A82EF091FC1D
:100E400000220492402105A82EF08BFC387AC107BD
:100E50005ED5384600F07EF8050059D0D5F8F80088
:100E60002D4C0368D3F810C06A4605A9E047B0F5D9
:100E7000003F3CD1D5F8F80001684A689047B0F5CA
:100E8000003F34D1D5F87C118A6828469047D5F8C0
:100E9000F830024618461B68D3F80CC005F1FC0177
:100EA000E047B0F5003F22D1D5F87C014168884782
:100EB000D5F8F830024618461B68D3F80CC005A9CF
:100EC000E047B0F5003F12D1D5F8F8000268796824
:100ED00093689847B0F5003F09D1D5F8F80003684A
:100EE0001D6904AA15A9A847B0F5003F01D0204606
:100EF0000FE00A4B0A490B4A0396029101924046C1
:100F00001C68049B009415AA796800F0E5F900E0DC
:100F1000054826B0BDE8F08101000300546D0308C8
:100F2000936E030026C703000200030004B0010112
:100F300000170145E90A0008090B00082D0B0008FD
:100F4000BD030008550B00081D0D0008590D0008D1
:100F50002D0E00080168024A914218BF0020704718
:100F6000340F000810B5040008BF002404D0034863
:100F70002060204609688847204610BD340F0008CD
:100F800020225C302EF0E9BBF0B58468A308002273
:100F900004F0030407E000F15C0555F8226035BA5F
:100FA00041F82250521C9A42F5D300220BE000F186
:100FB0005C0502EB830755F82360D500C5F11805E1
:100FC000EE40CE55521CA242F1D3F0BD30B5C468FC
:100FD00003690022E31AD5188C5C0544521C082AC8
:100FE0002C77F8D330BD0360C1600261704738B51B
:100FF000044615460022626023685A689047002024
:101000006061A061A5604FF4003032BD81604FF493
:10101000003070472DE9F84304462079D4F80C805D
:10102000450748BF244845D466691D46A8F101001C
:1010300000EAD60306EBC506B6EBC50F666102D221
:10104000A669761CA6611746A66906EB5576A661C9
:101050000E46E918884225D2A8EB03094A463146D4
:10106000F8182EF07AFB2268136839460FE04246E2
:1010700038462EF072FB23681A683946204690479E
:1010800007E0311811F00300F1D1226813682046FF
:101090009847484600EB0809A9F10101A942F0D39D
:1010A000002300E000202A1A3118F8182EF055FB12
:1010B0004FF40030BDE8F283040002002DE9FC4F3C
:1010C000024685B0D0681369DFF86CC1DFF86C8127
:1010D000A0EB030A506840F004005060002703A80A
:1010E00002900DF10C0ED8E9003403A8544DC0E96C
:1010F00000342878534D00280CBF00230423994660
:101100005CF803305EF80940234401261D601C682A
:101110009E60DCF80430039DDCF80090DEF804608B
:101120005D406540484C654089EA0606474C66408C
:101130007519474C6540D8E9006B03AC0028C4E939
:10114000006B0EBF002404200424029E5CF8000003
:10115000345920183F4C04600126046886600398C7
:10116000029E43406340384C7068634089EA000047
:10117000364C6040034438484340280018BF0120E3
:101180005B1E9B41042F2CBFC0B2D80F02F1140389
:1011900053F8200007F00303C3F10303DB00D8403A
:1011A0000DF807007F1C082F9DD315460C466A6971
:1011B000AB69E868D20842EA4372401E00EA0207BF
:1011C000002302409B420AD8524508D28020E055B5
:1011D0007F1C574516D2AAEB0701E01910E08020CA
:1011E000E05500E0E355E8687F1C8742FAD32A689F
:1011F000136828469847BAF1000F03D0514620469D
:101200002EF0AFFA2A68069E059F93686946284625
:1012100098472A68D2F8009021462846C8472B688C
:10122000DA683946284690470EB1A86830604FF416
:10123000003007B0BDE8F08F4C6D03085C12000869
:10124000640800205FC5109304850012FC68017AD1
:10125000C0F524FF24AF33D426AF698B04B001015D
:1012600000170145F8B501240094002300240DE087
:10127000009D065D0F5D7E40F643761CF60F86F0FE
:10128000010635400095641C009DEB189442EFD395
:101290001846F2BDF8B5002301240094002A11E09D
:1012A000009C85188F1815F8016C17F8015C6E40CA
:1012B000F643761CF60F86F0010634400094009C3D
:1012C000E318521EECD11846F2BD0000651200086A
:1012D00095120008010000002DE9F84F1D46DDF8C9
:1012E00028900B9F0D9C4FF0FF3300930E469246C3
:1012F000D9F800B0804632465146D847834664B399
:10130000D9F8043032465146404698476FEA0B02FE
:10131000521C42EA0B0200996FEAD2735B1C19401F
:10132000C2430091521C024300996FEAD2735B1CC6
:101330001940009186F05531484087EA000181F05C
:101340005531216080F05531C943491C0843009A4A
:101350006FEAD070401C82430092D9F8080001283F
:1013600009D17540E943491C0D4300986FEAD572D5
:10137000521C90430AE0F11C85EA9102D243521CB0
:10138000154300986FEAD5735B1C984386F0AA3624
:10139000009086EA0B0686F0AA33F243DB430C98F2
:1013A000C2F3C0725B1C42EAD3720099D243521C52
:1013B00091430091774000998843009987F0AA37BC
:1013C0000F403843BDE8F28F00000000000000002D
:1013D00001F0FF01102A2BDB10F0070F08D010F8E6
:1013E000013B013A8B422DD010F0070F42B3F6D1EA
:1013F000F0B441EA012141EA014122F007047FF003
:1014000000070023F0E80256083C85EA010586EA59
:10141000010685FA47F5A3FA87F586FA47F6A5FA95
:1014200087F68EB9EED1F0BC01F0FF0102F00702A1
:1014300032B110F8013B013A83EA010313B1F8D14C
:101440000020704701387047002D06BF354603382D
:10145000073815F0010F07D1013015F4807F02BF66
:10146000013015F4C03F0130F0BC0138704700BFB7
:10147000034613F8012B002AFBD1181A01387047D4
:1014800081F0004102E000BF83F0004330B54FEA35
:1014900041044FEA430594EA050F08BF90EA020FA2
:1014A0001FBF54EA000C55EA020C7FEA645C7FEA35
:1014B000655C00F0E2804FEA5454D4EB5555B8BF58
:1014C0006D420CDD2C4480EA020281EA030382EAC9
:1014D000000083EA010180EA020281EA0303362D5B
:1014E00088BF30BD11F0004F4FEA01314FF4801C2E
:1014F0004CEA113102D0404261EB410113F0004F40
:101500004FEA03334CEA133302D0524263EB4303F6
:1015100094EA050F00F0A780A4F10104D5F1200E94
:101520000DDB02FA0EFC22FA05F2801841F10001EF
:1015300003FA0EF2801843FA05F359410EE0A5F1C3
:1015400020050EF1200E012A03FA0EFC28BF4CF0F4
:10155000020C43FA05F3C01851EBE37101F00045AA
:1015600007D54FF0000EDCF1000C7EEB00006EEBB7
:101570000101B1F5801F1BD3B1F5001F0CD3490841
:101580005FEA30004FEA3C0C04F101044FEA445298
:1015900012F5800F80F09A80BCF1004F08BF5FEA1F
:1015A000500C50F1000041EB045141EA050130BDFF
:1015B0005FEA4C0C404141EB0101013C28BFB1F511
:1015C000801FE9D291F0000F04BF01460020B1FA5C
:1015D00081F308BF2033A3F10B03B3F120020CDA2F
:1015E0000C3208DD02F1140CC2F10C0201FA0CF00D
:1015F00021FA02F10CE002F11402D8BFC2F1200C72
:1016000001FA02F120FA0CFCDCBF41EA0C01904027
:10161000E41AA2BF01EB0451294330BD6FEA040470
:101620001F3C1CDA0C340EDC04F11404C4F120025B
:1016300020FA04F001FA02F340EA030021FA04F36D
:1016400045EA030130BDC4F10C04C4F1200220FAC4
:1016500002F001FA04F340EA0300294630BD21FA02
:1016600004F0294630BD94F0000F83F4801306BFC8
:1016700081F480110134013D4EE77FEA645C18BFBC
:101680007FEA655C29D094EA050F08BF90EA020F53
:1016900005D054EA000C04BF1946104630BD91EA4B
:1016A000030F1EBF0021002030BD5FEA545C05D14E
:1016B0004000494128BF41F0004130BD14F580048D
:1016C0003CBF01F5801130BD01F0004545F0FE4101
:1016D00041F470014FF0000030BD7FEA645C1ABF36
:1016E000194610467FEA655C1CBF0B46024650EA6D
:1016F000013406BF52EA033591EA030F41F4002199
:1017000030BD00BF90F0000F04BF0021704730B51E
:101710004FF4806404F132044FF000054FF00001F3
:1017200050E700BF90F0000F04BF0021704730B5B4
:101730004FF4806404F1320410F0004548BF404289
:101740004FF000013EE700BF42004FEAE2014FEADE
:1017500031014FEA02701FBF12F07F4393F07F4FB9
:1017600081F06051704732F07F4208BF704793F0BC
:101770007F4F04BF41F40021704730B54FF46074CF
:1017800001F0004521F000411CE700BF50EA0102D2
:1017900008BF704730B54FF000050AE050EA01027B
:1017A00008BF704730B511F0004502D5404261EBEB
:1017B00041014FF4806404F132045FEA915C3FF42C
:1017C000D8AE4FF003025FEADC0C18BF03325FEAC9
:1017D000DC0C18BF033202EBDC02C2F1200300FA7A
:1017E00003FC20FA02F001FA03FE40EA0E0021FA9F
:1017F00002F11444BDE600BF70B54FF0FF0C4CF48D
:10180000E06C1CEA11541DBF1CEA135594EA0C0F3E
:1018100095EA0C0F00F0DEF82C4481EA030621EA79
:101820004C5123EA4C5350EA013518BF52EA0335B4
:1018300041F4801143F4801338D0A0FB02CE4FF066
:101840000005E1FB02E506F00042E0FB03E54FF096
:101850000006E1FB03569CF0000F18BF4EF0010E8E
:10186000A4F1FF04B6F5007F64F5407404D25FEA8A
:101870004E0E6D4146EB060642EAC62141EA55513D
:101880004FEAC52040EA5E504FEACE2EB4F1FD0C7F
:1018900088BFBCF5E06F1ED8BEF1004F08BF5FEAFD
:1018A000500E50F1000041EB045170BD06F00046AF
:1018B00046EA010140EA020081EA0301B4EB5C045C
:1018C000C2BFD4EB0C0541EA045170BD41F4801154
:1018D0004FF0000E013C00F3AB8014F1360FDEBF79
:1018E000002001F0004170BDC4F10004203C35DA55
:1018F0000C341BDC04F11404C4F1200500FA05F3D8
:1019000020FA04F001FA05F240EA020001F0004278
:1019100021F0004110EBD37021FA04F642EB0601EE
:101920005EEA430E08BF20EAD37070BDC4F10C0418
:10193000C4F1200500FA04F320FA05F001FA04F2DC
:1019400040EA020001F0004110EBD37041F10001C8
:101950005EEA430E08BF20EAD37070BDC4F12005D3
:1019600000FA05F24EEA020E20FA04F301FA05F23B
:1019700043EA020321FA04F001F0004121FA04F2E3
:1019800020EA020000EBD3705EEA430E08BF20EAB3
:10199000D37070BD94F0000F0FD101F000464000ED
:1019A00041EB010111F4801F08BF013CF7D041EA6F
:1019B000060195F0000F18BF704703F00046520073
:1019C00043EB030313F4801F08BF013DF7D043EA44
:1019D0000603704794EA0C0F0CEA135518BF95EAFA
:1019E0000C0F0CD050EA410618BF52EA4306D1D181
:1019F00081EA030101F000414FF0000070BD50EAA0
:101A0000410606BF1046194652EA430619D094EA29
:101A10000C0F02D150EA013613D195EA0C0F05D113
:101A200052EA03361CBF104619460AD181EA030167
:101A300001F0004141F0FE4141F470014FF000001F
:101A400070BD41F0FE4141F4780170BD70B54FF0BA
:101A5000FF0C4CF4E06C1CEA11541DBF1CEA13553A
:101A600094EA0C0F95EA0C0F00F0A7F8A4EB05041C
:101A700081EA030E52EA03354FEA013100F0888013
:101A80004FEA03334FF0805545EA131343EA1263DC
:101A90004FEA022245EA111545EA10654FEA002691
:101AA0000EF000419D4208BF964244F1FD0404F54A
:101AB000407402D25B084FEA3202B61A65EB0305A6
:101AC0005B084FEA32024FF480104FF4002CB6EB63
:101AD000020E75EB030E22BFB61A754640EA0C00E3
:101AE0005B084FEA3202B6EB020E75EB030E22BF23
:101AF000B61A754640EA5C005B084FEA3202B6EB64
:101B0000020E75EB030E22BFB61A754640EA9C0022
:101B10005B084FEA3202B6EB020E75EB030E22BFF2
:101B2000B61A754640EADC0055EA060E18D04FEAB0
:101B3000051545EA16754FEA06164FEAC30343EA50
:101B400052734FEAC2025FEA1C1CC0D111F4801F1D
:101B50000BD141EA00014FF000004FF0004CB6E716
:101B600011F4801F04BF01430020B4F1FD0C88BFB5
:101B7000BCF5E06F3FF6AFAEB5EB030C04BFB6EBC0
:101B8000020C5FEA500C50F1000041EB045170BDB3
:101B90000EF0004E4EEA113114EB5C04C2BFD4EBE0
:101BA0000C0541EA045170BD41F480114FF0000E64
:101BB000013C90E645EA060E8DE60CEA135594EAE0
:101BC0000C0F08BF95EA0C0F3FF43BAF94EA0C0FE3
:101BD0000AD150EA01347FF434AF95EA0C0F7FF458
:101BE00025AF104619462CE795EA0C0F06D152EAAC
:101BF00003353FF4FDAE1046194622E750EA410690
:101C000018BF52EA43067FF4C5AE50EA41047FF4A0
:101C10000DAF52EA43057FF4EBAE12E74FF0FF3C05
:101C200006E000BF4FF0010C02E000BF4FF0010CD6
:101C30004DF804CD4FEA410C7FEA6C5C4FEA430C4F
:101C400018BF7FEA6C5C1BD001B050EA410C0CBF9E
:101C500052EA430C91EA030F02BF90EA020F002000
:101C6000704710F1000F91EA030F58BF994208BF67
:101C700090422CBFD8176FEAE37040F00100704724
:101C80004FEA410C7FEA6C5C02D150EA013C07D17B
:101C90004FEA430C7FEA6C5CD6D152EA033CD3D0C6
:101CA0005DF8040B704700BF8446104662468C46C0
:101CB0001946634600E000BF01B5FFF7B7FF0028F3
:101CC00048BF10F1000F01BD4DF808EDFFF7F4FF1C
:101CD0000CBF012000205DF808FB00BF4DF808EDA7
:101CE000FFF7EAFF34BF012000205DF808FB00BFCA
:101CF0004DF808EDFFF7E0FF94BF012000205DF8EC
:101D000008FB00BF4DF808EDFFF7CEFF94BF0120A0
:101D100000205DF808FB00BF4DF808EDFFF7C4FF99
:101D200034BF012000205DF808FB00BF4FEA410CE2
:101D30007FEA6C5C02D150EA013C0AD14FEA430CC5
:101D40007FEA6C5C02D152EA033C02D14FF0000002
:101D500070474FF0010070474FEA410212F5001240
:101D600015D211D56FF47873B3EB625212D94FEAE2
:101D7000C12343F0004343EA505311F0004F23FACC
:101D800002F018BF404270474FF00000704750EA21
:101D9000013005D111F0004008BF6FF000407047DE
:101DA0004FF00000704700BF4FEA4102B2F1E0433C
:101DB00024BFB3F5001CDCF1FE5C0DD901F0004C32
:101DC0004FEAC0024CEA5070B2F1004F40EB830082
:101DD00008BF20F00100704711F0804F21D113F1AE
:101DE0003872BCBF01F00040704741F480114FEAE7
:101DF0005252C2F11802C2F1200C10FA0CF320FA70
:101E000002F018BF40F001004FEAC1234FEAD3238C
:101E100003FA0CFC40EA0C0023FA02F34FEA4303F6
:101E2000CCE77FEA625307D150EA01331EBF4FF07F
:101E3000FE4040F44000704701F0004040F0FE409A
:101E400040F40000704700BF80F0004002E000BF97
:101E500081F0004142001FBF5FEA410392EA030F95
:101E60007FEA226C7FEA236C6AD04FEA1262D2EBDF
:101E70001363C1BFD218414048404140B8BF5B42E4
:101E8000192B88BF704710F0004F40F4000020F07D
:101E90007F4018BF404211F0004F41F4000121F093
:101EA0007F4118BF494292EA030F3FD0A2F10102DD
:101EB00041FA03FC10EB0C00C3F1200301FA03F11B
:101EC00000F0004302D5494260EB4000B0F5000F3E
:101ED00013D3B0F1807F06D340084FEA310102F1FD
:101EE0000102FE2A51D2B1F1004F40EBC25008BFAF
:101EF00020F0010040EA03007047490040EB000079
:101F0000013A28BFB0F5000FEDD2B0FA80FCACF179
:101F1000080CB2EB0C0200FA0CF0AABF00EBC250A6
:101F200052421843BCBFD0401843704792F0000F94
:101F300081F4000106BF80F400000132013BB5E7E7
:101F40004FEA41037FEA226C18BF7FEA236C21D05D
:101F500092EA030F04D092F0000F08BF08467047C2
:101F600090EA010F1CBF0020704712F07F4F04D190
:101F7000400028BF40F00040704712F100723CBFA3
:101F800000F50000704700F0004343F0FE4040F4CD
:101F9000000070477FEA226216BF08467FEA23638B
:101FA0000146420206BF5FEA412390EA010F40F476
:101FB000800070474FF0000304E000BF10F00043C2
:101FC00048BF40425FEA000C08BF704743F09643A9
:101FD00001464FF000001CE050EA010208BF7047C4
:101FE0004FF000030AE000BF50EA010208BF70474B
:101FF00011F0004302D5404261EB41015FEA010C60
:1020000002BF84460146002043F0B64308BFA3F157
:102010008053A3F50003BCFA8CF2083AA3EBC25339
:1020200010DB01FA02FC634400FA02FCC2F1200258
:10203000BCF1004F20FA02F243EB020008BF20F08F
:102040000100704702F1200201FA02FCC2F12002F5
:1020500050EA4C0021FA02F243EB020008BF20EAEA
:10206000DC7070474FF0FF0C1CEAD0521EBF1CEA18
:10207000D15392EA0C0F93EA0C0F6FD01A4480EA06
:10208000010C400218BF5FEA41211ED04FF00063EF
:1020900043EA501043EA5111A0FB01310CF000401B
:1020A000B1F5000F3EBF490041EAD3715B0040EA41
:1020B000010062F17F02FD2A1DD8B3F1004F40EB11
:1020C000C25008BF20F00100704790F0000F0CF0E4
:1020D000004C08BF49024CEA502040EA51207F3AA8
:1020E000C2BFD2F1FF0340EAC250704740F4000083
:1020F0004FF00003013A5DDC12F1190FDCBF00F074
:1021000000407047C2F10002410021FA02F1C2F121
:10211000200200FA02FC5FEA310040F1000053EABD
:102120004C0308BF20EADC70704792F0000F00F00B
:10213000004C02BF400010F4000F013AF9D040EA11
:102140000C0093F0000F01F0004C02BF490011F4A5
:10215000000F013BF9D041EA0C018FE70CEAD153A3
:1021600092EA0C0F18BF93EA0C0F0AD030F0004C23
:1021700018BF31F0004CD8D180EA010000F00040D7
:10218000704790F0000F17BF90F0004F084691F095
:10219000000F91F0004F14D092EA0C0F01D14202CF
:1021A0000FD193EA0C0F03D14B0218BF084608D198
:1021B00080EA010000F0004040F0FE4040F40000E2
:1021C000704740F0FE4040F4400070474FF0FF0C75
:1021D0001CEAD0521EBF1CEAD15392EA0C0F93EABC
:1021E0000C0F69D0A2EB030280EA010C49024FEA0E
:1021F000402037D04FF0805343EA111143EA1013C7
:102200000CF000408B4238BF5B0042F17D024FF47E
:10221000000C8B4224BF5B1A40EA0C00B3EB510F59
:1022200024BFA3EB510340EA5C00B3EB910F24BF42
:10223000A3EB910340EA9C00B3EBD10F24BFA3EBC7
:10224000D10340EADC001B0118BF5FEA1C1CE0D18F
:10225000FD2A3FF650AF8B4240EBC25008BF20F042
:10226000010070470CF0004C4CEA50207F32C2BF96
:10227000D2F1FF0340EAC250704740F400004FF033
:102280000003013A37E792F0000F00F0004C02BF64
:10229000400010F4000F013AF9D040EA0C0093F02E
:1022A000000F01F0004C02BF490011F4000F013B88
:1022B000F9D041EA0C0195E70CEAD15392EA0C0FF0
:1022C00008D142027FF47DAF93EA0C0F7FF470AF28
:1022D000084676E793EA0C0F04D14B023FF44CAF6B
:1022E00008466EE730F0004C18BF31F0004CCAD100
:1022F00030F000427FF45CAF31F000437FF43CAF3C
:102300005FE700BF4FF0FF3C06E000BF4FF0010C5D
:1023100002E000BF4FF0010C4DF804CD4FEA40023F
:102320004FEA41037FEA226C18BF7FEA236C11D089
:1023300001B052EA530C18BF90EA010F58BFB2EB3C
:10234000030088BFC81738BF6FEAE17018BF40F0BC
:10235000010070477FEA226C02D15FEA402C05D170
:102360007FEA236CE4D15FEA412CE1D05DF8040BF5
:10237000704700BF844608466146FFE70FB5FFF788
:10238000C9FF002848BF10F1000F0FBD4DF808ED40
:10239000FFF7F4FF0CBF012000205DF808FB00BF31
:1023A0004DF808EDFFF7EAFF34BF012000205DF88B
:1023B00008FB00BF4DF808EDFFF7E0FF94BF0120D8
:1023C00000205DF808FB00BF4DF808EDFFF7D2FFD5
:1023D00094BF012000205DF808FB00BF4DF808ED18
:1023E000FFF7C8FF34BF012000205DF808FB00BFE5
:1023F0004FEA40024FEA41037FEA226C02D15FEAD2
:10240000402C08D17FEA236C02D15FEA412C02D133
:102410004FF0000070474FF0010070474FEA400254
:10242000B2F1FE4F0FD34FF09E03B3EB12620DD902
:102430004FEA002343F0004310F0004F23FA02F06C
:1024400018BF404270474FF00000704712F1610F13
:1024500001D1420205D110F0004008BF6FF00040EA
:1024600070474FF00000704742000ED2B2F1FE4FAD
:102470000BD34FF09E03B3EB126209D44FEA002353
:1024800043F0004323FA02F070474FF0000070471A
:1024900012F1610F01D1420202D14FF0FF307047BB
:1024A0004FF00000704700BF53B94AB9002908BF78
:1024B00000281CBF4FF0FF314FF0FF3000F06AB929
:1024C000ADF1080C6DE904CE00F006F8DDF804E08B
:1024D000DDE9022304B070472DE9F047089D0C4662
:1024E000002B4ED194468C458646B2FA82F262D9D0
:1024F0004AB1C2F12003914020FA03F30CFA02FC26
:10250000194300FA02FE4FEA1C471FFA8CF6B1FB92
:10251000F7F44FEA1E4307FB141143EA014304FB9F
:1025200006F199420AD91CEB030304F1FF3080F055
:102530001281994240F20F81023C6344591A1FFAFA
:102540008EF3B1FBF7F007FB101143EA014300FBE8
:1025500006F69E420AD91CEB030300F1FF3180F01E
:10256000FC809E4240F2F980634402389B1B40EAA3
:10257000044000211DB1D3400022C5E90032BDE86E
:10258000F0878B4205D90DB1C5E90001002108464D
:10259000F5E7B3FA83F1002946D1A34202D3904272
:1025A000C0F0F080861A64EB03030120002DE6D012
:1025B000C5E90063E3E7002A40F09080A1EB0C043A
:1025C0004FEA1C481FFA8CF70121B4FBF8F64FEADA
:1025D0001E4308FB164443EA044307FB06F09842F7
:1025E00008D91CEB030306F1FF3402D2984200F233
:1025F000CD8026461C1A1FFA8EF3B4FBF8F008FBB8
:10260000104443EA044300FB07F79F4208D91CEB40
:10261000030300F1FF3402D29F4200F2B080204653
:10262000DB1B40EA0640A5E7C1F120068B4022FAF9
:1026300006F71F4320FA06FC04FA01F343EA0C03F1
:10264000F44000FA01F8380C4FEA1349B4FBF0FEED
:102650001FFA87FC00FB1E4449EA04440EFB0CF9F8
:10266000A14502FA01F20AD93C190EF1FF3A80F0B5
:102670008480A14540F28180AEF1020E3C44A4EB7F
:1026800009041FFA83F9B4FBF0F300FB134449EA91
:10269000044403FB0CFCA44507D93C1903F1FF30AB
:1026A00067D2A44565D9023B3C4443EA0E40A0FBF7
:1026B0000293A4EB0C049C42CE469C4651D34ED0D0
:1026C00055B1B8EB0E0364EB0C0404FA06F6CB40EC
:1026D0001E43CC40C5E90064002150E7C2F120034D
:1026E00020FA03F10CFA02FC24FA03F394400C43A1
:1026F0004FEA1C4800FA02FE1FFA8CF7B3FBF8F011
:1027000008FB1031230C43EA014300FB07F1994217
:1027100008D91CEB030300F1FF362CD299422AD9C9
:10272000023863445B1AA4B2B3FBF8F108FB11331F
:1027300044EA034401FB07F3A34208D91CEB040459
:1027400001F1FF3613D2A34211D902396444E41ACD
:1027500041EA004139E70446F0E6084606E7C84585
:10276000AED2B9EB020E63EB070C0138A8E7314695
:10277000EDE7034699E73046D4E7D6467FE7634462
:1027800002384DE70646234608460FE7023E6344FB
:1027900030E700BF704700BF00487047001BB74BD1
:1027A00070B50C4601F0D8F9104E054608213046A8
:1027B00006F094F8012804D001F0CEF9431BA3429F
:1027C00007D30821094806F089F8431E58425841AA
:1027D00070BD72B60821304606F080F8012800D09E
:1027E00030BF62B6BFF36F8FE0E700BF0004004860
:1027F00008B5002210214FF0904006F075F805480A
:102800000022202106F070F8BDE80840022001F007
:10281000ABB900BF0004004810B50C4C01221021D8
:10282000204606F061F8052001F09EF920460122BD
:10283000202106F059F84FF090400122102106F0B7
:1028400053F8BDE81040022001F08EB900040048A2
:1028500070B54FF090400C46164610210022144DE2
:1028600006F042F800232B701248B3B222462146EC
:1028700007F02EFAD8B901F06FF941F28736044615
:102880002B783BB1BDE87040012210214FF0904001
:1028900006F02AB801F060F9031BB342F2D872B611
:1028A0002B7803B930BF62B6BFF36F8FE8E770BD16
:1028B00065080020C8090020014B01221A707047EA
:1028C0006508002000487047586D030813B5114B88
:1028D0000446186800909B88ADF804300120FFF78B
:1028E0009BFF062269460120FFF7B2FF0120FFF798
:1028F0007FFF9DF80430112B08D19DF80520122A86
:1029000004D101202370627002B010BD00231A466A
:102910001846F7E7202C03080CB4F0B5ADB032AB85
:1029200006AF53F8042B059305460E46384696210C
:102930002CF066FE9528C1BF42F62E63ADF8AA3092
:102940002E23ADF8AC3000F037F83C24042D4FF4C2
:102950007A7E1449B0FBFEFCB0FBF1F14EF6602329
:10296000B0FBF3F3B3FBF4F204FB1232BCFBF4F361
:1029700004FB13C30EFB1C049ABF0B48405D3F20B1
:10298000CDE90040CDE9026708482CF0B9FD084BBD
:102990001B6898682CF0DEFC2DB0BDE8F04002B05A
:1029A000704700BF80EE3600B66D0308946D0308D3
:1029B0007006002001F0D8B801F0CEB81348144AD0
:1029C00008B54FF00043C0E9002304224261012210
:1029D0000023C2614FF480510722C0E90233C0E9ED
:1029E0000933C0E90C1203610383837680F8203039
:1029F00080F82C30826380F83C30C36404F0C6FE5B
:102A000018B1BDE8084000F099BB08BD6808002077
:102A1000002401400268084B9A4282B00AD14FF06C
:102A2000B0431A6E42F400721A661B6E03F4007310
:102A30000193019B02B07047002401400268054BDE
:102A40009A4201BF4FF0B042136E23F40073136635
:102A5000704700BF0024014030B585B00024054612
:102A6000CDE901440394FFF7A9FF144805F022FAC9
:102A700008B100F063FB1148039401A9CDE90154AA
:102A800004F0E2FF08B100F059FB0C4805F03CF9F6
:102A900008B100F053FB4FF0FF31084804F076FF17
:102AA000064805F0E9F9054804F0CAFF0446034862
:102AB00005F08CF9204605B030BD00BF6808002045
:102AC000014B024A1A607047680800200024014048
:102AD00008B50948FFF7C0FF68B1084BB3F8AA3042
:102AE0004FF6FF72934216BF40F6E442044B534345
:102AF000B3FBF0F398B208BD002000B40075FF1FCF
:102B0000D8084C0013B50023ADF80630FFF7E0FFFE
:102B100004461948FFF7A0FF184BB3F8C820B3F8D4
:102B2000A8108A4204FB00F018D040F6E443B0FB42
:102B3000F3F364205B1A4343521A93FBF2F31E3300
:102B40001BB2ADF80630BDF806305BB21B02ADF823
:102B50000630BDF8060000B202B010BD4FF47A7224
:102B600040F6FF73B0FBF3F35343A3F53923A3F50A
:102B70000C6340F6C412E0E7001000B00075FF1FC0
:102B80004FF0B04382B09A6A22F480529A629A6CF3
:102B900042F480529A649B6C03F480530193019B2E
:102BA000002002B070474FF0B04307B59A6C42F076
:102BB00004029A649A6C02F004020192019A9A6CDF
:102BC00042F001029A649B6C002203F0010311465B
:102BD00000930B20009B05F00BFA0B2005F03AFA4E
:102BE000002211460C2005F003FA0C2005F032FA01
:102BF000002211460D2005F0FBF90D2005F02AFA00
:102C0000002202210F2005F0F3F90F2005F022FA2F
:102C100000221146102005F0EBF9102005F01AFAF9
:102C200000221146112005F0E3F9112003B05DF8F0
:102C300004EB05F00FBA000008B505F04FFC10B129
:102C40006FF0040008BD064B9A6942F040429A6159
:102C50004CF2FA321A6105F053FC0028F2D0EFE78B
:102C600000400058F0B585B000230D46009306469D
:102C7000A8B3FFF7E1FF044670BB05F02FFC88BB4B
:102C80001A481B4A02230193D0F8E01506F1784355
:102C900002EA8121B3FBF1F701FB1733DB0A029350
:102CA000D0F8E00505F178410139314402EA80228B
:102CB000B1FBF2F002FB1011C3EBD12301336946E3
:102CC00001A8039305F09CFC20B1022814BF6FF00B
:102CD0000104012405F014FC204605B0F0BD6FF09E
:102CE0000504F9E76FF00404F6E700BF0070FF1F6A
:102CF00000FCFF03014B186000207047CC08002047
:102D00002DE9F04FB0F1006F89B006460F469046AE
:102D1000C0F0C080DFF89091644DD9F8E03505EA45
:102D2000832303F10063013B984200F2B380002942
:102D300000F0B38040EA02035B0740F0AE80FFF78B
:102D40007BFF044690BB05F0C9FB002840F0A8803B
:102D5000D9F8E015009705EA812106F17842B2FB27
:102D6000F1F301FB132208F17843013B3344B3FB39
:102D7000F1F001FB1033DB0A01334FEAD22AA3EB57
:102D8000D222012A039388BFC6F30A050AF58037C9
:102D9000C6F108038CBFC5F500654546FF02B34682
:102DA0000693039B9A4505D305F0AAFB204609B07C
:102DB000BDE8F08FA6F10803069A1A4495421CD884
:102DC000009B04950193CDF814B04FF00009059BCA
:102DD00009EB0301049B99453DD3009BAB442B4475
:102DE000A8EB0505B5F5006F009328BF4FF400650B
:102DF0000AF1010A07F50067D3E753F8081F5A687C
:102E0000B2F1FF3F08BFB1F1FF3FD5D0284B1868A2
:102E100010B96FF00504C7E727B14FF400623946D7
:102E200012F0F0FDDFF888900099D9F80030CBF36C
:102E30000A001844AAB212F0E5FD4FF400613846CA
:102E4000FFF710FF00BBD9F8003001934FF4006387
:102E500005970493B9E7019B07914B440293012026
:102E6000D3E9002305F086FB88B90799019BD1E9D6
:102E7000000259F80310029B5B689A4208BF88421F
:102E800005D109F10809A2E76FF001048CE76FF0A2
:102E9000030489E74FF0FF3488E76FF0050485E706
:102EA0006FF0040482E700BF0070FF1F00FCFF0307
:102EB000CC080020B1F1006F70B510D30B4BD3F8E4
:102EC000E0650B4B03EA862303F10063013B994263
:102ED00005D838B192B212F095FD002070BD4FF0C8
:102EE000FF30FBE76FF00500F8E700BF0070FF1F41
:102EF00000FCFF03B0F1006F10B40DD3084BD3F802
:102F0000E045084B03EA842303F10063013B984248
:102F100002D810BCFFF7A6BE4FF0FF3010BC7047C0
:102F20000070FF1F00FCFF034FF0B04382B0DA6C6B
:102F30000243DA64DB6C03400193019B02B07047EB
:102F40002DE9F04186B01422002101A82CF076FB77
:102F50000220464EFFF7E8FF0420FFF7E5FF0120BF
:102F6000FFF7E2FF04213046002205F0BDFC0022FD
:102F700010214FF0904005F0B7FC042300240125F8
:102F800002270DEB03013046CDE901354FF0100863
:102F9000CDE9034705F082FB01A93046CDE9018563
:102FA000CDE9037405F07AFB202301A93046CDE971
:102FB0000135CDE9037405F071FB01A94FF0904094
:102FC000CDE90185CDE9034405F068FB08224FF403
:102FD000881301A93046CDE901234FF00308CDE95C
:102FE000034705F05BFB4FF4441301A94FF09040F9
:102FF000CDE90183CDE9035705F050FB4FF4405371
:1030000001A93046CDE90135CDE9034805F046FB7D
:103010004FF404134021CDE901131548039501A98C
:1030200005F03CFB22460F21062004F0E1FF0620BC
:1030300005F010F822460F21072004F0D9FF0720E1
:1030400005F008F822462146092004F0D1FF0920A6
:1030500005F000F822462146092004F0C9FF0920A6
:1030600004F0F8FF06B0BDE8F08100BF000400489E
:103070000008004800B59BB04822002108A82CF0A9
:10308000DDFA1822002102A82CF0D8FA05F046FC3F
:103090004FF0B0420120D2F8903023F01803C2F86C
:1030A0009030D2F8003423F4C06343F40073C2F8C4
:1030B0000034D2F8003403F4C0630193019B24234D
:1030C000089381230B930023CDE91003B02208A8B5
:1030D000CDE9122305F09AFD08B172B6FEE74F2341
:1030E000CDE90230CDE90400CDE90600022102A8B5
:1030F00006F026F808B172B6FEE71BB05DF804FBD7
:1031000008B504F0F1FAFFF7B5FFFFF719FFFFF775
:103110004AFD00F0C7FF00F059FE00F089F80648AC
:103120000122042105F0E0FB02F046FC00F0F4FB74
:1031300002F049FCFCE700BF0004004872B6FEE75D
:1031400000B58DB02C22002101A82CF077FA174889
:10315000174B03601F2383604FF080420023C0E9B8
:103160000433C0E9072383614FF48073436206F0A0
:103170008DFA08B1FFF7E2FF0C4806F0B3FB08B187
:10318000FFF7DCFF4FF00053002207930748089237
:103190004FF4807301A9029206920B9306F0D6FABF
:1031A00008B1FFF7CBFF0DB05DF804FBD00800209D
:1031B0000028004010B5044690B03822002102A833
:1031C0002CF03CFA2268194B9A422CD14FF48033F0
:1031D000029302A84FF480730F9306F0D5F808B15C
:1031E000FFF7ACFF4FF0B0430220D3F8902042F439
:1031F0000042C3F890209A6D42F480629A659B6DFC
:10320000002203F4806311460193019B04F0F0FE59
:10321000022004F01FFF00222A20114604F0E8FEDD
:103220002A2004F017FF10B010BD00BF0028004096
:103230001148124A08B54FF48273C0E900230023F5
:103240004FF4E062C0E902324FF400712822C0E975
:1032500006120722C0E90433C0E90833C0E90B2392
:1032600083620823436306F0ADFC18B1BDE8084053
:10327000FFF764BF08BD00BFC8090020003001404F
:10328000F0B5054689B01422002103A82CF0D6F928
:103290002A68374B9A4269D14FF0B04302261A6E22
:1032A00042F480521A661A6E02F480520292029A16
:1032B000DA6C42F00102DA64DA6C02F00102019287
:1032C000019ADA6C42F00202DA64DB6C03F002036A
:1032D00000930524009B0327D02303A94FF09040BF
:1032E000CDE90336CDE9067405F0D8F92023CDE900
:1032F00003364FF09040002603A90794CDE90567F7
:103300001C4C05F0CBF91C4826620723C4E90003D6
:1033100080232046C4E90266C4E90436C4E906668F
:1033200004F0F8FE08B1FFF709FF144AAC65A56286
:10333000134C0823C4E900231021002380222046D7
:10334000C4E90213C4E90423C4E90633236204F088
:10335000E1FE08B1FFF7F2FE002222206C65114663
:10336000A56204F045FE222004F074FE09B0F0BD11
:1033700000300140680900201C000240300002407B
:10338000080900207047000008B504F0C3F9044B99
:103390000120C3F88800BDE8084005F017BB00BF56
:1033A0000004005808B504F0BCF900F08BFFFFF7EB
:1033B000C7FDFFF7F8FB00F009FDBDE80840FFF787
:1033C00037BF08B504F0ADF9FFF7BAFDFFF7EBFB27
:1033D000BDE80840FFF72CBF08B504F09BF9BDE835
:1033E00008400121002005F0A1BA70477047FEE7B0
:1033F000FEE7FEE7FEE7FEE770477047704770475D
:10340000014806F095BA00BFD0080020024B012009
:10341000187005F077BA00BF161F0020024B01227A
:1034200002201A7005F06EBA151F0020082005F062
:1034300069BA0000014804F0E3BF00BFD4130020C4
:10344000014804F0DDBF00BF68090020014804F016
:10345000D7BF00BF0809002070470000014804F0F2
:10346000CFBF00BF8814002070470000014806F05D
:103470001DBE00BFC8090020014807F09BBF00BF68
:10348000E8140020014806F087B800BFD0080020EB
:10349000014807F09CB800BFC01300202DE9F0439D
:1034A00089B080460020109E0790894615461F4629
:1034B000FCF7BEFEF0B9104CCDE90090CDE9020456
:1034C00007AB0E480593142304933A464346294616
:1034D0000068FCF777FF2346324604F1140153F8E5
:1034E000044B42F8044B8B42F9D1079B337509B06A
:1034F000BDE8F0830120FAE7420A0020486D030886
:103500007FB5124C00253C2302A86375CDE9025516
:10351000257500F0CBFA042303AA009412210C486D
:10352000FFF7BCFF0B49142220462CF077F8064623
:10353000B0FA80F040096075074B00902A46294692
:10354000022012F059F9304604B070BD2C0A002058
:10355000F26D0308DA210020D46D0308034A044801
:1035600040F21B53002107F055BD00BF560A002052
:1035700034140020312BF0B52DD81825102415FB5C
:103580000343194D00244FF0800C4CFA04F6A3F1CC
:103590001007314205EB470714BF4FF0240E4FF0E0
:1035A000140EA7F806E0A3F10807304205EB470721
:1035B00014BF4FF0240E4FF0140E0134324205EBCD
:1035C0004306A7F806E00CBF14272427082CF78031
:1035D00003F10103D9D1054B1B781BB9BDE8F040BD
:1035E000FFF7BCBFF0BD00BF560A0020801F0020BF
:1035F00010B500240022E3B2114610460134FFF753
:10360000B9FF322CF6D1BDE81040FFF7A7BF00008C
:1036100070B504460D46FFF7EBFF0F4B04EB440477
:1036200000261C44142000F09FFAA27861782078CC
:1036300012FB05F211FB05F110FB05F0F3B2D2B25B
:10364000C9B2C0B20136FFF795FF322EEAD1BDE80C
:1036500070400A2000F088BA080000202DE9F041EF
:1036600006460F462048904600214FF416622BF084
:10367000E5FF1E4A10254FF0800C2B4600244CFA23
:1036800004F1A3F110000F4202EB400014BF4FF011
:10369000240E4FF0140EA0F806E0A3F108000E422D
:1036A00002EB400014BF4FF0240E4FF0140E013413
:1036B00018EA010F02EB4301A0F806E00CBF14204A
:1036C0002420082CC88003F10103D8D11835B5F5A2
:1036D000986FD2D1064B1B781BB9BDE8F041FFF7BC
:1036E0003DBFBDE8F08100BF5C0A0020560A002003
:1036F000801F002000F00F000B4607281ED8DFE8CF
:1037000000F004070A0F1316191B0022114600E0EF
:103710000022104602E0002211461846FFF79EBF25
:103720000A4600210020F9E700220846F6E70A468B
:103730000021EEE70A46F5E70A46E7E77047000092
:10374000024B1878024B1978FFF7D4BF060000200F
:103750000000002070B55B485B4C0378DBB20A2B9D
:103760000CD8DFE803F006262A3037657A89979768
:103770009700564B1B78DBB2554A13700378554EB1
:10378000012B06D0544D2A7802F0FF03002A00F0E6
:1037900086804F4A0023137023703370FFF728FF91
:1037A0004E4A002313704E4A13704E4B01221A707A
:1037B00070BD474B00221A70E0E74B4A1278012A8D
:1037C00008BF0123D8E7494B1A78002A50D1404B53
:1037D0000122F0E7454B46491A7852B9454A12781A
:1037E000012A06D10A78012AD5B202D1384B1D70C0
:1037F000C4E71B78012B05D03E4B1B7813B10B7827
:10380000002BBBD1324B02221A703B4A1578022D95
:10381000EAB206D0032A03D0012A04D1232200E011
:10382000042222701A700A78002AA7D12322C2E744
:103830002E4B1A783AB92C4A1278012AD1B202D109
:10384000234B19709AE71B78012B03D0264B1B786A
:10385000002B93D11E4B0222ADE7244B1A781AB9E4
:10386000264A1278002AB2D01B78012BF2D0234BC3
:103870001B78012B82D1EDE71C4B1A781AB9204A2C
:103880001278042AA3D01B78012BE3D01C4B1B78A1
:10389000052BEFE71A4B1A78042AF8D197E72A7814
:1038A00012B90B4B1B78DBB22370164B20781978BA
:1038B000FFF720FF2B7803B123782378DBB2337036
:1038C0006EE700BF06010020060000200400002073
:1038D0000700002001000020801F00200E1F002094
:1038E0000D1F0020781F0020D92100200B1F002071
:1038F000090100200A010020921500200A1F002063
:10390000091F0020000000200248036800215963BD
:1039100007F0FABB34140020002270B50F4B11469B
:10392000022011F069FF01240A252946204614359A
:10393000FFF7E0FEEDB2322000F016F96E2DF4D163
:103940000134E4B2FFF754FE082CEDD10022BDE8AB
:103950007040034B1146022011F04EBF046E030865
:10396000376E0308054808B50823036006F04CFCD1
:1039700018B1BDE80840FFF7E1BB08BDC013002047
:103980004FF0B04307B55A6E42F001025A665B6EC3
:10399000002203F00103019311463220019B04F041
:1039A00027FB322003B05DF804EB04F053BB0000AA
:1039B0000CB407B5054A05AB1021019312F0EEFBDC
:1039C00003B05DF804EB02B0704700BF6D6E0308F2
:1039D00030B585B0044602A80D4612F077F9BDF95E
:1039E0000C30064A00931021029B2046FFF7E0FFAF
:1039F0002046FDF73DFD288005B030BD6D6E030803
:103A00004FF0B04210B5936823F40043936012F076
:103A100079FA104B01241C7000F0ACF811F082FE12
:103A20000D4811F099FE0D4B4FF400421A6102202F
:103A300011F098FEFFF744F800F002F911F08CFF46
:103A40002146204611F0A8FF21462046BDE810403F
:103A500011F08CBFCC130020D13900080040005871
:103A600011F0B0BF08B5FFF733F840F6B83398420D
:103A70000CD8B0F5E16F0BD3FE23A0F5E1605843FD
:103A80004FF49663B0FBF3F0C0B208BDFE20FCE734
:103A90000020FAE77FB5684600F0B6F80198FEF717
:103AA000BDFC00B207B05DF804FB0000194A38B550
:103AB000D2F88035591C044619D103F039FE054669
:103AC00003F042FE054403F039FE2B0EE3712B0C8C
:103AD000A3712B0A6371030EE370C0F30742C0F3B6
:103AE00007232571C0B2A2706370207038BD190A17
:103AF000C3718171190C1B0E41710371D2F88435A9
:103B0000C370D2F88405C0F30722C0F30743000E48
:103B1000E9E700BF0070FF1F38B5094BD3F88035C7
:103B200003600133054609D103F002FE044603F0A9
:103B300005FE444003F008FE44402C6038BD00BF41
:103B40000070FF1F0121022011F010BF0021022090
:103B500011F00CBF00207047024B187808B100F03C
:103B6000DDB97047CC13002082B00190019802B0FB
:103B700000F070BAF0B5224A224CD2F8903043F4EB
:103B8000804389B0C2F8903003F0E4FD03F0EAFD11
:103B900003F0F0FD012304930323069300254FF067
:103BA000B04305950795DA6C42F00202DA64DA6CEC
:103BB00002F002020292029ADA6C42F00202DA6425
:103BC000DB6C03F0020301934FF4805703A92046F6
:103BD000019B03974FF4005604F060FD03A92046B3
:103BE000039604F05BFD2A463946204604F07CFE2D
:103BF0002A463146204604F077FE09B0F0BD00BFEA
:103C0000000800580004004810B50446FEF77AFF8B
:103C1000074BA36040F30F20FEF7D0F9054B064A8F
:103C20002360064B6060C4E90323002010BD00BF81
:103C30000000484200007A440D093E00AB03050035
:103C4000002070470120704708B52BF059FD16235E
:103C500003604FF0FF3008BD08B52BF051FD16236F
:103C60000360FEE770B50D4614460E46731B9C427A
:103C700001DC204670BDAFF3008006F8010BF5E7CC
:103C800030B5104600234FF06042834200DB30BD68
:103C9000D2F8804EE50707D5D2F8004EE40703D5E9
:103CA000CC5C156815B114700133EEE700BFF8E77E
:103CB0004FF0FF3070474FF400534B6000207047C7
:103CC00001207047002070470B4A116810B5034669
:103CD00009B90A491160106809490A4C0344091BD3
:103CE0008B4206D92BF00CFD0C2303604FF0FF3004
:103CF00010BD1360FCE700BFD0130020204200205D
:103D0000000001200008000037B5184B02689A42F5
:103D1000054628D14FF0B043154C1A6E42F40062AC
:103D20001A661B6E134A03F400630193019B172369
:103D3000C4E90023102100238020C4E902134FF4BA
:103D40008073C4E904034FF4806C2023C4E906C3E4
:103D500020464FF40053236204F0DCF908B1FFF76A
:103D6000EDF96C62A56203B030BD00BF002C0140CC
:103D7000D41300200800024010B5044686B0142277
:103D8000002101A82BF05AFC22680F4B9A4218D14F
:103D90004FF0B04301A9DA6C42F00102DA64DB6C47
:103DA00003F0010300930222009B4FF48073CDE9DE
:103DB00001324FF090400123CDE90332059304F026
:103DC0006DFC06B010BD00BF002C014010B51022E4
:103DD0009CB0002400210DEB02002BF02FFC1C22D4
:103DE000214608A8CDE9014403942BF027FC342296
:103DF00021460FA82BF022FC2B482C4B8460C0E9F5
:103E000000343B23C0E90334C0E9054406F048FE12
:103E100008B1FFF793F94FF480532348049304A9A2
:103E200006F05CFF08B1FFF789F91F4806F068FE4D
:103E300008B1FFF783F900241B48039401A9CDE9D9
:103E4000014407F063F908B1FFF778F960231648D9
:103E50000E94002208A9CDE90834CDE90A44CDE941
:103E60000C4406F0B5FE08B1FFF768F900234FF4E3
:103E70000052CDE914230C4813934FF000720FA9A0
:103E8000CDE90F33CDE91133CDE91633CDE9182350
:103E9000CDE91A3307F066F908B1FFF74FF9024888
:103EA000FFF76AFF1CB010BD34140020002C014045
:103EB000014B1868704700BF801400200320704732
:103EC00008B501464FF47A7200238002890DFEF78F
:103ED000EBFA08BD4FF47A73A0FB0303800A40EAB3
:103EE00083507047034B98689A689042FBD1C04357
:103EF000704700BF0028004008B5FFF7F3FF014BF3
:103F0000186008BD8014002008B5FFF7EBFF024BD6
:103F10001B68C01A08BD00BF80140020024B18782F
:103F200008B1FFF7DFBF70478414002010B5074BBE
:103F3000074C0122DA654FF48071204605F0F2FA51
:103F40004FF0FF332363002010BD00BF0028004066
:103F5000D008002002460021014805F0FABC00BF4D
:103F6000D008002002460121014805F0F2BC00BF44
:103F7000D008002010B58CB02C220021044601A8E6
:103F80002BF05CFBFFF7D2FF0C4B0D481B681C4469
:103F90000023089306934FF00053E4430793012254
:103FA0004FF4807301A902940B9305F0CFFB08B185
:103FB000FFF7C4F800200CB010BD00BF8014002033
:103FC000D008002038B50546FFF78CFF02210446D3
:103FD000074805F0C5FCC4F309024FF47A71A2FB4F
:103FE0000121920AA30A2A8043EA805038BD00BF0B
:103FF000D00800200148002105F0B2BCD008002004
:104000000148012105F0ACBCD0080020F8B50F4DE7
:104010002E78CEB90E4C4FF0FF372763FFF790F89C
:10402000FFF784FF4FF48071204605F07BFA2046AD
:10403000276305F039FC32462046022105F089FC51
:10404000FFF75AFF01232B700020F8BD84140020D5
:10405000D0080020014610B54FF47A720023800288
:10406000890DFEF721FA0146FFF73CFF0446FFF7F2
:1040700039FF031B8B4200D310BD00BFF7E712F0DE
:1040800049B8000010B5064C0221204605F068FC36
:104090000221421C2046BDE8104005F05ABC00BF7A
:1040A000D00800201648174A08B54FF4E133C0E99C
:1040B000002300230C22C0E90233C0E90523C0E934
:1040C0000733C0E90933036107F059FF08B1FFF76F
:1040D00035F80B48002108F0CAF808B1FFF72EF8B0
:1040E0000748002108F0E3F808B1FFF727F8044873
:1040F00008F09DF818B1BDE80840FFF71FB808BDEB
:10410000E81400200044004070B596B00646142222
:10411000002103A82BF092FA3822002108A82BF0E6
:104120008DFA3268274B9A424AD10223089308A895
:104130004FF440230A9305F027F908B1FEF7FEFF7C
:104140004FF0B04300259A6D1F4C42F400329A653F
:104150009A6D02F400320292029ADA6C42F0010285
:10416000DA64DB6C03F001030193019B0C22022350
:10417000CDE9032303A907234FF090400793CDE92E
:10418000055504F08BFA114925621423C4E9001384
:104190001023C4E9023520468023C4E90435C4E96C
:1041A000065503F0B7FF08B1FEF7C8FF2520F467F6
:1041B00000220221A66203F01BFF252003F04AFF24
:1041C00016B070BD004400408814002080000240FA
:1041D00002680C4B9A4210B5044612D14FF0B0421F
:1041E0000C21936D23F4003393654FF0904004F05D
:1041F00001FBE06F04F000F8BDE81040252003F05B
:1042000037BF10BD0044004008B50A4601460248C9
:1042100007F034F8002008BDE814002013B5114B56
:10422000114C18604FF40013009302AB13E9060021
:10423000204607F0A0FF2368DA69D103FCD4DA69CD
:104240005202FCD59A68084842F480029A6007F04E
:10425000D8FF06490448012207F046FF002002B0BB
:1042600010BD00BF7C150020E8140020841500203C
:1042700008B5074B1860FEF796FCFFF713FF054AD9
:10428000D2F8803043F00063C2F88030002008BDCF
:10429000801500200008005808B54FF0B0430848CA
:1042A0009A6B42F400329A639A6B22F400329A635A
:1042B000FFF78EFF112003F0DBFE002008BD00BFDA
:1042C000E814002008B5074807F059FE08B1FEF7CA
:1042D00035FF054803F01EFF18B1BDE80840FEF7A2
:1042E0002DBF08BDE8140020881400200268044B8C
:1042F0009A4203D1034B00201B681847704700BF48
:10430000004400408015002002680B4B9A4210B513
:1043100004460FD1094B1B682BB1D0F8902012B97D
:1043200007480121984720460549BDE81040012271
:1043300007F0DABE10BD00BF004400407C1500202D
:10434000841500202DE9F04F9DB0FEF7BBFA14F064
:1043500089FB024640B90146644B022011F04CFA39
:1043600001201DB0BDE8F08F012014F023FC13F0F4
:104370001FF90446039040B9024601465C4B0220F7
:1043800011F03AFA14F0E2FBEAE75A4D296813F00B
:104390005FFD6968204613F075FD297A204613F009
:1043A000A5FD697A204613F0D5FD6969204613F012
:1043B00061FEE868FEF758F881B2204613F0E4FD8C
:1043C0002969204613F0ACFDA97A204613F074FD4C
:1043D0000221204613F026FE1021204613F064FE31
:1043E000039813F06DF90246049040B90146424B20
:1043F000022011F001FA03A813F03AF9C2E703A86A
:1044000013F036F9049813F0C3FC024640B9014694
:104410003A4B022011F0F0F904A813F06FFAB1E75B
:10442000374EDFF8E0A0DFF8E0B0002333604FF054
:104430000208049805AB0A2208A913F09BFA054666
:1044400028BB02460146314B022011F0D5F93068F5
:104450002C49FDF707FE4FF07C51FDF703FE30605D
:10446000049813F0C5FC044604A813F047FA14F0AE
:104470006DFB002C3FF474AF002D3FF471AF0022B0
:10448000234B1146032011F0B7F9002069E731688A
:104490000998FDF7DFFCBDF81890306000221D4B35
:1044A000CDF800901146022011F0A6F908AC0027C3
:1044B000BBB2994504F1080405D8B8F1010FC6D084
:1044C0004FF00108B5E754F8040C5146FDF7CAFD5A
:1044D000FDF7CAFF019034F8083C009300225B46C8
:1044E0001146022011F088F90137E1E7C86E030890
:1044F000E06E030820000020156F03083C6F0308DE
:10450000181F002000007A449F6F0308656F03089E
:10451000B66F03088E6F030830B5044685B00846B1
:1045200014491546FDF79EFDFDF778FFCCB1114902
:1045300002902846FDF796FDFDF770FF0E490190A9
:104540002846FDF785FC0D49FDF740FEFDF78CFF81
:10455000002200900A4B1146032011F04DF905B0DE
:1045600030BD0090074B22462146032011F044F94C
:10457000F5E700BF00007A44CDCC4C3FCDCCCC3E1B
:10458000CF6F0308FC6F03082DE9F04FADF2344DF7
:104590004FF4007200210CA82BF050F84FF4007279
:1045A00000218CA8B34E2BF049F8002537464FF078
:1045B00000082C46B9682046FDF74CFC7968044693
:1045C0002846FDF747FC08F10408B8F5007F0546CA
:1045D00007F11007EED14FF070512046FDF742FD74
:1045E0004FF0705104462846FDF73CFD0025DFF8EA
:1045F000848207464FF00009AA46D8F808002146F1
:10460000FDF726FC0146FDF72DFD01465046FDF75E
:1046100021FC39468246D8F80400FDF719FC014612
:10462000FDF720FD01462846FDF714FC09F10409B9
:10463000B9F5007F054608F11008DED14FF0705142
:104640005046FDF70FFD4FF070510A902846FDF7D8
:1046500009FD82460A98FDF777F8874B00222CF077
:1046600063FFCDE904015046FDF76EF8824B00224E
:104670002CF05AFFFDF798FB0DF130090546C846AE
:1046800000234FF0000BB168B0690693FDF7E0FB23
:10469000FDF7C4FE0028B8BF4042FDF78FFC48F884
:1046A000040B01465846FDF7D5FB069B0433B3F5D2
:1046B000FE7F834606F11006E5D17049FDF786FDC1
:1046C0000DF13008064600234FF0000B314658F834
:1046D000040B0693FDF7BCFB0146FDF7C3FC069BEC
:1046E00001461846FDF7B6FB0BF1010B1FFA8BFBD9
:1046F000BBF17F0F0346E9D16049FDF767FDFDF788
:1047000023F85D4B00222CF00FFFCDE906010DF5DB
:104710000C78C346002200234846D9F800104068B0
:104720000B930892FDF794FBFDF778FE0028B8BFC5
:104730004042FDF743FC089A4BF8040B0146104633
:10474000FDF788FB0B9B01339BB27E2B09F104091B
:104750000246E1D14A49FDF739FD4FF0000B814691
:104760000023494658F8040B0893FDF771FB0146F6
:10477000FDF778FC089B01461846FDF76BFB0BF133
:10478000010B1FFA8BFBBBF17E0F0346E9D13C49BD
:10479000FDF71CFDFCF7D8FF374B00222CF0C4FEC0
:1047A000CDE9080137492846FDF75CFCFDF736FEE8
:1047B000344902905046FDF755FCFDF72FFE314974
:1047C00001903846FDF74EFCFDF728FE00222E4BE7
:1047D00000901146022011F00FF82C4A13889BB26A
:1047E000FA2B00F2D580108880B2FDF7E7FB29464E
:1047F000FDF7EAFD264F08B105233B70254B1A78DB
:10480000254B1B889BB29A4280F08D80234B1A78EF
:10481000234B1B889BB29A4206D222492046FDF7C1
:10482000DDFD08B101233B701F4FDFF880A03B88FE
:104830000A9A01339BB23B803B889BB20A2B04BF90
:1048400000233B803B884FF01C0B9BB20BFB03F318
:10485000DDE904014AF803403B889BB20BFB03A34C
:104860005A603B889BB20BFB03A8FDF79DFA3B887F
:104870001EE000BFAC1600200000E03F0000FE423A
:104880000000FC4200007A44127003083C00002043
:1048900092150020A70300208A150020A6030020FF
:1048A00088150020CDCC4C3FAC1E00209415002074
:1048B000C8F808009BB20BFB03A34FF08641DD60F4
:1048C0003D883046FDF7CEFBADB20BFB05A5286158
:1048D0003D88DDE90601FDF767FA4FF08641FDF7F7
:1048E000C1FBADB23B880BFB05A59BB26861334DA4
:1048F0000BFB03AA2A788AF81820DDE90801FDF7E6
:1049000053FA4FF08641FDF7ADFBFDF7ADFD2C4BA3
:10491000C0B218802B78012B05D10022294B1146FB
:10492000022010F069FF284F244D3B78DFF89C806F
:10493000012B24D1DFF89890264EB9F80030B9F851
:1049400000204FF01C0A9BB292B20AFB03F30AFB51
:104950000262F0589168FDF77DFA2146FDF73EFDB1
:10496000C0B102232B702B78022BD8B204D10022C5
:10497000194B114610F040FF2B78DBB23B702B78BF
:10498000DBB23B70C8F800400DF2344DBDE8F08F4B
:1049900012482CE7B9F80030D8F800909BB20AFB17
:1049A00003662046B168FDF755FA4946FDF716FD46
:1049B00010B103232B70E2E72870E0E79215002086
:1049C0008615002058700308901500208C150020D3
:1049D000AC1E0020941500209D70030800007A434F
:1049E0002DE9F04F9FB0FDF76DFF14F03BF8024644
:1049F00040B90146A84B032010F0FEFE01201FB075
:104A0000BDE8F08F012014F0D5F811F0E9FC044660
:104A10000D9040B902460146A04B032010F0ECFE79
:104A200014F094F8EAE79E4F3B78012BDDB252D0A8
:104A3000022D6FD0002D39D1042112F097F80121F9
:104A4000204611F0C1FF9749204611F0F1FF964929
:104A5000204611F0D3FF9549204611F081FF94497B
:104A6000204611F097FF0221204612F0B3F8914939
:104A7000204612F095F8214606A811F0F3FF8E4A61
:104A800019928E4A1A924FF07C53002218A92046A0
:104A900018931B921C921D9312F010F82946204681
:104AA00012F030F80321204612F046F80D98002449
:104AB0003C7011F02BFD02460E9000286DD1804B0A
:104AC0000146032010F098FE0DA811F0F7FC0EA887
:104AD00011F0AAFDA4E77B4E294611F075FF71493C
:104AE000204611F0A5FFB168204611F039FFF168AA
:104AF000204611F04FFF716A204611F07FFFF16CE4
:104B0000204612F04DF8704B00221146012010F0A3
:104B100073FECBE76B4D012111F056FFE96920468A
:104B200011F086FF696A204611F068FFA9682046E7
:104B300011F016FFE968204611F02CFFA86CFDF774
:104B400093FC81B2204612F045F8E96C204612F041
:104B500027F8214606A811F085FF2B6B18936B6B85
:104B60001993AB6B1A93EB6B1B932B6C1C9318A9CB
:104B70006B6C1D93204611F0A1FFA86AFDF774FC31
:104B8000C1B2204611F0BEFF286AFDF76DFCC1B22C
:104B9000204612F039F84D4BB6E711F0DBFD38B97D
:104BA00000224B4B1146032010F026FE002026E782
:104BB0001422214613A82AF041FD0026DFF8EC80DC
:104BC000DFF81091DFF810A1212537460E980FA9C4
:104BD00011F018FE0246002840F08A8001463F4B43
:104BE000032010F009FEDFF8F8800E9811F0D2FDD6
:104BF000B8F8003000229BB2114600930320394BD5
:104C000010F0FAFD0D9D0121284611F0DDFE042172
:104C1000284611F0ABFF2349284611F009FF22492D
:104C2000284611F0EBFE2149284611F099FE204953
:104C3000284611F0AFFE0221284611F0CBFF1D4996
:104C4000284611F0ADFF294606A811F00BFF1A4ABD
:104C50001992254A1B924FF07C534FF07E5218A9AF
:104C600028461C9218931A931D9311F027FF0021D8
:104C7000284611F047FF0321284611F05DFF0D99EA
:104C80000EA811F0FBFC0246002840F0848001468B
:104C9000164B022016E700BFC86E0308E270030837
:104CA000141F0020000082429A99993FCDCC4C3FBE
:104CB000000020406666263F000020410AD7233CC2
:104CC00064710308B01E00200271030832710308EA
:104CD0007F710308CDCCCC3EA40300209D71030856
:104CE000AE1E0020C6710308CDCC4C3EFB710308FC
:104CF000119A10999DF83C00FFF70EFC9DF83C308E
:104D0000FBB1DDF844B038465946FDF7A3F81099D9
:104D100007463046FDF79EF8414606465846FDF7E1
:104D200097F84946FDF752FAFDF79EFB1EAB80B29D
:104D300003EB4000013430F82C3C0133E4B220F89E
:104D40002C3C9AF80030012B1ED1DFF81CB2874AA8
:104D5000BBF8003011999BB202EB03139960BBF8CA
:104D600000309BB202EB0312109B5360BBF8003083
:104D70009BB25A1C92B2802BABF8002004D1FFF7F3
:104D800003FC0023ABF800300F20FDF713FE013DBC
:104D90007FF41CAF27E70E9811F0DCFC00283FF4ED
:104DA000FFAE0DA811F08AFBDFF8C4B14FF0210966
:104DB0000E980FA911F026FD054600287ED1024667
:104DC00001466C4B032010F017FDB8F80030DFF8F7
:104DD000A891DFF8A8B100229BB2114600930320EE
:104DE000674B10F009FD012C94BF0023012389F8C3
:104DF000003000F0CBFD99F800300022CDE90043EF
:104E00001146604B032010F0F7FC0DF14C084FF0F9
:104E1000000A38F8022B3AB1CDE900A200225B4625
:104E20001146012010F0E8FC0AF1010ABAF10A0F5C
:104E3000EFD155493846FDF715F907462046FDF7ED
:104E4000BDF8804601463846FDF7C0F94E49074691
:104E50003046FDF707F94146FDF7B8F94B4B1F60A7
:104E60004B4B002118608046FDF790FA0646A8B922
:104E70004223404699F80090CDE90343FDF7CEFA6E
:104E800002903846FDF7CAFA5FFA89F9CDE9009039
:104E9000404B32463146032010F0AEFC0E9811F024
:104EA00079FC04460EA811F0BFFB13F04FFE002C56
:104EB0003FF4A4AD85F00100C0B2A0E5119A1099AD
:104EC0009DF83C00FFF728FB9DF84930002B43D1AB
:104ED0009DF83C30FBB1DDF844A038465146FCF764
:104EE000B9FF109907463046FCF7B4FF2A49064639
:104EF0005046FCF7ADFF5946FDF768F9FDF7B4FAE7
:104F00001EAB80B203EB4000013430F82C3C01337F
:104F1000E4B220F82C3C214B1B78012B1CD1B8F8B3
:104F20000030124A11999BB202EB03139960B8F852
:104F300000309BB202EB0312109B5360B8F80030B4
:104F40009BB25A1C92B2802BA8F8002004D1FFF724
:104F50001BFB0023A8F800300F20FDF72BFDB9F153
:104F600001097FF425AF30E7AE1E0020AC1600200B
:104F7000CDCCCC3E9D7103080B1F00207A72030834
:104F80001B7203084672030800007A44041F0020C5
:104F9000001F00209A720308CDCC4C3FA4030020D0
:104FA0002DE9F043ADB014230DF10E0204A9ADF8C4
:104FB0000E3013F0DFFF044648B902460146194B94
:104FC000032010F019FC20462DB0BDE8F08300222C
:104FD000154B164FDFF85880DFF858901146032024
:104FE00010F00AFC0025BDF80E30AAB29342EAD9AF
:104FF000AAB22CAB03EBC202032012F89C6C52F84D
:10500000A03C002E14BF3A464246CDE900320022B1
:105010004B46114610F0F0FB002E05F1010508BFCC
:105020003446E0E7F472030817730308EA720308D2
:10503000EF7203083B73030830B5102289B00025D6
:10504000294604460DEB020003952AF0F7FA15F005
:105050003BFB2A46A34B00902946032010F0CCFBD3
:10506000FDF730FC13F0FEFC8DF80C0013F0A4FDEE
:10507000431B18BF012301218DF80D30029013F05E
:10508000B9FD029813F058FF029813F0CDFD029875
:10509000FFF786FF002840F0008102A813F09CFD76
:1050A00013F054FD029813F0DBFD029813F0F4FDA9
:1050B0000298FFF775FF002840F0F38002A813F074
:1050C0008BFD13F043FD029813F002FE0022864B85
:1050D0001146032010F090FB029813F015FE029881
:1050E000FFF75EFF002840F0E08002A813F074FD97
:1050F00013F02CFD029813F023FE002211467B4B87
:10510000032010F079FB0022794B1146032010F0A8
:1051100073FB029813F0A0FE0298FFF741FF0028EE
:1051200040F0C78002A813F057FD13F00FFD02985E
:1051300013F0AEFE002211466E4B032010F05CFB14
:1051400000226D4B1146032010F056FB029813F01D
:10515000BBFE0298FFF724FF002840F0AE8002A8B3
:1051600013F03AFD13F0F2FC029813F0C9FE00228E
:105170001146624B032010F03FFB0022604B1146AA
:10518000032010F039FB029813F0F6FD0298FFF7A8
:1051900007FF002840F0958002A813F01DFD13F0D2
:1051A000D5FC029813F004FE00221146554B032053
:1051B00010F022FB0022544B1146032010F01CFB80
:1051C000029813F011FE0298FFF7EAFE00287CD146
:1051D00002A813F001FD13F0B9FC029813F020FEB1
:1051E00000221146494B032010F006FB0022404BE1
:1051F0001146032010F000FB029813F02DFE0298D8
:10520000FFF7CEFE002864D102A813F0E5FC13F0EE
:105210009DFC029813F03CFE00221146354B032002
:1052200010F0EAFA0022344B1146032010F0E4FAA1
:10523000029813F049FE0298FFF7B2FE00284CD105
:1052400002A813F0C9FC13F081FC029813F058FE79
:1052500000221146294B032010F0CEFA00221146FD
:105260002B4B032010F0C8FA01238DF8173003AB45
:1052700003CB00222060186861600C23A0601146F7
:1052800000930320234B10F0B7FA02A813F0A4FCFC
:1052900013F05CFC002009B030BD01238DF80E3006
:1052A00000E701238DF80F300DE701238DF8103052
:1052B00020E701238DF8113039E701238DF81230F2
:1052C00052E701238DF813306BE701238DF814307A
:1052D00083E701238DF815309BE701238DF8163005
:1052E000B3E700BF517303087A730308AD73030873
:1052F000DE7303080D7403083A7403086F7403081F
:10530000A2740308D57403080675030836750308EC
:10531000647503089175030802480122102103F007
:10532000E3BA00BF0004004802480022102103F045
:10533000DBBA00BF0004004813B5134C23785BB9F7
:10534000E37C03F0FF023BB9104B1146022002B090
:10535000BDE8104010F050BAFEF7D2F800380C4B00
:1053600018BF0120400018701A78022A02BF0022DC
:105370002270E2741B7800930022064B1146032032
:1053800010F03AFA02B010BDDA210020B07503081F
:10539000801F0020CC75030838B5184C23785BBB00
:1053A000E37C03F0FF023BBB154D2B68012B0CD9AE
:1053B0002B68042B09D81146124B022010F01CFA5E
:1053C000114A0421012000F0A3FF2B68042B13D9FC
:1053D00000220E4B1146022010F00EFAFEF790F854
:1053E00000380B4B18BF0120400018701B78022BAF
:1053F00002BF00232370E37438BD00BFDA21002010
:105400007C1F0020E3750308087603080D76030867
:10541000801F002010B5124C237863B101214FF09A
:10542000904003F05BFA0F4B0022187022701B783B
:105430000D4ADBB213700D4C237863B102214FF09B
:10544000904003F04BFA0A4B0022187022701B7830
:10545000084ADBB21370BDE81040FEF77BB900BF0D
:10546000161F00200A01002008010020151F00203F
:10547000090100200701002010B5164B1A78022AF6
:1054800026D91B78072B23D8FFF7AAFA1248134A0C
:10549000037811785B1A124918BF01230B70037847
:1054A0001048DBB21370104B104A1C780378E31AD3
:1054B00018BF012313700E4B04701B7823B1002317
:1054C0000B700C490B701370BDE81040FEF742B929
:1054D00010BD00BF060100200B1F0020081F002088
:1054E0000C1F00209015002092150020911500201F
:1054F000801F00200E1F002008B501214FF09040B2
:1055000003F0ECF9064B012816BF022218701A703E
:105510001878044B1978BDE80840FEF779B800BF49
:10552000060000200000002038B5324D324C287BA8
:10553000FCF740FD3149FCF795FDA060687BFCF766
:1055400039FD2E49FCF78EFDE060A87BFCF732FDAB
:105550002A49FCF787FD6062E87BFCF72BFD2849B0
:10556000FCF780FD274BE0642361287CFCF722FDDB
:105570006060687CFCF71EFDA061A87CFCF71AFD4A
:10558000E061E87CFCF716FD2062287DFCF712FD47
:10559000A062687DFCF712FD1849FCF763FD2063EB
:1055A000A87DFCF707FD6063E87DFCF707FD144963
:1055B000FCF758FDA063287EFCF7FCFCE063687EE6
:1055C000FCF7FCFC0D49FCF74DFD2064A87EFCF7C0
:1055D000F5FC0A49FCF746FD6064E87EFCF7EAFC4E
:1055E000A064287FFCF7E6FC074BE06202221A70F9
:1055F00038BD00BF58030020B01E0020CDCCCC3DEC
:105600000AD7233CCDCCCC3E141F002038B5114D19
:10561000114C287BFCF7D2FC1049FCF723FDA0605D
:10562000687BFCF7CBFC0D49FCF71CFDE060A87B18
:10563000FCF7C4FC0949FCF715FD6062E87BFCF748
:10564000BDFC0749FCF70EFD064BE06401221A7011
:1056500038BD00BF58030020B01E0020CDCCCC3D8B
:105660000AD7233C141F002073B52F4D2F4E2B78E3
:1056700003702F4B1B784370044601214FF090407C
:1056800003F02CF93378A070E37002214FF09040C2
:1056900003F024F9274B20711B7863713378012BB9
:1056A0003ED1254B1868FCF7DFFE244BE0801868DC
:1056B000FCF7DAFE80B2224BA0831B78191F4A4206
:1056C0004A41A2771F4A92F82B1084F82B10D26A15
:1056D000E262012B84F828300FD11B4B009300228B
:1056E0001A4B1146022010F087F8194B1B8884F8DA
:1056F0002930184B1B8884F82A30174B1B7853B17C
:10570000164B1B683BB1164B1B78012B01BF154A8A
:10571000232313702B70144B01221A7002B070BD3A
:105720000020E080C7E700BF060000200B1F00201C
:10573000060100200A1F0020041F0020001F002077
:10574000921500201C1F0020520000204076030804
:105750008A15002086150020A5030020101F0020B8
:10576000D721002007000020781F0020024B0122D3
:105770000021032010F040B86E76030808B501221E
:10578000074B0021032010F037F8FFF7C5FDFFF7A6
:10579000CBFE044A00231370034A137008BD00BFF8
:1057A000B4760308141F0020D521002010B5134B38
:1057B00001220021022010F01FF8114B04225A7020
:1057C0000024012263211A7083F8331083F83420F7
:1057D0009C63DC631C645C649C64DC641C655C65C9
:1057E00083F82B40DC625C629C77FFF795FDFFF746
:1057F000BDFFFFF7C3FF034B1C7010BDEA76030823
:105800001C1F0020D52100201FB5114B11491C6819
:1058100058681A7A5B7ACDE90223FCF723FCFCF77F
:1058200023FE0C4901902046FCF71CFCFCF71CFEF3
:105830000022094B0090114603200FF0DDFFFEF718
:1058400081FD642004B0BDE81040FEF78DB900BFB3
:105850002000002000007A44217703082DE9F04160
:1058600086B00D460446FFF757FD01F03DFFFDF7FA
:1058700067FB9620FEF778F9154F00264FF00508D4
:10588000AE420FD14FF47A70FEF76EF901AB03CB45
:105890001B8823810F4B2060002261601A7006B0C4
:1058A000BDE8F081FEF738F887F80080FDF748FF83
:1058B0004FF47A70FEF758F901A8FFF7BDFB41F2EB
:1058C0008830FEF751F90136FFF79EFFD8E700BF99
:1058D00006000020D521002030B585B00446002503
:1058E00003A8ADF80C50FCF7F1FF70B19DF80C3037
:1058F0009DF80D20237062702946CDE90032032007
:10590000034B2A460FF078FF012005B030BD00BFE1
:1059100056770308022801D8FFF7FEBC704702281B
:1059200001D8FFF701BD7047022803D802481021B3
:1059300002F0DFBF704700BF0004004807B56846AB
:1059400010F0EAF9054B1B782BB9054A009B9363CD
:10595000916B5B1AD36303B05DF804FB0300002076
:105960001C1F002007B5684610F0D6F9054B1B78C0
:105970002BB9054A009B1364116C5B1A536403B086
:105980005DF804FB020000201C1F002007B56846DC
:1059900010F0C2F9064B1B78012B05D1054A009B7C
:1059A0009364916C5B1AD36403B05DF804FB00BF91
:1059B0000B1F00201C1F002008B5FEF721F8BDE8D2
:1059C000084000F009BF4FF0FF3010F05FB870479B
:1059D000014B01221A707047E41F0020014BD87060
:1059E000704700BF18010020014B1874704700BFBA
:1059F0001801002007B5064B00221B5C00931146DE
:105A0000044B02200FF0F8FE03B05DF804FB00BF6A
:105A1000957703087B77030808B5002102200FF073
:105A2000FDFF0A4B1B7803F0FF014BB9084B1A68C6
:105A3000042A05D81A68102001321A600FF0EEFF10
:105A4000BDE80840034810F013BB00BFDA21002076
:105A50007C1F00203C210020002101200FF0DEBF30
:105A600013B5104A104C42F21073002818BF0346B9
:105A70000E482360136010F0ADFA21680B4810F057
:105A800031FB0A4810F0F4FA23684FF47A72B3FB42
:105A9000F2F3002200931146054B01200FF0ACFEFB
:105AA00002B010BD9C030020140100203C21002006
:105AB0009977030813B50D4C206023680BB90C4B84
:105AC00023600C4810F086FA21680A4810F00AFB9F
:105AD000084810F0CDFA236800930022064B1146C7
:105AE00003200FF089FE02B010BD00BF9C03002010
:105AF000A0860100841F0020C577030813B50F4C52
:105B00002060236813B942F2107323600C4810F030
:105B100061FA21680A4810F0E5FA094810F0A8FA7D
:105B200023684FF47A72B3FBF2F30022009311461C
:105B3000044B01200FF060FE02B010BDA003002056
:105B40009C1F00200178030837B5044600283DD08B
:105B500090F90650002D46D1264810F03BFAFDF78B
:105B600047FD254B01221A70FDF7F8FC2A4629460D
:105B7000224B02200FF040FEE379012B0CBF204B9B
:105B8000204B2A46294602201F4D0FF035FEE379AF
:105B90002B701E4B1868FFF78DFF29781C4A1D4B90
:105BA000012908BF13460022009311461A4B012019
:105BB0000FF022FE94F90530019394F9043000931C
:105BC0000022164B114603200FF016FE144B012243
:105BD000002102201A700FF021FF124803B0BDE827
:105BE000304010F045BA00220F4B114602200FF052
:105BF00003FEDFE7E81F00200600002043780308CB
:105C00005878030875780308D62100209C030020EB
:105C10003A7803083E78030892780308CA780308A4
:105C2000D4210020CC1F0020B17803080A46014986
:105C3000FDF740B900F0030870B5164810F0CAF936
:105C400006F096FF044650B10022134B1146022085
:105C50000FF0D2FDBDE87040104810F009BA104DA9
:105C6000104B0246014602200FF0C6FD01260E4BE6
:105C70002E702246214602200FF0BEFD0B4806F092
:105C80000BFE2878314606F05FFB024810F0F0F971
:105C9000E0E700BF3C210020F37803082421002026
:105CA0007C010020117903082579030818010020E0
:105CB000F0B5A3B0FDF7D6FE054606F03FFC07465B
:105CC000002843D1704C0BA8FFF7CEFC13232370A0
:105CD0006E4B1A7802F0FF06002A48D01F7014237A
:105CE00023706B4B62681B7863F07F0313706368EB
:105CF00028B200EB400000EB4010FE22B0FBF2F0B7
:105D000058700223634A1278012A88BF0023637007
:105D1000614B1B780BB907F04DF9604C637A33B1D6
:105D200006F0F8FB012802D1204610F053F95C4B35
:105D30005548D978002206F017FC0146002840F0AB
:105D40008E800122574B10460FF056FD0024564816
:105D500010F040F9554B54481968A14238BF21460C
:105D600010F0C0F9504810F083F923B0F0BD504A4C
:105D7000117801F0FF030029C4D0454B16701B7841
:105D8000626863F07F03137063689DF82C505D7048
:105D900062689DF82D30937062689DF82E10D17066
:105DA00062689DF82F10117162689DF83010517172
:105DB00062689DF831109171BDF832206168120A55
:105DC000CA716068BDF832200272BDF84820120A1C
:105DD0004272BDF8482082729DF84A20C2729DF836
:105DE000542002739DF857204273169A120A827348
:105DF000169AC27303EB83032E4A03EB8303134407
:105E000001932D4B05EB850503EB450300933246CB
:105E10002A4B314601200FF0EFFC9DF854300893D7
:105E2000149B07939DF84A300693BDF848300593BC
:105E3000BDF8323004939DF8313003939DF8303033
:105E400002939DF82F3001939DF82E300093324637
:105E50001B4B314601200FF0CFFC102352E70631D7
:105E60007FF474AF06F050FB044600283FF46EAF99
:105E700001224FF47A730021B0FBF3F31046009334
:105E8000104B0FF0B9FC62E70C010020D421002078
:105E900030200020801F0020E41F0020E81F002089
:105EA00018010020797A03083C2100201401002009
:105EB000781F00207D010020F402002044790308AF
:105EC0006C790308887A030813B568460FF024FF3D
:105ED000164B009A1978164B11B9996B511AD96360
:105EE0001448DC6B01788C4281BF012183F82B10B0
:105EF000D96BD9621049097811B9196C511A5964D2
:105F00000E490978012902BF996C521ADA64D96CDA
:105F10000278914205D9012283F83220DA6C92B2DC
:105F20001A86074B1B7802B010BD00BF030000208B
:105F30001C1F0020A5030020020000200B1F0020D2
:105F40009215002000B503468DB000282CD0407873
:105F500002280AD003282AD0164B0022114602201C
:105F60000DB05DF804EB0FF047BC1A7F0B92DA7EA0
:105F70000A929A7E09925A7E08921A7E0792DA7DD8
:105F800006929A7D05925A680492DA68039293F910
:105F900014200292B3F9122001921B7C009300227C
:105FA000054B11460FF028FC0DB05DF804FB034BC8
:105FB000D3E700BFA67A0308BD7A03082F7B030846
:105FC00001284FF000020CBF024B034B1146022088
:105FD0000FF012BC4E7B0308607B03081FB504461C
:105FE000002831D00378002B2ED01D4810F040F847
:105FF000002211461B4B02200FF0FEFB94F91830D3
:10600000039394F90A300293237C0193E36800938D
:1060100000221146144B03200FF0EEFB0022134B1D
:10602000114603200FF0E8FB237A012B0ED1617A91
:106030000F4A104B002918BF134600220093114647
:106040000D4B03200FF0D8FB04B010BD00220B4B0A
:106050001146032004B0BDE810400FF0CDBB00BFD7
:1060600018200020797B0308AA7B0308DB7B030848
:10607000757B0308747B0308E87B0308F97B03083E
:1060800008B5104B0122002102201A700FF0C6FC47
:106090000D480FF0EDFF0D4B1B788BB10C4B1A78B0
:1060A00072B9DB7C63B90B4B1A68042A9EBF1A686D
:1060B00001321A600021BDE8084010200FF0AEBC8C
:1060C00008BD00BFD4210020841F0020D62100205D
:1060D000DA2100207C1F002008B5002140200FF0AD
:1060E0009DFC074B1B7853B1064B1A78012A06D149
:1060F00000211970BDE8084002200FF08FBC08BDD8
:10610000D62100200C1F0020044B1B78022B03D14A
:10611000002108200FF082BC704700BF7C010020E6
:10612000044B1B78012B03D0002180200FF076BC9C
:10613000704700BF0601002008B506F022FD80B9B7
:1061400006F0E8F901280CD1BFF34F8F0549064B43
:10615000CA6802F4E0621343CB60BFF34F8F00BF05
:10616000FDE708BD00ED00E00400FA0538B504467F
:106170000D4607484FF40061FCF7BCFE30B92A46D3
:1061800021460348BDE83840FCF7BABD38BD00BF22
:1061900000F0030810B506F09FFD10F1080F07D1BD
:1061A000064B0022BDE81040114602200FF024BB30
:1061B000013001D1024BF4E710BD00BF077C03089A
:1061C0001D7C030838B5104C237822781809D2B208
:1061D0000CD10E4D2A7823789A4206D020781E21C1
:1061E000FDF788FA2378DBB22B7038BD084C237892
:1061F0001E2133B1FDF77EFA237883F0010323706B
:10620000F3E702F00F00F5E706000020D821002098
:106210009803002070470000022837B5044636D0A6
:1062200040285CD001285DD12F4B1B78002B59D022
:10623000FA20FDF799FC21464FF0904002F04EFB0A
:106240002A4B214618704FF0904002F047FB214640
:1062500005464FF0904002F041FB254A254B0028AF
:1062600008BF13460022CDE900531146224B0220FD
:106270000FF0C2FAFFF762FB002120200FF0CEFBE7
:106280000021022003B0BDE830400FF0C7BB1B4B1C
:106290001B783BB3FA20FDF767FC21464FF0904096
:1062A00002F01CFB164B214618704FF0904002F094
:1062B00015FB214605464FF0904002F00FFB114AB6
:1062C000114B002808BF13460022CDE900531146A8
:1062D0000E4B20460FF090FAFFF744FBCCE700216D
:1062E0000420CFE703B030BD161F002003000020BC
:1062F000357C0308417C0308677C0308151F0020D8
:10630000020000204D7C03085A7C03088D7C0308A2
:1063100073B505460C46164606F010F903460028EC
:1063200040D000242A480FF055FE2A4B284819680F
:10633000A14238BF21460FF0D5FE254802B0BDE886
:1063400070400FF095BE4A68F05CD0540133DAB269
:106350009442F8D8204B0D701A781B78012A88BF18
:1063600000244C700022CDE900341C4C1C4B11461B
:1063700001200FF041FA637A33B106F0CBF801281F
:1063800002D120460FF026FE164B1748D97800227E
:1063900006F0EAF8014638B9144B012203200FF049
:1063A0002BFABEE71049D2E70631BAD106F0ACF8B5
:1063B00004460028B6D04FF47A730122B0FBF3F301
:1063C0000021009303200A4B0FF016FAAAE700BF42
:1063D0003C21002014010020801F0020E81F002025
:1063E000B27C0308180100200C010020797A030810
:1063F000887A0308044B1B7823B9044A052101203D
:10640000FFF786BF704700BF801F0020E37C0308B2
:1064100010B5002490B03C22214601A8009429F038
:106420000DF9454B2022DA7219788DF80010597851
:106430008DF8011099788DF80210D9788DF8031035
:1064400019798DF8041059798DF8051099798DF81E
:106450000610D9798DF80710197A8DF80810597A35
:106460008DF80910997A8DF80A108DF80B202146C5
:106470000DF10B0258180131007B02F8010F1429AD
:10648000F8D193F820208DF8202093F821208DF862
:10649000212093F822208DF8222093F823208DF8D4
:1064A000232093F824208DF8242093F825208DF8BC
:1064B000252093F826208DF8262093F827208DF8A4
:1064C000272093F828208DF8282093F829208DF88C
:1064D000292093F82A208DF82A2093F82B2093F86E
:1064E00028108DF82B20154A19BB93F8291001F0BC
:1064F000FF00F1B9107093F82C206AB193F83F2097
:1065000052B10DF12B0100229818013290F82C00A5
:1065100001F8010F142AF7D109484FF40061FCF784
:10652000E9FC20B9064840226946FCF7E9FB10B0B7
:1065300010BD01211170DEE758030020A4030020E4
:1065400000F8030810B5002204461146054B02204E
:106550000FF052F920460449BDE8104040220FF0E8
:1065600051BA00BFE97C030800F8030838B5434C72
:10657000207963794D2BC0B269D1C0EB0010800047
:106580000A2838BF0A204FF47A7358433C4B1860EE
:10659000A379E2794D2ADBB261D1C3EB03139B00EF
:1065A0004FF47A7202FB03F594F82C30002B5ED185
:1065B00094F83F30002B5AD142F21070FFF750FA96
:1065C000304B1868FFF776FA237A2F4A2F49DBB24F
:1065D00013702F4B01221A70637A2E4ADBB21370AC
:1065E00094F827302C4ADBB2137094F828302B4AE9
:1065F00003EB83035B00DBB2137094F82930284A65
:1066000003EB83035B00DBB2137094F82A30254A56
:106610000133DBB2DB01138094F82B30224A03EB09
:1066200083035B00DBB213700023E21892F82C2086
:10663000D2B2CA540133142BF7D1A378012B1CD149
:10664000E37A202B19D1BDE83840FFF7AFB8637962
:10665000482B0ABF4FF461636379584390E7E279AE
:10666000482A0ABF4FF46162E279534398E7FFF783
:10667000F7F92846FFF742FAA6E738BD580300208D
:10668000140100209C03002006010020DA210020D4
:1066900006000020801F002005000020A703002026
:1066A000A60300203C000020A503002010B590B0F8
:1066B00000213C2201A8009128F0C0FF402243495C
:1066C00068460FF09FF99DF800203AB99DF8010047
:1066D000072803D19DF8021001290FD000223C4B5E
:1066E000114602200FF088F8FFF792FE4FF47A70FF
:1066F000FDF73AFAFFF73AFF10B010BD354B1A70AC
:10670000587099709DF80310D9709DF80410197194
:106710009DF8051059719DF8061099719DF80710A4
:10672000D9719DF8081019729DF8091059729DF8D9
:106730000A1099729DF80B1001F03F01D9720DF10A
:106740000B019818013211F8014F0473142AF8D183
:106750009DF8202083F820209DF8212083F8212017
:106760009DF8222083F822209DF8232083F82320FF
:106770009DF8242083F824209DF8252083F82520E7
:106780009DF8262083F826209DF8272083F82620D0
:1067900083F827209DF8282083F828209DF82920B9
:1067A00083F829209DF82A2083F82A209DF82B20A1
:1067B00083F82B200DF12B0100229818013211F8DB
:1067C000014F80F82C40142AF7D193E700F8030812
:1067D000FD7C030858030020F0B506238BB0052686
:1067E00000240125CDE9053618220723CDE903321F
:1067F0002146744B029422460327CDE9005502201E
:1068000009940EF0F9FF704B029422462146CDE91F
:10681000005702200EF0F0FFCDE9016402266B4B19
:1068200000962246214630460EF0E6FF684B009562
:1068300022462146CDE9017430460EF0DDFF09A95C
:10684000204606F083F9099BC3F307220292C3F3A3
:1068500007421B0E0192009322465E4B21463046B2
:106860000EF0CAFF09A9284606F070F9099BDAB2B2
:106870000392C3F307220292C3F307421B0E019255
:1068800000932246544B214630460EF0B5FF534B41
:106890005348009422464FF4FA710FF03DFB514BE0
:1068A0005148009422464FF4FA710FF035FB4F4BDC
:1068B0004F4800942A464FF4FA710FF02DFB4D4BD0
:1068C0004D4800942A464FF4FA710FF025FB4B4BCC
:1068D0004B4800942A4642F210710FF01DFB2046EF
:1068E000FCF708FA08B1FCF729FC464B009400229B
:1068F0004FF4FA6144480FF00FFB444A0021012095
:106900000FF048F9424A002102200FF043F9414AB2
:10691000002104200FF03EF93F4A002108200FF02B
:1069200039F90021012006F093F83C4B1C7000F06F
:1069300035FE3B493B4806F0BFF83B4805F0ACFF4D
:106940002B480FF095FB394B0021187805F0FCFC23
:1069500037490094374B0968374800220FF0DCFABA
:1069600035480FF085FBFFF7A1FE344A00211020C7
:106970000FF010F9324A002120200FF00BF9314AB4
:10698000002140200FF006F92F4A002180200FF04F
:1069900001F92E4B2E4819682E4B009401220FF05E
:1069A000BBFA2B480FF064FB2B4B2C4819682C4B7F
:1069B000009401220FF0B0FA28480FF059FB0BB0F9
:1069C000F0BD00BF3D7D03087D7D03089E7D03086B
:1069D000BF7D0308E07D0308017E0308CF5900084E
:1069E0001820002015620008002000202161000806
:1069F000E81F0020C5610008CC1F0020C95E000808
:106A0000B41F002009610008242100209DC6000851
:106A1000B15C000895610008395C0008E41F0020A3
:106A20000000030130010020180100207C0100203B
:106A300014010020195A00083C2100209953000835
:106A40001554000879540008F9540008A0030020E8
:106A50009C1F0020D96000089C030020841F002098
:106A60008160000873B50D4D00262E60FEF7CCFE48
:106A7000C820FDF779F828683146FBF787FC044603
:106A80000028F3D12868FBF7C9FC054B009022468B
:106A9000214601200EF0B0FE02B070BD181F00208C
:106AA000257E030830B50024A5B07C22214605A828
:106AB000049428F0C3FD53238DF81030012540F2D3
:106AC0000713ADF81230ADF800408DF81450FCF704
:106AD000C9FFFE23B0FBF3F000EB400000EB4010D9
:106AE0003A4B8DF815002246214603200EF084FE15
:106AF0006846FEF7F1FE9DF800309DF80120134333
:106B000014D158238DF816300724802200213048F4
:106B100028F094FD224604A92D4828F025FE2C4A91
:106B200021460120FFF7F4FB25B030BD0E23294696
:106B300001A8CDE901448DF81630ADF80C40FEF700
:106B40008DFE01AB03CB234C1B88CDF81B10ADF899
:106B50001F30CDF81700FEF757FE2068FBF784FCC6
:106B60000A254FF47A7380B2B0FBF3F0B0FBF5F373
:106B700005FB130030308DF821002068FBF774FC12
:106B8000642380B2B0FBF3F0B0FBF5F305FB130018
:106B900030308DF822002068FBF766FC80B2B0FB35
:106BA000F5F0B0FBF5F305FB130030308DF8230052
:106BB0002068FBF759FC80B2B0FBF5F305FB13002E
:106BC00030308DF8240015249FE700BF587E03085D
:106BD00054210020181F00202DE9F047044698B0EA
:106BE000B9480D46802200210EF016FF2378592B5C
:106BF00040F05982052D5ED86378443B162B5AD855
:106C0000DFE813F09B0159008B01590093015900F3
:106C1000590059005900BD0059007601590059002A
:106C20005900F60159005900E70059005900590070
:106C30001700A678482E17D1A44A14210120FFF787
:106C400067FB41F28830FCF78FFF0022A04B114612
:106C500003200EF0D1FD40F6B830FCF785FF18B0E8
:106C6000BDE8F047FFF768BA532E0DD1FFF71AFFC2
:106C700041F28830FCF778FF934A1521012018B0C3
:106C8000BDE8F047FFF744BB432E17D1002408A806
:106C90008DF8204005F078FD8B4A4C2313700723B4
:106CA00093709DF82030547001204133D0701371DF
:106CB0000521FFF72DFB18B0BDE8F087442EFAD16F
:106CC000814C844DA670592323705A236370FFF7BB
:106CD000C9FE2868FBF7A2FB00227F4B00901146FB
:106CE00003200EF089FD7F220021601C28F0A6FC05
:106CF000072326700126A370E6702671FCF7B2FE0A
:106D0000FE23B0FBF3F000EB4000042300EB401047
:106D10006071A3712868FBF7A7FB0A274FF47A7309
:106D200080B2B0FBF3F0B0FBF7F307FB1300303099
:106D3000E0712868FBF798FB642380B2B0FBF3F0A6
:106D4000B0FBF7F307FB1300303020722868FBF725
:106D50008BFB80B2B0FBF7F0B0FBF7F307FB13003F
:106D6000303060722868FBF77FFB80B2B0FBF7F32E
:106D700007FB13003030A07222460B217EE7A37878
:106D8000303BDBB2092B96D8544C554A23702378FC
:106D9000DBB253724C4A592313704D23537023783E
:106DA0000321303301209370FFF7B2FA2378009368
:106DB00000224C4B114601200EF01EFDFFF728FB70
:106DC0002378002B3FF477AF18B0BDE8F047FCF70D
:106DD0000FBCA578482D39D13B4C5623237007238F
:106DE000A37018236371062300250126A37106A84A
:106DF0000523E3716570E67026710EF067FF069853
:106E000008A912380EF0EAFF0D9B03F26C7305938C
:106E10000C9B334404930B9B0393089B0293099BA5
:106E200001930A9B00932A462F4B294602200EF01D
:106E3000E3FC224608213046FFF76AFA2B4B009408
:106E40002A46114602200EF0D7FC34E7432D7FF48A
:106E500032AF00213C2209A81B4C089128F0EEFB20
:106E600008A8FFF76FFB9DF8203063709DF8213074
:106E7000A3709DF82230E3709DF8233023719DF8B4
:106E8000243063719DF82530A3719DF82630E3719D
:106E90009DF82730257023729DF82B509DF82830DF
:106EA00063729DF82930A3722A469DF82A30E37256
:106EB0000BA904F10D00257328F056FC05F10D0116
:106EC0002246C9B20120F4E654210020717E030855
:106ED000867E0308181F0020A87E0308801F00205C
:106EE00058030020CB7E0308F47E03081E7F0308AE
:106EF000A07839280CD83038C0B2FEF70BFD8E4A86
:106F00002378137063785370A37893700321B5E6E8
:106F100018B0BDE8F047FFF76DBAA0783928F7D868
:106F20003038C0B2FEF7FBFCE9E7A0783928EFD88B
:106F30003038C0B2FEF7F8FCE1E7A378303BDAB2B4
:106F4000092AE5D8E578303DEAB2092AE0D8217966
:106F5000A1F14802D2B20B2ADAD8784840FA02F2FC
:106F6000D007D5D40A224D2902FB03553BD13C233F
:106F70005D43734B4FF47A7068431860714B18602F
:106F8000FEF798FD6C4A2378137063785370A378EA
:106F90009370E378D3700521237913710120FFF7F3
:106FA000B7F9694B002607221E705A7001229A70A9
:106FB000DA70A178303901EB8100E178303901EBEA
:106FC0004001C9B2197122795A71604A1278D2B25D
:106FD0001A725F4A1278D2B25A72FFF719FA5D4BF1
:106FE000009532462DE74829C3D14FF46163BFE7CE
:106FF000A278303AD3B2092B8AD8E378303BD9B2A1
:10700000092985D82079A0F14801C9B20B293FF69A
:107010007FAF4A4D45FA01F1C9073FF579AF0A2123
:107020004D2801FB023339D13C2253434FF47A728D
:107030005343494A13601068FEF760FD3E4A2378C7
:10704000137063785370A3789370E378D37005213D
:10705000237913710120FFF75BF93B4B00221A7073
:1070600007225A7001229A70DA70A278303A02EB45
:107070008201E278303A02EB4102D2B29A7122796F
:10708000DA71324A1278D2B21A72314A1278D2B216
:107090005A7218B0BDE8F047FFF7BAB94828C5D111
:1070A0004FF46162C1E7502B40F0A581022D7FF6BD
:1070B00002AE6178A1F13003012B3FF6FCADA3785D
:1070C000312B7FF4F8AD052D4ED1E378302B40F015
:1070D000C1801E4D214E00232B702B7803F0FF0240
:1070E00053B92379303BDBB23370337800931146C8
:1070F0001B4B02200EF080FB15491A4A00230B702F
:107100003378DBB213702B780F4ADBB213720B7833
:10711000DBB25372FFF77CF9074B22781A70627862
:107120005A70A2789A70E278DA7022791A71FCF7B4
:1071300011FB0521004AA1E554210020DEF7FFFFE5
:10714000140100209C0300205803002006010020A9
:10715000801F0020487F0308A003002004000020B7
:107160007F7F030806000020082D67D1E378462BB7
:1071700040F0EA802179A1F13000C0B2092800F284
:1071800038816279A2F13003092B00F23281A679AD
:10719000A6F13003092B00F22C81E379A3F130052D
:1071A000092D00F2268101EB81014900AF4D20310C
:1071B00002EB8202C9B2520029702032AC49D2B22D
:1071C0002F3E0A70F6B2AB4A03EB8303F6015B0075
:1071D00016802033A84ADBB21370A84A82F8280030
:1071E0006379303BDBB282F82930A3792F3BDBB2E5
:1071F00082F82A30E379303BDBB282F82B302B78EF
:107200002BB90B7803F0FF020BB99D4B1A70FFF7F7
:10721000FFF89C4B22781A7062785A70A2789A70A4
:10722000E278DA7022791A7162795A71A2799A71C8
:10723000E279DA71FCF78EFA08217BE7042D2FD171
:10724000E278A2F13003DBB2092B11D9A2F141039C
:10725000192B0AD9FFF7CEF800228B4B11460120DB
:1072600018B0BDE8F0470EF0C7BAA2F13703DBB2A1
:1072700086480370834B20785970312118709970BB
:10728000DA70824B7D4A1B78DBB21372804B1B781D
:10729000DBB25372FFF7BCF8FCF75CFA042149E754
:1072A0001D2D4FD9A61C0025DFF8D091DFF8E4A1F1
:1072B0003746A84617F8012F303AD2B2092A3ED8ED
:1072C00009EB050303201A731B7BCDE902533B78BE
:1072D0000022CDE90053114653460EF08DFA0135D8
:1072E0001E2DE7D1B8F1000FB4D1FEF71DF9654BA3
:1072F00050221A7000225A7007229A700122DA7006
:1073000003F8042F203416F8012F03F8012FB4429C
:10731000F9D15A4B00221A7007225A7001229A7032
:10732000DA705A4A1278D2B21A72594A1278D2B224
:107330005A721E22DA72FFF76BF82321FAE64FF039
:107340000108CCE7072D85D900254C4FDFF8448193
:1073500002342E4614F8012F303AD2B2092A46D808
:10736000791903200A730B7BCDE90253237800229D
:10737000CDE90053114643460EF03EFA0135082D83
:10738000E8D1002E7FF466AFFEF740F93D4B3B4C51
:1073900050221A7007229A701A460121002502F81D
:1073A000041F5D70D97061190135097B082D01F149
:1073B000300102F8011FF6D100221146009301208E
:1073C000354B0EF019FA0023237007236370012355
:1073D000A370E3702D4B1B78DBB223722C4B1B7810
:1073E000DBB26372E572FFF713F80D21A2E6012606
:1073F000C4E700219EE6412B7FF45DAC6378432B0C
:107400007FF459AC162D7FF456AC244D621C00233A
:1074100012F8011FE9540133142BF9D1FDF78CFF49
:107420001F4B5B7D012B1DD114490023EA5CC8185A
:107430000133D2B2142B80F82C20F7D1144B002248
:107440001A701B78DBB24B72FEF7E2FF0D4A631E27
:10745000153413F8011F02F8011BA342F9D1094AA0
:1074600016210BE40A4B02221A70EFE7A703002053
:10747000A60300203C000020A503002058030020A4
:10748000A403002054210020DE7F03080601002011
:10749000801F00209B7F0308C37F0308DA210020A0
:1074A0002C0A002070B5054688B00C46002951D042
:1074B00033480EF0DDFD26789EB3002D5ED068685F
:1074C0002E7870B3032E0BD0132E45D0022E28D168
:1074D0006978012925D00B0623D4FFF77DFB20E036
:1074E0006B78012B07D10078012802D0022800D048
:1074F00008B905F003F900250DF11F008DF81F50A4
:1075000005F042F91F4A4C231370072393709DF82E
:107510001F305570012041330521D0701371FEF7E3
:10752000F7FE237C052B15D894F90A20059294F9CF
:1075300009200492144A52F82330039394F9083036
:10754000CDE901630022E368009311460F4B03204D
:107550000EF052F908B070BD6B78012BE1D10278C2
:107560000B4B02F001021A702AB90A4B1146032094
:107570000EF042F9D5E7084B0022F7E72E46D0E798
:107580000020002054210020688003081680030892
:1075900030200020038003080D800308034B0022E5
:1075A000C3E902220122C3E900227047F021002032
:1075B00000487047F02100204FF0B04382B0DA6CF1
:1075C0000243DA64DB6C03400193019B02B0704715
:1075D0002DE9F04186B000240220154D0594FFF7F7
:1075E000EBFF0420FFF7E8FF124F03944FF480767F
:1075F00001230DEB0001CDE9016328460323049329
:107600004FF4005801F04AF801A93846CDF804803B
:1076100001F044F822464146384601F065F9284613
:107620002246314601F060F9204606B0BDE8F081FF
:107630000004004800080048032810B50ED80128AF
:1076400010D868B902460B484FF4807101F04CF92C
:10765000002209484FF4005101F046F9002010BD06
:107660000122F0E7002203484FF4807101F03CF959
:107670000122EEE70004004800080048022070479D
:107680000020704701207047002814BF16200F20EB
:10769000704700000D48854600F025F80C480D495C
:1076A0000D4A002302E0D458C4500433C4188C425D
:1076B000F9D30A4A0A4C002301E013600432A242C3
:1076C000FBD328F023F8FBF71BFDFEE700000120A9
:1076D000000000204808002028E703084808002090
:1076E0001C420020FEE7704710B5032000F06EFC3E
:1076F00001F07CFA064B18600F20FCF72BFA0446C9
:1077000018B9FBF773FE204610BD0124FBE700BF4C
:10771000A80300204FF0E022136923F00203136155
:1077200070474FF0E022136943F002031361704782
:10773000014BD3F8900570470070FF1F014BD3F841
:10774000940570470070FF1F014BD3F898057047F0
:107750000070FF1F024A536843F0010353607047F3
:10776000002004E0024A536843F00203536070476C
:10777000002004E0024A536843F00403536070475A
:10778000002004E08068C0F380007047F7B5002354
:1077900001930446002800F0E980856D25B9FBF7C8
:1077A00039F9E56584F8545023689A68D00040F1AF
:1077B000A1809A68D10000F1B480A26D42F010025D
:1077C000A265E26D42F00102E26501251846FFF76D
:1077D000D9FFA26D02F01002024340F0C980A26DF1
:1077E000206922F4817242F00202A2659A68D207EF
:1077F0005DD4226BA67E94F82CC0003A18BF0122FB
:107800001703D4E902120A43217E42EA8132617EE3
:1078100042EAC13242EA4632002842EA4C02B4BF90
:1078200020F000414FF400113A430A4394F820102D
:10783000012903D1002E76D142F48032616A21B150
:10784000A66A01F4E07131430A43D968E66C21F479
:10785000FE3121F4FF711143D96094F83C20616836
:10786000012A01F0404C4CEA060609D1D4E9102760
:107870003A433243A66C324342EA0C0242F001061C
:107880001F693E4A3A4032431A6121F00042B2F188
:10789000804F0CD0B1F1004F09D0394ED6F80827EF
:1078A00001F4701122F470120A43C6F808275A69CD
:1078B000666BA16B22F0070232435A615A6922F0CB
:1078C000700242EA01125A61002835D19A6A62F0C8
:1078D0000F029A625B6903F007039E423CD10023CA
:1078E000E365A36D23F0030343F00103A36528467A
:1078F00003B0F0BD9A68234922F0104222F017022B
:1079000042F080529A60204A1268B2FBF1F20132D2
:1079100052000192019A002A3FF44BAF019A013ABA
:10792000F7E7002552E7A16D41F02001A165E16D67
:1079300041F00101E16581E7B0F5001FCAD19A6A03
:10794000E269013A92006FF00F0102F01C0201FAA5
:1079500002F2216E0A43BCE7A36D23F0120343F049
:107960001003A365E36D43F00103E3650125BEE762
:10797000A36D43F01003A365F8E700BF02FCFF1FEF
:1079800000200140400D0300A8030020F8B5456920
:10799000082D04460E460AD00368DB68D80705D5D3
:1079A000A36D43F02003A3650120F8BD0425FCF777
:1079B000D3F8074623681A682A4220D0A26D42F401
:1079C0000072A265DA6812F4406F14D1A27E92B9F7
:1079D0001A6812070FD51846FFF7D4FE20BB5A6865
:1079E00022F00C025A60A26D22F4807222F0010291
:1079F00042F00102A265227EFAB10020D5E7711C97
:107A0000D9D0FCF7A9F8C01BB04201D8002ED1D1C3
:107A100023681B682B40CDD1A26D84F8543042F00E
:107A20000402A2650320C0E7A26D42F02002A26515
:107A3000E26D42F00102E265DDE70C221A60DCE74C
:107A40000368186C70470000F7B50023019390F8A5
:107A50005430012B044600F0C08005680269012300
:107A600080F854302846FFF78DFE002840F0AF80A4
:107A7000D1E90030022822F004027ED0B2F1004F9A
:107A8000C3F3110E35D1AA6A42EA0E02AA628A68CD
:107A9000686902EA032222F07C4222F0FF0220EA17
:107AA00003210A43002B6A611DDA4D4A4D4DD2F87D
:107AB0000817AB4201F0E07043D10D0213D4D2F8A5
:107AC000083723F0E073034343F40003C2F8083798
:107AD000454B1A68454BB2FBF3F20C2302FB033310
:107AE0000193019B53BB0020002384F8543003B062
:107AF000F0BD226E00F01F074FF00F0C0CFA07FCD0
:107B00006FEA0C0622EA0C0CBEF1000F11D1C3F390
:107B10008462BA4042EA0C0222668008E2690130BF
:107B20009042B4D8A86AC3F38362BA400640324395
:107B3000ACE793FAA3F2B2FA82F2EAE7019B013BC7
:107B4000CEE72B4DAB420BD1C901CCD4D2F80837CC
:107B500023F0E073034343F08073C2F80837C2E7B1
:107B6000244DAB42BFD14B02BDD4D2F8083723F02D
:107B7000E073034343F48003EFE7B2F1004F01BF2A
:107B8000AA6AC3F311018A43AA62002BABDA154833
:107B900013498342D1F8082709D1D1F8083702F0F8
:107BA000A07223F0E0731A43C1F808279BE710483E
:107BB000834204D1D1F8083702F44002F1E70D48BE
:107BC000834290D1D1F8083702F0C072E9E7A26D84
:107BD00042F02002A265184686E7022087E700BF30
:107BE00000200140001000B0A8030020400D030059
:107BF000004000B8002000B4026838B504461046C2
:107C0000FFF7C0FD08B9002038BD9368990707D475
:107C1000936823F0004323F0170343F010039360AD
:107C2000FBF79AFF054623689B685B07EBD5FBF7DC
:107C300093FF401B0228F6D923689B685A07F2D5A8
:107C4000A36D43F01003A365E36D43F00103E36507
:107C50000120D9E773B50023026801939368DD071B
:107C6000044602D5002002B070BD9168214B194234
:107C700009D0A36D43F01003A365E36D43F0010346
:107C8000E3650120EFE7936823F0004323F0170337
:107C900043F001039360184BD3F8083718021CD443
:107CA000637E012BDED0FBF757FF144E054622689A
:107CB0001368DB07D6D49368D9075FBF9368334056
:107CC00043F001039360FBF747FF401B0228EED906
:107CD00023681B68DA07EAD4CBE7094B094A1B681B
:107CE000B3FBF2F301330193019B002BD8D0019B2E
:107CF000013BF8E71700008000200140E8FFFF7F0C
:107D0000A8030020400D030038B504460068FFF7C3
:107D100039FD054620BB94F85430012B20D00123B7
:107D200084F854302046FFF795FFB0B9A36D226860
:107D300023F4706323F0010343F48073A3651C23D1
:107D4000E065136084F85400936823F0004323F047
:107D5000170343F00403936038BD84F85450FBE7E5
:107D60000220F9E7026838B5936891680446C807AD
:107D700001D4002038BD9907FBD4936803F00503B4
:107D8000012B19D1936823F0004323F0170343F02C
:107D90000203936003231360FBF7DEFE05462368AE
:107DA0009B68DB07E5D5FBF7D7FE401B0228F6D919
:107DB00023689B68DA07F2D5A36D43F01003A3652F
:107DC000E36D43F00103E3650120D3E770B504469A
:107DD00000284BD0836D43F002038365FFF70CFF4F
:107DE000054668B92046FFF7BDFF054608B90123DF
:107DF000A3652268936823F0104323F01703936070
:107E000023685A6822F4677222F003025A6040F233
:107E10009F321A60D968164A0A40DA601A6922F05D
:107E200040421A615A6922F007025A611A6A02F046
:107E3000F0221A625A6A02F0F0225A62DA6A02F0FA
:107E4000F022DA629A6A0B4A00269E62D2F808375C
:107E500023F0FE73C2F808372046FAF7EFFDE66517
:107E60002666A66584F85460284670BD0125FBE7A8
:107E700000023E830020014010B590F85430012BE1
:107E8000044615D0012380F85430FFF7B5FE58B9E9
:107E90002046FFF767FF38B9A36D23F4807323F002
:107EA000010343F00103A365002384F8543010BD9F
:107EB0000220FCE7F7B50023019390F85430012B22
:107EC00004467FD0012380F85430FFF74BFF23682E
:107ED0009A6812F00102054607D0A36D43F0100323
:107EE000A365002384F854302DE0A16D364F21F4B2
:107EF000817141F00201A165DE68D96826F4FF4670
:107F000026F07C0621F40041360421F00301360CF2
:107F1000D96008209968394041F00041996099681A
:107F2000002913DA0199013101910199B1F52E3F30
:107F3000F5D3A36D23F0120343F01003A3650023D0
:107F400084F854300125284603B0F0BDD3F8B410AE
:107F5000013801F07F010A44DCD199681A480140D8
:107F600041F001019960D3F8B41021F07F0141EA9A
:107F7000D202C3F8B4209A68024042F002029A602A
:107F8000FBF7EAFD074623689A68D20708D4DA6847
:107F90003243DA60A36D23F0030343F001039FE74C
:107FA000FBF7DAFDC01B0228EDD923689B68D907CF
:107FB000E9D5A36D43F01003A365E36D43F001031E
:107FC000E365BFE70225BEE7E8FFFF7F0749CA6810
:107FD00022F4E0620302120403F4E063120C134380
:107FE00043F0BF6343F40033CB60704700ED00E023
:107FF000164B30B5DC68C4F30224C4F10703251D19
:10800000042B28BF0423062D4FF0FF358CBF033C03
:10801000002405FA03F321EA0303A54022EA05023E
:10802000A340002843EA0203ACBF00F16040084AC5
:108030004FEA0313B8BF00F00F00DBB2AABF00F590
:108040006140135480F8003330BD00BF00ED00E004
:1080500014ED00E0002807DB044A4109012300F089
:108060001F00834042F82130704700BF00E100E06C
:1080700000280CDB4309064900F01F0020330122D1
:10808000824041F82320BFF34F8FBFF36F8F7047BB
:1080900000E100E070B5D0E913456560446D14B1AE
:1080A000D0E916456560D0E9105404F01C0601249F
:1080B000B4406C60046863608368102B0BBFA260DF
:1080C000A160E160E26070BD0268416CD3B210B59E
:1080D000083B1424B3FBF4F30B4CA24288BF0B4AB9
:1080E00021F0030199BF01F1804202F502325218DA
:1080F00007338264064AC26403F01F03012202FAB6
:1081000003F3036510BD00BF070402401C080240D2
:108110008008024038B500285CD002682E4B9A4295
:108120004FF014014AD82D4B1344B3FBF1F32C4903
:108130009B00C0E91013022380F8253013680569FD
:1081400023F4FF4323F070031360D0E90243234379
:108150002B43456911682B4385692B43C5692B4324
:10816000056A2B430B431360FFF7AEFFB4F5804F56
:1081700004BF002343604368816C03F07F020A6000
:10818000D0E91314013B032B4C601ED8154B164944
:10819000816513449B000121013A01FA02F200219A
:1081A0004365C2651960114B5A6400230122C36301
:1081B00080F8243080F82520184638BD0C4B134435
:1081C000B3FBF1F30B499B00B3E70023C0E9153380
:1081D000C365EAE70120F0E707040240F8FFFDBFAE
:1081E000000002403F8200104009024000090240A6
:1081F000F8FBFDBF0004024038B5002841D00268FA
:10820000136823F0010313601F4B9A424FF01401CF
:1082100030D81E4B1344B3FBF1F31D499B00C0E95A
:108220001013012403F01C0304FA03F30025156066
:108230004B60FFF749FF836C41681D60D0E9133242
:108240005A604A1E032A06D8124B0B449B009440E6
:108250001D60114B5C640023C363C0E91533C0E9A2
:108260000B33C0E90D33C36580F8253080F8243026
:10827000184638BD094B1344B3FBF1F308499B0082
:10828000CDE70120F5E700BF07040240F8FFFDBF7E
:10829000000002403F82001000090240F8FBFDBFD1
:1082A0000004024070B590F82450012D04463BD0E4
:1082B00090F825600125AE4280F824504FF000066A
:1082C0002CD1022580F825500568C6632E6826F05B
:1082D00001062E60FFF7DEFE036BBBB12B6843F097
:1082E0000E032B60A36C1A68D20342BF1A6842F4D3
:1082F00080721A60636D1BB11A6842F480721A6052
:108300002B6843F001032B60002070BD2B6823F025
:1083100004032B602B6843F00A03E2E78023C36366
:1083200080F824602846F0E70220EEE7034640B1DB
:1083300090F82520022A06D00422C263002280F889
:108340002420012070470268806C116821F00E0122
:108350001160016821F480710160116821F0010150
:108360001160D3E9100202F01C0101228A40426030
:10837000D3E9132151605A6D32B1116821F4807133
:108380001160D3E9162151600122002083F82520D5
:1083900083F82400704708B590F82530022B03D0ED
:1083A0000423C363012008BD03681A6822F00E028B
:1083B0001A601A6822F001021A60826C136823F4B2
:1083C00080731360D0E9101303F01C020123934063
:1083D0004B60D0E913325A60436D33B11A6822F40E
:1083E00080721A60D0E916325A60012380F8253075
:1083F000002380F82430836B03B198470020D2E734
:1084000070B4426C046C036826681D6802F01C029C
:108410000421914031420FD015F0040F0CD01A689E
:1084200092065EBF1A6822F004021A60036B616054
:10843000002B33D070BC184702219140314217D035
:1084400015F0020F14D01A68940606D41A6822F0A8
:108450000A021A60012280F82520114A93428CBF3B
:10846000104B114B5960002380F82430C36ADFE7BA
:1084700008219140314211D029070FD5196821F008
:108480000E011960012303FA02F26260C36380F8EF
:108490002530002380F82430436BC9E770BC704757
:1084A0008000024000040240000002400A4A536972
:1084B00043F4802330B55361EFF3108472B6002388
:1084C000CD58C5500433B3F5807FF9D11369DB0370
:1084D000FCD484F3108830BD00400058064B5A6924
:1084E000002ABFBF054A9A6002F188329A60BABF7B
:1084F0005869C00F002070470040005823016745AD
:10850000044B5A6942F000425A615869C043C00F97
:10851000704700BF0040005870B50546FBF71CFBD4
:10852000124E04463369D90313D43369DA0744BFC2
:10853000012232614CF2FA32134011D10B4E3069F4
:1085400010F480200BD0FBF707FB001BA842F6D3EA
:1085500004E0FBF701FB001BA842E3D3032070BD3E
:10856000024A1361024A01205360F8E700400058B4
:10857000002200202DE9F041184D98462B78012B60
:1085800006460C46174626D001232B704FF47A700E
:1085900000236B60FFF7C0FFA0B9012E16D1104A6F
:1085A000536943F0010353612760BFF36F8FC4F831
:1085B00004804FF47A70FFF7AFFF094A536923EA4A
:1085C0000603536100232B70BDE8F0813946204635
:1085D000FFF76CFFEDE70220F6E700BF0022002066
:1085E00000400058054A536923F47E7343EAC000F3
:1085F00040F4803040F00200506170470040005865
:108600002DE9F041234F3B78012B054688463FD0AA
:1086100001233B704FF47A7000237B60FFF77CFFEF
:10862000044688B92B68042B13D11B4A536943F4C1
:10863000803343F0040353614FF47A70FFF76CFF0B
:108640000446154B1A681B6800233B702046BDE8A2
:10865000F0814FF0FF33C8F800306E68D5E9013281
:108660001344B3420AD93046FFF7BCFF4FF47A7087
:10867000FFF752FF50B1C8F800600446064A53693C
:1086800023F47E7323F002035361DAE70136E5E752
:108690000224DBE700220020004000582DE9F04FC3
:1086A000524C00234FF00F090A6832FA03F501D14A
:1086B000BDE8F08F012505FA03F818EA020200F080
:1086C0008E804E68032706F003054FEA430E07FA33
:1086D0000EFC6F1E012F6FEA0C0C32D8876807EA78
:1086E0000C0ACF6807FA0EF747EA0A07876047685F
:1086F00027EA0808C6F300179F4047EA08074760C3
:10870000C76807EA0C088F6807FA0EF747EA0807F8
:10871000022DC76017D14FEAD30800EB880803F099
:10872000070AD8F820704FEA8A0A09FA0AFB27EAF2
:108730000B0B0F6907FA0AF747EA0B07C8F8207016
:1087400001E0032DDCD1076805FA0EF507EA0C07F6
:108750003D4316F4403F056041D023F0030707F185
:10876000804707F5803703F0030CBD684FEA8C0C97
:108770004FF0070E0EFA0CFEB0F1904F25EA0E0EE8
:108780002FD01B4DA8422ED005F58065A84214BFFE
:108790000725022505FA0CF545EA0E05BD6025689A
:1087A000D74316F4801F0CBF3D4015432560656814
:1087B00016F4001F0CBF3D4015436560D4F880508F
:1087C00016F4803F0CBF3D401543C4F88050D4F8E8
:1087D0008450B60354BF3D401543C4F88450013360
:1087E00062E70025D6E70125D4E700BF000800585E
:1087F00000040048374A2DE9F04F00234FF0010AEA
:108800004FF0070B4FF00F0931FA03F401D1BDE827
:10881000F08F0AFA03FC1CEA010654D023F003048B
:1088200004F1804404F5803403F00307A568BF0019
:108830000BFA07F8B0F1904F08EA050E45D0264D27
:10884000A84244D005F58065A8420CBF0225072543
:10885000BD40754517D1D2F8805025EA0605C2F80B
:108860008050D2F8845025EA0605C2F88450156875
:1088700025EA06051560556825EA06055560A568D0
:1088800025EA0805A560056803265C0006FA04F4DD
:1088900023FA06F6254300EB8606056003F007057C
:1088A000376AAD0009FA05F527EA050737628568DA
:1088B00025EA04058560456825EA0C054560C5681C
:1088C00025EA0404C46001339EE70025C0E70125C2
:1088D000BEE700BF000800580004004803691942C1
:1088E00014BF0120002070470AB181617047816286
:1088F0007047436901EA030221EA030141EA0241A8
:1089000081617047044AD168014208B502D0D06045
:10891000FDF782FC08BD00BF00080058024A13683A
:1089200043F4807313607047000400580D4B10B57A
:108930005B690C4628B99A0507D500F027F820B1E5
:1089400010BD9B0501D400F019F8074A1369012CEA
:1089500023F00403136101D130BFF1E740BF20BF12
:1089600020BFEDE70004005800ED00E0024B18685E
:1089700000F4C060704700BF00040058024A13684A
:1089800043F4804313607047000400580C4A136896
:1089900023F4804313600B4B1B6832214B430A497D
:1089A000B3FBF1F35169890500D533B9536913F469
:1089B000007F14BF032000207047013BF2E700BF97
:1089C00000040058A803002040420F000B4A13681F
:1089D00023F0070343F002031360094B1A690128CF
:1089E00042F004021A6105D130BF1A6922F0040274
:1089F0001A61704740BF20BF20BFF6E7000400584F
:108A000000ED00E04FF0B0431868C0F340407047FD
:108A10004FF0B0431868C0F3400070474FF0B042C9
:108A2000536823F47F4343EA0023536070474FF0B9
:108A3000B0431868C0F34060704700007FB54FF046
:108A4000B0432C4AD3F80831C0F3031003F00F03EE
:108A500052F82040284A52F82330B4FBF3F4FFF7D1
:108A600085FF264B054693E80700B5F5007F04AB6C
:108A700003E9070010D0224B9C4218D303F5B7033B
:108A800003F67F539C4229D903F5741303F5106351
:108A90009C4225D802230BE01A4B9C4207D91A4B63
:108AA0009C421BD903F5370303F5D853F0E70023A5
:108AB00004AA02EB830353F80C4C144D2B6823F0EB
:108AC000070323432B60FBF747F806462B6803F0A8
:108AD00007039C4206D1002004B070BD0123E7E7E4
:108AE0000024EAE7FBF738F8801B0228EED90320C0
:108AF000F2E700BF80800308E0800308282C030809
:108B0000C0CF6A00BFEA21013F9334020040005801
:108B10004FF0B04310B59A68D96812F00C0205D036
:108B20000C2A4AD101F00303012B51D14FF0B0417F
:108B30002B480B6813F0080306D00B6813F00803EA
:108B400037D1D1F8941007E00C68240756BFD1F84C
:108B500094300968C3F3032350F82330002A0CBF74
:108B6000184600204FF0B0418A6802F00C020C2A2F
:108B70001ED1CA6802F00302022A2ED0032A06D1AF
:108B80000B68184A13F4801F174B18BF13464FF099
:108B9000B042D068D168D268C0F306205843C1F310
:108BA00002130133B0FBF3F0530F0133B0FBF3F0CA
:108BB00010BD0B68C3F30313CEE7042A05D0082ABF
:108BC00006D11B6813F4801305D006480023C9E7BB
:108BD00000231846C6E70448C4E7024BD7E700BFA6
:108BE000808003080024F4000048E80108B5FFF77E
:108BF0008FFF4FF0B043044A9B68C3F3031352F84E
:108C00002330B0FBF3F008BDE08003082DE9F0410C
:108C10000446002853D04FF0B0439D68DE680368D7
:108C20009B0605F00C0506F0030668D5026A1DB127
:108C30000C2D46D1012E44D1002A40D04FF0B04334
:108C4000A16A1A68170756BFD3F894301B681B092E
:108C500003F0F00399421FD90846FFF7EFFE002802
:108C60002DD14FF0B042136843F00803136013682E
:108C7000A16A23F0F0030B431360606AFFF7CEFE96
:108C8000FFF7B4FFAB4B1860AB4B1868FAF762FF05
:108C9000002834D0BDE8F0814FF0B042136843F0B3
:108CA00008031360136823F0F0030B431360606A3A
:108CB000FFF7B4FE0846FFF7C1FE0028E0D0012010
:108CC000E8E74FF0B043002A54D01A6842F001029E
:108CD0001A60FAF741FF0746FFF79AFE002842D0D4
:108CE0004FF0B042136843F0080313601368A16AA1
:108CF00023F0F0030B431360606AFFF78FFE2368D5
:108D0000D80748D42368990700F18C8023681E0790
:108D100040F1FA80A3694FF0B046002B00F0E180EB
:108D2000D6F89430E16903F01002914200F0C4805B
:108D300003F00302022AC2D0D80740F1B380D6F86C
:108D4000943023F00103C6F89430FAF705FF074684
:108D5000D6F89430990740F1A580FAF7FDFEC31BC1
:108D6000112BF5D904E0FAF7F7FEC01B0228B3D99E
:108D700003208FE71A6822F001021A60FAF7ECFE6E
:108D80000746FFF745FE0028B9D0FAF7E5FEC01BFD
:108D90000228F6D9ECE7082D03D00C2D05D1032EBF
:108DA00003D16368002BADD189E74FF0B043A168D0
:108DB0001A6822F480120A431A606268B2F5803F92
:108DC00010D11A6842F480321A60FAF7C5FE0746DD
:108DD000FFF718FE002895D1FAF7BEFEC01B6428E5
:108DE000F6D9C5E7B2F5041F04D11A6842F400129F
:108DF0001A60E6E7196821F480311960196821F4D6
:108E000000111960002AE0D1FAF7A6FE0746FFF725
:108E1000F9FD00283FF476AFFAF79EFEC01B6428E8
:108E2000F5D9A5E7042D236903D00C2D0ED1022E10
:108E30000CD1002B3FF443AF4FF0B042616953684F
:108E400023F0FE4343EA016353605FE74FF0B0460F
:108E5000BBB1336843F480733360FAF77DFE074695
:108E600033685A0505D4FAF777FEC31B022BF7D9EE
:108E70007EE77368626923F0FE4343EA026373602E
:108E800044E7336823F480733360FAF765FE0746DE
:108E900033685B057FF53AAFFAF75EFEC31B022B22
:108EA000F6D965E74FF0B042E169D2F8943023F08B
:108EB00010030B43C2F894304FF0B047D7F894300A
:108EC00043F00103C7F89430FAF746FE0646D7F898
:108ED00094309A0718D4FAF73FFE831B112BF6D96A
:108EE00046E7D6F8943023F00103C6F89430FAF739
:108EF00033FE0746D6F894309B0705D5FAF72CFECB
:108F0000C31B112BF6D933E72368580754D50B4FF1
:108F10003B68D90514D4FFF701FDFAF71DFE06469C
:108F20003B68DA050CD4FAF717FE831B022BF7D93E
:108F30001EE700BFA8030020AC0300200004005877
:108F4000E3684FF0B046002B58D023F08003052B88
:108F500002BFD6F8903043F00403C6F890304FF0CB
:108F6000B046FAF7F9FDD6F8903043F00103074612
:108F7000C6F8903041F28838D6F890309B0705D477
:108F8000FAF7EAFDC31B4345F6D9F1E6E36823F09F
:108F90000403812B1BD1FAF7DFFDD6F8903043F0A4
:108FA0008003C6F8903007464FF0B04641F288384B
:108FB000D6F89030180504D5E36A002B4AD100207A
:108FC00068E6FAF7C9FDC01B4045F1D9D0E6FAF7CB
:108FD000C3FDD6F8903023F08003C6F890300746E2
:108FE0004FF0B04641F28838D6F890301905E3D5F5
:108FF000FAF7B2FDC01B4045F6D9B9E6FAF7ACFD69
:10900000D6F8903023F080030746C6F8903041F23E
:109010008838D6F890301A0516D4FAF79DFDD6F8A0
:10902000903023F00103C6F8903007464FF0B04867
:1090300041F28836D8F890309B07BDD5FAF78CFD01
:10904000C31BB342F6D993E6FAF786FDC01B404531
:10905000DFD98DE60C2D4ED0022B4FF0B0431A68AD
:1090600022F080721A6033D1FAF776FD0546FFF7D9
:10907000DEFC38BBD4E90C314FF0B0420B43D06872
:109080002D4901400B43E16B0B43216C0B43616C99
:109090000B43A16B43EA0123D360136843F0807351
:1090A0001360D36843F08053D360FAF755FD04464C
:1090B000FFF7BDFC002882D1FAF74EFD001B0A28FD
:1090C000F6D955E6FAF748FD401B0A28CFD94FE6F6
:1090D000FAF742FD0446FFF7AAFC30B94FF0B04260
:1090E000164BD1680B40D36069E7FAF735FD001BDA
:1090F0000A28F0D93CE6012B3FF4E1AD4FF0B04334
:10910000D868236B00F003029A427FF4D8AD626BFB
:1091100000F0700393427FF4D2ADA26B00F4FE43E3
:10912000B3EB022F7FF4CBAD636C00F06040C01A4C
:1091300018BF0120AEE500BF8C80C111FCFFFEEE20
:109140002DE9F0410D46044610B90120BDE8F0813B
:10915000684E336803F007038B4216D323689A07DF
:1091600027D54FF0B047A268BB6823F0F003134344
:10917000BB60FAF7F1FC0646BB68DB0319D4FAF7CB
:10918000EBFC831B022BF7D911E0336823F00703B4
:109190000B433360FAF7E0FC0746336803F007033C
:1091A000AB42DBD0FAF7D8FCC01B0228F5D903206C
:1091B000CCE72368580617D54FF0B0476269D7F857
:1091C000083123F00F0343EA1213C7F80831FAF706
:1091D000C3FC0646D7F80831D90305D4FAF7BCFC1E
:1091E000831B022BF6D9E2E723685A0713D54FF009
:1091F000B047E268BB6823F4E0631343BB60FAF74F
:10920000ABFC0646BB689B0305D4FAF7A5FC831BA1
:10921000022BF7D9CBE72368180714D54FF0B047D6
:109220002269BB6823F4605343EAC203BB60FAF7C8
:1092300093FC0646BB68590305D4FAF78DFC831BE3
:10924000022BF7D9B3E72368DA070FD4294C236838
:1092500003F00703AB4239D8FFF7C8FC264B186070
:10926000264BBDE8F0411868FAF774BC6268022A20
:109270001DD1FFF7C7FB00283FF467AF4FF0B046A2
:1092800041F28838B36823F003031343B360FAF75D
:1092900063FC0746B368626803F00C03B3EB820F0C
:1092A000D4D0FAF759FCC01B4045F3D97FE7032A15
:1092B00002D1FFF7BCFBDEE712B9FFF7A9FBDAE743
:1092C0004FF0B0431B685B05D8D43EE7236823F01A
:1092D00007032B432360FAF73FFC0646236803F09D
:1092E0000703AB42B8D0FAF737FC801B0228F5D948
:1092F0005DE700BF00400058A8030020AC03002039
:1093000008B5FFF773FC4FF0B043044A9B68C3F302
:10931000022352F82330D84008BD00BFC0800308A4
:1093200008B5FFF763FC4FF0B043044A9B68C3F3F2
:10933000C22352F82330D84008BD00BFC0800308C4
:109340004FF0B043D3F89000C0F3400070474FF0A7
:10935000B0410209D1F8883002F47F22000123EAEB
:10936000020300F47F200343C1F8883070474FF0B8
:10937000B041020CD1F88830120423EA020343EA18
:109380000040C1F8880070470368DA0370B50446EE
:1093900039D5FFF7C3FAFAF7DFFB614E05463368AC
:1093A000DB0532D54FF0B043616BD3F8902002F467
:1093B000407291421DD0D3F89010D3F8902042F41F
:1093C0008032C3F89020D3F8902021F4407022F42A
:1093D00080328D07C3F89020C3F8900009D5FAF7C2
:1093E000BBFB41F288360546FFF7AAFF012840F093
:1093F00090804FF0B042616BD2F8903023F440730C
:109400000B43C2F89030002605E0FAF7A5FB401B9D
:109410000228C4D903262568E8070AD54FF0B041D1
:109420006268D1F8883023EA124392B21343C1F83C
:109430008830A9070AD54FF0B041A268D1F888302A
:1094400023EA124392B21343C1F88830AA0609D521
:109450004FF0B0422169D2F8883023F440630B43C7
:10946000C2F88830AB0502D5206AFFF780FF680597
:1094700002D5606AFFF77BFF290502D5A06AFFF7D6
:1094800076FF6A0602D56069FFF761FF2B0602D5F9
:10949000A069FFF75CFFE80502D5E069FFF757FF19
:1094A000E90610D54FF0B042E168D2F8883023F4D5
:1094B00040730B43C2F88830B1F5807F02BFD36898
:1094C00043F08073D3602A040ED54FF0B042216B75
:1094D000D2F8883023F040430B43C2F8883019B9E2
:1094E000D36843F08073D3606B0410D54FF0B04263
:1094F000E16AD2F8883023F040530B43B1F1005FAA
:10950000C2F8883003D1D36843F48033D360304647
:1095100070BDFAF721FB401BB0427FF665AF79E7DB
:109520000004005830B590F82C30012B02464FF063
:10953000020022D0174B82F82D00CA24012582F8A0
:109540002C505C6253245C62B1F5807F146B996986
:1095500014D121F488519961596C24F0010421F04F
:10956000004159641463DD650A4BFF2159620020F4
:10957000012382F82D3082F82C0030BD21F40851EF
:109580009961D96C24F0020421F00041D96414637C
:10959000D865E9E70028004070B50B4E036B756D88
:1095A0001D40EA07044603D50123F365FAF767FD7A
:1095B000AB0704D50223F365204600F0C9F9012367
:1095C00084F82D3070BD00BF0028004038B50A4C2B
:1095D000E36823F02003E360FAF7BEFA0546E36888
:1095E0009B0601D5002038BDFAF7B6FA401BB0F54E
:1095F0007A7FF4D90320F6E700280040F8B5114D32
:10960000EC6814F0400406461AD1EB6843F080037E
:10961000EB60FAF7A1FA23460746EC6814F0400421
:1096200001D1032B01D11846F8BDFAF795FAC01BFA
:10963000B0F57A7F234684BF032386F82D30ECE70C
:109640000023F0E70028004038B50F4CE36823F012
:109650008003E360A3699B06054606D4FFF7B6FFC7
:1096600010B1032085F82D0038BDA36923F0200335
:10967000A361FFF7ABFF10B1032085F82D00A369AC
:1096800043F02003A361EFE70028004038B504460B
:1096900000284BD090F82D3003F0FF021BB980F862
:1096A0002C20F9F787FD0223214D84F82D30EB683B
:1096B000DB0636D4CA236B6253236B622046FFF766
:1096C0009DFF10B1FF236B6238BDAB6923F08E6341
:1096D00023F04003AB6121696368AA690B4313431C
:1096E000A2691343AB61D4E9022343EA02432B612D
:1096F000D4E90931EA680B4322F4F8521343EB60D2
:109700002046FFF7A1FF0028DCD1D4E90713AA699E
:109710000B4322F06042134362691343AB61FF23A2
:109720006B62012384F82D300020CDE70120CBE7C8
:10973000002800400023092803D840EA0310C0B2E3
:1097400070470A380133C0B2F5E700002DE9F04751
:1097500090F82C30012B05464FF0020069D0012310
:1097600085F82C304E4B85F82D00DE6806F44076E7
:10977000B6F5807F78D04C69087891F8019091F81F
:1097800002A091F82470002A55D19B6913F0400380
:1097900008BFCB70FFF7CEFF80464846FFF7CAFFF1
:1097A00002465046FFF7C6FF81463846FFF7C2FF24
:1097B0000B6ACF78234343EA875343EA090343EA1A
:1097C000084343EA022343EA0063354ACA20506251
:1097D000532050628C6A8869B4F5807F946945D1C2
:1097E00024F4885494610124D465B6F5807F09BFC0
:1097F000CB6913640343536418BF5064284B4A6811
:109800001A672A6B42F001022A639A6942F488526D
:109810009A61244AD2F8803043F40033C2F8803091
:109820001F4BFF225A620020012385F82D3085F856
:109830002C00BDE8F087B4F1803F07D0B4F5000FED
:1098400004D09B6913F0400308BFCB700B6ACA7841
:109850001C4344EA0A0444EA004343EA092343EA76
:10986000825343EA0763B0E70023AEE724F40854C9
:1098700094610224D465B6F5807F09BFCB699364F7
:109880000343D36418BFD064054B4A685A672A6BF8
:1098900042F002022A639A6942F40852B8E700BF14
:1098A000002800400008005890F82C20012A0346A8
:1098B0004FF0020012D00A4A83F82D00CA215162EB
:1098C00053215162916941F020019161FF21516260
:1098D0000020012283F82D2083F82C00704700BF60
:1098E0000028004090F82C20012A03464FF0020087
:1098F00019D00D4A83F82D00CA21516253215162BB
:1099000091690A4841F080019161D0F8801041F4DA
:109910008021C0F88010FF2151620020012283F8CD
:109920002D2083F82C0070470028004000080058C4
:10993000064B5A6D520610B5044603D54022DA652F
:10994000FAF7A0FB012384F82D3010BD0028004059
:109950007047890001F1804101F531410A6070478B
:10996000890001F1804101F531410868704700002C
:109970002DE9F3471F46894690460446FAF7ECF86E
:109980000A9D3D442D1AFAF7E7F8264B1E68C6F3E8
:10999000CB366E43824601962268936839EA030308
:1099A0000CBF01230023434501D100202EE07B1C86
:1099B000F3D0FAF7D1F8A0EB0A00A84229D3236824
:1099C0005A6822F0E0025A606268B2F5827F0AD1DA
:1099D000A268B2F5004F02D0B2F5806F03D11A68C9
:1099E00022F040021A60A26AB2F5005F07D11A683D
:1099F00022F400521A601A6842F400521A600123DD
:109A000084F85D30002384F85C30032002B0BDE8A8
:109A1000F087019A019B002A03F1FF33019308BFED
:109A20001546B9E7A80300202DE9F74F9946002312
:109A30008DF80330044688461746FAF78DF80C9DDA
:109A40004D442D1AFAF788F82C4BD4F800B01E6854
:109A500023235E43360D6E43824601962268936847
:109A600003EA0803BB4201D100203AE0B8F5C06F19
:109A700007D137B99BF80C30DBB28DF803309DF875
:109A80000330B9F1FF3FEAD0FAF766F8A0EB0A001D
:109A9000A84229D323685A6822F0E0025A6062681B
:109AA000B2F5827F0AD1A268B2F5004F02D0B2F5BA
:109AB000806F03D11A6822F040021A60A26AB2F5E0
:109AC000005F07D11A6822F400521A601A6842F443
:109AD00000521A60012384F85D30002384F85C3062
:109AE000032003B0BDE8F08F019A019B002A03F127
:109AF000FF33019308BF1546B0E700BFA80300205D
:109B000073B50B4600920D4616464FF4C051002225
:109B10000446FFF789FF024630B1236E43F020036D
:109B20002366032002B070BD00962B46802120469C
:109B3000FFF71EFF02460028EFD100962B464FF498
:109B4000C0612046FFF770FF0028EBD0E5E74368CF
:109B5000B3F5827FF7B504460E4617460BD18368EE
:109B6000B3F5004F02D0B3F5806F04D122681368BB
:109B700023F04003136000973346002280212046E3
:109B8000FFF7F6FE054628B1236E43F02003236657
:109B9000032514E06368B3F5827F10D1A368B3F5A1
:109BA000004F02D0B3F5806F09D1009733460022F1
:109BB0004FF4C0612046FFF737FF0028E4D1284664
:109BC00003B0F0BDF8B5044600287ED0436A002BF0
:109BD00050D14268B2F5827F00D0C36194F85D3005
:109BE00003F0FF0223B984F85C202046F9F748FB14
:109BF0002268E068022384F85D301368B0F5E06FF6
:109C000023F0400313604FF0000337D91D46B0F531
:109C1000706F18BFA362A7686368A169A66A07F49A
:109C2000044703F482733B43276907F002073B4371
:109C3000676907F001073B4301F400773B43E7699D
:109C400007F038073B43276A07F080073B4306F4D9
:109C500000573B43B6F5005F136014D1236B8BBBF9
:109C6000B0F5E06F0DD902232363136843F400635A
:109C7000136008E00023C0E90433AFE74FF48055D8
:109C8000C7E701232363636A676B03F0100307F0E0
:109C9000080700F470603B43090C034301F0040122
:109CA0000B432B43B6F5005F536004BFA38D1361D4
:109CB000D36923F40063D36100200123206684F874
:109CC0005D30F8BD022BDED1CFE70120F9E70000BF
:109CD00070B5044690F85C00012800F0CF800120A8
:109CE00084F85C0094F85D0066680128C5B20AD06B
:109CF000B6F5827F40F0C080A068002840F0BC80AC
:109D0000042D40F0B980002951D0002A4FD0002BFB
:109D10004DD094F85D00A16304281CBF052084F891
:109D20005D0000202066C4E91300A06AE387B0F557
:109D3000005F2168A3872264A4F84430A4F8463069
:109D400007D1086820F400500860086840F400500B
:109D50000860486820F4C0404860E068B0F5E06FF3
:109D6000A06D29D94B6823F480534B6094F85D3083
:109D7000434E444D042B444B18BF1D46434B18BF64
:109D80003346C0E90B35424B436300238363B4F889
:109D900046300C319BB2FEF785FA0346002848D0C6
:109DA000236E43F010032366012384F85D30012005
:109DB000002384F85C3070BD4D6845F480554D60DB
:109DC000656DAD69B5F5806F0AD113F0010F4B6871
:109DD0001ED123F480434B60E38FC3F34E03E3872C
:109DE0008369B3F5806FC1D14B6823F480534B6016
:109DF000B4F8463013F0010F4B6811D123F400532F
:109E00004B60B4F84630C3F34E03A4F84630ADE7D8
:109E100043F480434B60E38FC3F34E030133DEE72B
:109E200043F400534B60B4F84630C3F34E030133A0
:109E3000EBE72268606D516841F001015160C0E9B3
:109E40000B33C0E90D33E38FA16B9BB20C32FEF7ED
:109E500029FA0028A4D123681A6852065EBF1A683E
:109E600042F040021A605A6842F020025A605A6872
:109E700042F002025A609BE7022099E702209AE72B
:109E8000C99F0008999E0008A59E0008D39E00085F
:109E9000B19E00087047704708B5806AFFF7FBFF66
:109EA00008BD704708B5806AFFF7FBFF08BD704723
:109EB000806A026808B5536823F003035360036E99
:109EC00043F010030366012380F85D30FFF7EFFFD6
:109ED00008BD7FB5064600230393846A8DF80B30D6
:109EE000F9F73AFE33681B689A06054668D422687B
:109EF000536823F020035360A36AB3F5005F13D1C6
:109F000001220090642311462046FFF731FD18B16D
:109F1000236E43F002032366E3682668B3F5E06F1F
:109F20002ED9F3680393039BA2682368002A43D1C8
:109F30006268B2F5827F3FD15A6822F003025A600C
:109F400064212A462046FFF702FE08B1202323663B
:109F50000023A4F846302268012384F85D3093681A
:109F6000DB0606D5236E43F0020323664FF6EF733C
:109F70009360236E23B32046FFF799FF04B070BDB2
:109F8000337BDBB28DF80B309DF80B30236B022B4B
:109F9000CAD101220095642311462046FFF7E8FC50
:109FA00018B1236E43F002032366337BDBB28DF8D6
:109FB0000B309DF80B30B7E75A6822F00102BEE77C
:109FC0002046FFF767FFD9E77FB5064600230393D6
:109FD000846A8DF80B30F9F7BFFD33681B6899066A
:109FE00005465ED42268536823F020035360A36AB9
:109FF000B3F5005F1BD1E368B3F5E06F3ED1236B8F
:10A00000012B3BD1009064234FF400724FF4C061E8
:10A010002046FFF709FD18B1236E43F002032366C3
:10A0200023681B7BDBB28DF80B309DF80B302A4682
:10A0300064212046FFF764FD18B1236E43F020032E
:10A04000236623685A6822F003025A600022E287DE
:10A05000A4F84620012284F85D209A68D20606D52D
:10A06000226E42F0020222664FF6EF729A60236E71
:10A07000BBB12046FFF71BFF04B070BD0095642301
:10A080004FF480624FF4C0612046FFF7CDFC18B159
:10A09000236E43F0020323662368DB680393039B6C
:10A0A000C5E72046F8F708FCE6E70000036830B58E
:10A0B00059689A6802F04105012D85B0044606D121
:10A0C0004D0604D5C36C05B0BDE830401847950770
:10A0D00004D5080602D5236D2046F4E712F4B07FBC
:10A0E00059D08D0657D550060FD594F85D0003283A
:10A0F0004FF0000549D0206E40F004002066009526
:10A10000D868009098680090009895060CD5206E4D
:10A1100040F00100206600200290986802901868C4
:10A1200020F0400018600298D00508D5226E42F059
:10A1300008022266002203929A680392039A226E12
:10A140004AB35A6822F0E0025A60012284F85D2086
:10A150008A0722D05A68A06D22F003025A6040B1EB
:10A16000104B8363FEF717F918B1236E43F04003D9
:10A170002366606D78B10B4B8363FEF70CF950B129
:10A18000236E43F04003236605E00195DA680192EF
:10A190009B680193019B05B030BD2046FFF787FE09
:10A1A000F9E700BFA9A1000808B5806A0023A0F85C
:10A1B0004630C387FFF77BFE08BD0000034AD2F894
:10A1C000903043F40043C2F89030704700040058C8
:10A1D000034AD2F8903023F40043C2F8903070471D
:10A1E00000040058074B1A6822F040021A6040F43D
:10A1F00041704FF4B85218605A601A6842F0400239
:10A200001A6070470000015837B5054600284ED047
:10A21000837903F0FF046BB1032C0BD0254B4FF473
:10A2200000629A612868FFF7DDFF002401232B718B
:10A23000AC602FE000236B712846F9F7A1FB1E4AA2
:10A24000D2F8903043F48053C2F89030002CE5D11E
:10A2500002234FF0B042AB71D2F8943023F40043A4
:10A26000C2F89430154B1B681C214B43DB0C642156
:10A270004B430193019B93B90124AC60FFF79EFF10
:10A280000C4B9A6842F400629A604FF400629A6143
:10A29000002CC7D00123AB71204603B030BD019B19
:10A2A000013B0193D2F894305B04E3D4E6E7012448
:10A2B000F2E700BF0004005800080058A80300207F
:10A2C00037B5174D2B6802461C204343DB0C642036
:10A2D000434314480193019B93B901209060114CB2
:10A2E00021732B681C214B43DB0C64214B430193EE
:10A2F000019B6BB9012090600A4BDB6803B030BD55
:10A30000019B013B019383689C07E4D50020E6E7AD
:10A31000019B013B0193A368DB07E9D5ECE700BF94
:10A32000A80300200000015837B5184D2B680246DD
:10A330001C204343DB0C6420434315480193019BDD
:10A34000A3B901209060124CFF2323732B681C25B6
:10A350006B43DB0C64256B430193019B73B90120B4
:10A3600090600B4BDB680B7003B030BD019B013B71
:10A37000019383689C07E2D50020E4E7019B013B41
:10A380000193A368DB07E8D5EBE700BFA803002033
:10A39000000001580E4B0F491B681822534382B02E
:10A3A0001B0D6422534301934B69019AC3F380034D
:10A3B00022B902238360012002B07047019A013A5A
:10A3C00001924A69920701D5002BEDD10020F3E7F5
:10A3D000A80300200004005807B50379012B0FD112
:10A3E0000A4B1B68182253431B0C0193FFF7F0FE26
:10A3F000019B013B0193019B002BF9D1FFF7DEFE8E
:10A4000003B05DF804EBFFF7C5BF00BFA803002051
:10A41000F8B51E468379012B154604460F46DAB27D
:10A420002DD14379012B2AD0022342718371FFF78A
:10A43000D3FF0D212046FFF7CBFEFFF741FF390A7E
:10A440002046FFF73DFFF9B22046FFF739FF2E44C3
:10A45000B5420ED12046FFF7B1FEFFF79BFFA06883
:10A4600001230038A3714FF0000318BF012063716E
:10A47000F8BD15F8011B2046FFF722FFE8E7022090
:10A48000F6E7F8B51E468379012B154604460F46BC
:10A49000DAB22FD14379012B2CD04271FFF79CFF08
:10A4A0001D212046FFF794FEFFF70AFF390A2046D8
:10A4B000FFF706FFF9B22046FFF702FF0021204612
:10A4C000FFF7FEFE2E44B5420ED12046FFF776FE82
:10A4D000FFF760FFA06801230038A3714FF000036D
:10A4E00018BF01206371F8BD29462046FFF71CFF05
:10A4F0000135E8E70220F6E7F8B51F468379012B1E
:10A50000154604460E46DAB22CD14379012B29D0E8
:10A510004271FFF761FF06F0EF03A3F1840253429B
:10A520005341237131462046FFF752FEFFF7C8FE24
:10A530002F44AF4210D1FFF741FE842E02D02046B7
:10A54000FFF728FFA06801230038A3714FF0000334
:10A5500018BF01206371F8BD15F8011B2046FFF7F5
:10A56000AFFEE6E70220F6E7F8B51E468379012B39
:10A57000154604460F46DAB227D14379012B24D081
:10A580004271FFF729FF39462046FFF721FEFFF70A
:10A5900097FE00212046FFF793FE2E44B5420ED1D0
:10A5A0002046FFF70BFEFFF7F5FEA06801230038F9
:10A5B000A3714FF0000318BF01206371F8BD294655
:10A5C0002046FFF7B1FE0135E8E70220F6E737B590
:10A5D0000023ADF8043001AA022312210546FFF73B
:10A5E000C3FFBDF80440022364BA01AAA4B219460D
:10A5F0002846FFF781FFE20702D528460AF094FFBC
:10A60000A30702D528460AF095FF600702D5284621
:10A610000AF0BAFF210702D528460AF0BBFFE2067E
:10A6200002D528460AF0BCFFA30602D528460AF048
:10A63000A5FF600602D528460AF082FF210606D54E
:10A6400014F4807118BF012128460AF07FFFA2058B
:10A6500002D528460AF08AFF630402D528460AF08C
:10A66000A5FF03B030BDF8B51E468379012B154612
:10A6700004460F46DAB227D14379012B24D0427128
:10A68000FFF7AAFE0E212046FFF7A2FDFFF718FEF6
:10A6900039462046FFF714FE2E44B5420ED120461F
:10A6A000FFF78CFDFFF776FEA06801230038A37149
:10A6B0004FF0000318BF01206371F8BD15F8011BAE
:10A6C0002046FFF7FDFDE8E70220F6E7F8B51E4655
:10A6D0008379012B154604460F46DAB22BD1437914
:10A6E000012B28D04271FFF777FE1E212046FFF78D
:10A6F0006FFDFFF7E5FD39462046FFF7E1FD00213C
:10A700002046FFF7DDFD2E44B5420ED12046FFF76F
:10A7100055FDFFF73FFEA06801230038A3714FF0FD
:10A72000000318BF01206371F8BD29462046FFF7DA
:10A73000FBFD0135E8E70220F6E70000036A23F09D
:10A7400001030362036A70B5446882690D6822F4EC
:10A75000803222F073022A438D6823F002032B43D8
:10A76000124DA84206D0124EB04203D0A6F5806624
:10A77000B04214D1CE6823F008033343A84223F03B
:10A78000040306D00B4DA84203D005F58065A8420E
:10A7900005D124F44075D1E9054634432C43446087
:10A7A00082614A684263036270BD00BF002C0140B1
:10A7B0000048014000440140036A23F480730362AF
:10A7C000036A426870B5C4690D6824F4803424F0CB
:10A7D00073042C438D6823F4007343EA05230F4D63
:10A7E000A8420ED1CD6823F4006343EA052323F485
:10A7F0008063D1E9055622F44052354342EA0512FE
:10A8000006E0074DA842F4D005F58065A842F0D0D7
:10A8100042604A68C461C263036270BD002C01409B
:10A8200000440140036A23F480530362026A30B596
:10A830004468C3690D6823F0807323F4E64343EA58
:10A8400005238D6822F4005242EA05320A4DA842DF
:10A8500007D005F5C055A84203D005F58065A8428C
:10A8600004D14D6924F4804444EA85144460C361F2
:10A870004B680364026230BD002C0140036A23F47C
:10A8800080330362026A30B54468436D0D6823F477
:10A89000803323F070032B438D6822F4003242EAA8
:10A8A00005420B4DA84207D005F5C055A84203D07C
:10A8B00005F58065A84204D14D6924F4803444EA4A
:10A8C0000524446043654B688365026230BD00BF68
:10A8D000002C0140036A23F480130362026A30B53E
:10A8E0004468436D0D6823F0807323F4E04343EA2A
:10A8F00005238D6822F4001242EA05520A4DA8424F
:10A9000007D005F5C055A84203D005F58065A842DB
:10A9100004D14D6924F4802444EA852444604365CD
:10A920004B68C365026230BD002C0140704710B512
:10A93000846A626A82420BD101232377D2690AB901
:10A9400084F83E302046F8F7DFFF0023237710BD60
:10A95000A36A834208D102222277DB69002BF1D15E
:10A96000012384F83F30EDE7E36A834208D10422F3
:10A970002277DB69002BE5D1012384F84030E1E741
:10A98000236B8342DED108222277DB69002BD9D1E9
:10A99000012384F84130D5E7704710B5846A636AB3
:10A9A000834207D1012323772046FFF7F5FF0023D9
:10A9B000237710BDA36A834201D10223F3E7E36A40
:10A9C000834201D10423EEE7236B8342ECD10823B9
:10A9D000E9E7704710B5846A636A834209D10123AD
:10A9E000237784F83E302046FFF7F3FF00232377D8
:10A9F00010BDA36A834205D102232377012384F883
:10AA00003F30F0E7E36A83424FF0010304D10422B0
:10AA1000227784F84030E6E7226B824203BF0822A7
:10AA2000227784F8413084F83D30DCE71A4A036825
:10AA3000904210B502D0B0F1804F09D14C6823F09C
:10AA40007003904243EA040309D0B0F1804F06D06E
:10AA5000124A904203D002F58062904203D1CA6844
:10AA600023F4407313434A6923F0800313430360C4
:10AA70008B68C3620B688362074B984207D003F56B
:10AA8000C053984203D003F58063984201D10B690B
:10AA900003630123436110BD002C014000440140C9
:10AAA00010B5044650B390F83D3003F0FF021BB9D7
:10AAB00080F83C20F9F728F90223206884F83D301B
:10AAC000211DFFF7B3FF012384F84830002084F8EC
:10AAD0003E3084F83F3084F8403084F8413084F8C8
:10AAE000423084F8433084F8443084F8453084F8A8
:10AAF000463084F8473084F83D3010BD0120FCE733
:10AB000010B5044650B390F83D3003F0FF021BB976
:10AB100080F83C20FFF70AFF0223206884F83D30CC
:10AB2000211DFFF783FF012384F84830002084F8BB
:10AB30003E3084F83F3084F8403084F8413084F867
:10AB4000423084F8433084F8443084F8453084F847
:10AB5000463084F8473084F83D3010BD0120FCE7D2
:10AB6000036A23F010030362036A426870B58469C4
:10AB70000D6824F0807424F4E64444EA05248D68CA
:10AB800023F0200343EA05130F4DA8420ED1CD68F0
:10AB900023F0800343EA051323F04003D1E905566F
:10ABA00022F44062354342EA850206E0074DA8429E
:10ABB000F4D005F58065A842F0D042604A6884610F
:10ABC0008263036270BD00BF002C0140004401405D
:10ABD00038B590F83C30012B044673D001200C2A84
:10ABE00084F83C004ED008D8042A2BD0082A39D04B
:10ABF000BAB1002384F83C3038BD102A52D0142A50
:10AC0000F7D12068FFF766FE436D0A6943F40063DD
:10AC10004365436D23F480634365436D43EA022338
:10AC20004EE02068FFF78AFD83690A6943F0080354
:10AC30008361836923F00403836183691343836120
:10AC40000020D6E72068FFF78BFF83690A6943F489
:10AC500000638361836923F480638361836943EACA
:10AC60000223ECE72068FFF7A7FDC3690A6943F0F8
:10AC70000803C361C36923F00403C361C3691343B9
:10AC8000C361DDE72068FFF7CDFDC3690A6943F4BE
:10AC90000063C361C36923F48063C361C36943EA8A
:10ACA0000223EDE72068FFF7E9FD436D0A6943F0F1
:10ACB00008034365436D23F004034365436D134369
:10ACC0004365BDE7022097E710B584680A4324F482
:10ACD0007F4442EA03222243826010BD38B590F8D7
:10ACE0003C30012B04464FF0020000F0958084F8C0
:10ACF0003D000122206884F83C208568474B2B40AA
:10AD000083600B68602B54D037D8402B6BD019D898
:10AD1000202B0DD00AD833F0100109D0012384F87C
:10AD20003D30002384F83C30104638BD302BF5D13F
:10AD3000826822F4401222F070021A4342F00702A5
:10AD400082602BE0502BE9D14A68CD68016A036A22
:10AD500023F001030362836921F00A0123F0F00369
:10AD600043EA05130A4383610262836823F44013B4
:10AD700023F0700343F057030FE0B3F5805F0DD06D
:10AD8000B3F5005F0CD0702BC8D1CB68D1E901219D
:10AD9000FFF79AFF836843F0770383600022BDE7E3
:10ADA000CB68D1E90121FFF78FFF836843F480432B
:10ADB000F3E7036A4D68C96823F0100303628269F0
:10ADC000036A22F4704223F0A00343EA051342EA27
:10ADD000013282610362836823F4401323F070031D
:10ADE00043F06703D9E74A68CD68016A036A23F034
:10ADF00001030362836921F00A0123F0F00343EAAF
:10AE000005130A4383610262836823F4401323F02D
:10AE1000700343F04703C0E7024685E78800CEFF92
:10AE2000036A01F01F0110B501248C4023EA0403DA
:10AE30000362036A8A401A43026210BD38B50D46A8
:10AE4000082D044611461BD005D85DB1042D14D041
:10AE500094F8430008E00C2D15D0102DF8D190F88F
:10AE6000420001E090F83E00A0F1020CDCF100008D
:10AE700040EB0C0050B1022076E090F83F00F3E781
:10AE800090F84000F0E790F84100EDE7082D1AD067
:10AE900007D86DB1042D13D094F84320012A19D09E
:10AEA0000CE00C2D27D0102DF6D194F842000CE0C8
:10AEB00094F83E20501E424242415AB9012053E0CC
:10AEC00094F83F20F6E794F84000421E504250416B
:10AED0000028F3D00029F1D0002BEFD0082D4FF03F
:10AEE000020256D00AD885B1042D3ED0042D84F834
:10AEF0004320E3D13BE094F84100E6E70C2D5CD021
:10AF0000102DF3D184F84220D8E7606A84F83E20FF
:10AF10003A4AC2623A4A02633A4A42632268343287
:10AF2000FDF7C0F90028C9D12268D36843F4007343
:10AF30002068D36029460122FFF772FF324A90420F
:10AF400050D0324B98424DD003F58063984249D09F
:10AF5000B0F1804F4DD182682D4B1340062B02D0AB
:10AF6000B3F5803F45D1002038BD84F83F20A06A6A
:10AF7000224AC262224A0263224A4263226838326B
:10AF8000FDF790F9002899D12268D36843F48063D3
:10AF9000CEE7E06A84F84020184AC262184A026389
:10AFA000184A426322683C32FDF77CF9002885D1BB
:10AFB0002268D36843F40063BAE7206B84F8412029
:10AFC0000E4AC2620E4A02630E4A4263226840324F
:10AFD000FDF768F900287FF471AF2268D36843F465
:10AFE0008053A5E7436C904243F400434364B2D0DE
:10AFF000AEE7036843F001030360B4E72FA900083C
:10B000009BA90008D5A90008002C0140004401407C
:10B0100007000100FFF712BF082938B504460D46A6
:10B020004FD004D861B1042944D0012038BD0C2987
:10B03000FBD10268006BD36823F48053D36005E032
:10B040000268406AD36823F40073D360FDF7A3F964
:10B05000206800222946FFF7E3FE2A4B984207D0DA
:10B0600003F5C053984203D003F5806398420DD195
:10B07000026A41F211131A4208D1026A40F24443B3
:10B080001A4202BF436C23F400434364026A41F254
:10B0900011131A4208D1026A40F244431A4202BF15
:10B0A000036823F00103036001238DB984F83E3067
:10B0B0000020BBE70268806AD36823F48063D36012
:10B0C000C4E70268C06AD36823F40063D360BDE7B5
:10B0D0000C2D13D007D8042D0AD0082D0BD0012336
:10B0E00084F84330E4E7102DF9D184F84230DFE7EB
:10B0F00084F83F30DCE784F84030D9E784F8413009
:10B10000D6E700BF002C0140FFF786BF70B590F86E
:10B110003C30012B02464FF0020020D082F83D0067
:10B120000F4D106843688468A84202BF4E6823F43C
:10B13000700333430E6823F070033343A842436027
:10B1400002D0B0F1804F04D1896824F080030B4312
:10B1500083600123002082F83D3082F83C0070BDFE
:10B16000002C014010B590F83C30012B02463BD03A
:10B17000CB6888681D4C23F440730343486823F46C
:10B1800080630343086823F400630343086923F4DE
:10B1900080530343486923F400530343086B23F4AB
:10B1A00080430343886923F4702343EA0043106813
:10B1B000A04214D1CC6923F0805323438C6A23F43A
:10B1C000700343EA04530C6A23F0807323434C6AF0
:10B1D000C96A23F00073234323F000530B434364F5
:10B1E000002082F83C0010BD0220FCE7002C01404A
:10B1F000026852E8003F23F0C00342E800310268D1
:10B200000029F5D102F1080353E8003F23F40003BD
:10B2100002F1080C4CE800310029F3D12023C0F8DA
:10B220008830704710B5026852E8003F23F49073ED
:10B2300042E8003102680029F5D10F4C02F1080301
:10B2400053E8003F234002F1080C4CE8003100298C
:10B25000F4D1C36E012B07D152E8003F23F0100355
:10B2600042E800310029F7D12023C0F88C300023B8
:10B27000C366436710BD00BFFEFFFFEFF8B504468D
:10B280001346D4F88850202D32D1F1B1EAB1E06FE5
:10B29000A4F85620A4F8542000262122C4F8906077
:10B2A0002165C4F88820226888B1124FC762124F06
:10B2B0000763124F2832C0E90D76FCF7F3FF30B177
:10B2C0001023C4F89030C4F888500120F8BD2368DA
:10B2D00040221A62226802F1080353E8003F43F05B
:10B2E000800302F1080141E800300028F3D1EDE7C6
:10B2F0000220EBE701B3000849B3000855B300088A
:10B3000008B50346806A1B681B6813F0200317D139
:10B31000A0F85630026802F1080353E8003F23F01A
:10B320008003083242E8003102680029F2D152E875
:10B33000003F43F0400342E800310029F7D108BD47
:10B34000F8F7D4FFFBE7704708B5806AFFF7FBFF0B
:10B3500008BD7047806A38B50468D0F88830D0F8E6
:10B360008C50A268120606D5212B04D10023A0F828
:10B370005630FFF73DFFA3685B0606D5222D04D1AA
:10B380000023A0F85E30FFF74DFFD0F8903043F077
:10B390001003C0F89030FFF7DCFF38BD08B5806AB5
:10B3A0000023A0F85E30A0F85630FFF7D2FF08BDAA
:10B3B000704700000368D9691A682DE9F04140F62A
:10B3C0000F0631429D68044610D18E0640F19780E9
:10B3D00002F0200605F080573E4300F09080436F56
:10B3E000002B00F08580BDE8F0411847AB4EAC481B
:10B3F0002E401040304300F08280CF0709D5D005A1
:10B4000007D501201862D4F8900040F00100C4F87C
:10B4100090008F0709D5E80707D502201862D4F8F5
:10B42000900040F00400C4F890004F0709D5E807E9
:10B4300007D504201862D4F8900040F00200C4F848
:10B4400090000F070BD502F02000304307D00820F2
:10B450001862D4F8900040F00800C4F890000E057F
:10B460000AD5500108D54FF400601862D4F8903026
:10B4700043F02003C4F89030D4F89030002B37D03C
:10B480008B0609D502F0200205F080552A4303D02F
:10B49000636F0BB1204698472668D4F89020B368B4
:10B4A00002F0280203F0400353EA0205204621D0AF
:10B4B000FFF7B8FEB3685F0617D5226802F10803EC
:10B4C00053E8003F23F04003083242E800310029EE
:10B4D000F3D1D4F8800040B1724B8363FCF75BFF7B
:10B4E00030B1D4F88000836B7DE72046FFF731FF51
:10B4F000BDE8F081FFF72DFFC4F89050F8E7E06E4B
:10B50000012840F08980CE0640F18680D00640F1C7
:10B51000838010221A629A6851064BD5D4F8802095
:10B5200011684A6892B2002AE2D0B4F85C009042F6
:10B53000DED9A4F85E200A6892062FD453E8002FC3
:10B5400022F4807243E800210029F7D103F10802B8
:10B5500052E8002F22F0010203F1080040E8002128
:10B560000029F3D103F1080252E8002F22F0400233
:10B5700003F1080040E800210029F3D12022C4F89B
:10B580008C20E16653E8002F22F0100243E80021EE
:10B590000029F7D1D4F88000FCF7C8FE0223236706
:10B5A000B4F85E30B4F85C10C91A89B22046FFF7CF
:10B5B000FFFE9DE7B4F85E20B4F85E00B4F85C10BE
:10B5C00080B292B2002893D0891A89B200298FD014
:10B5D00053E8002F22F4907243E800200028F7D1AE
:10B5E000314D03F1080252E8002F2A4003F108060A
:10B5F00046E800200028F4D12022C4F88C2060679F
:10B60000E06653E8002F22F0100243E800200028F3
:10B61000F7D102232367C9E7CF0209D56E0207D508
:10B620004FF4801220461A62BDE8F04100F0A0BD40
:10B6300008060BD502F0800005F40005284305D06C
:10B64000A36F002B3FF454AF2046CCE64F0611D534
:10B6500056060FD553E8002F22F0400243E80021A0
:10B660000029F7D12023C4F88830A1672046F8F7D5
:10B670003DFE3DE70D0206D5500004D52046BDE84D
:10B68000F04100F077BDCB017FF532AF002ABFF665
:10B690002FAF2046BDE8F04100F06BBD0100001067
:10B6A000200100049DB30008FEFFFFEFD0F88C20BE
:10B6B000B0F86010222A08B5036855D15B6A826D24
:10B6C0000B401370836D01338365B0F85E30013B2E
:10B6D0009BB2A0F85E30B0F85E309BB2002B42D136
:10B6E000026852E8003F23F4907342E80031036897
:10B6F0000029F5D103F1080252E8002F22F00102DF
:10B7000003F1080C4CE800210029F3D12022C0F8F5
:10B710008C20184A41679342016705D1C26E012A05
:10B720000ED0F8F7F1FD1EE05A681102F6D553E885
:10B73000002F22F0806243E800210029F7D1EDE7D5
:10B740000022C26653E8002F22F0100243E80021D5
:10B750000029F7D1DA69B0F85C10D20644BF102294
:10B760001A62FFF725FE08BD9A6942F008029A6145
:10B77000F9E700BF00800040D0F88C20B0F86010DE
:10B78000222A08B5036852D15A6A1140826D22F804
:10B79000021B8265B0F85E20013A92B2A0F85E20EA
:10B7A000B0F85E2092B2002A40D153E8002F22F474
:10B7B000907243E800210029F7D103F1080252E812
:10B7C000002F22F0010203F1080C4CE800210029AF
:10B7D000F3D12022C0F88C20174A416793420167B9
:10B7E00005D1C26E012A0ED0F8F78EFD1EE05A6810
:10B7F0001102F6D553E8002F22F0806243E80021C1
:10B800000029F7D1EDE70022C26653E8002F22F0AD
:10B81000100243E800210029F7D1DA69B0F85C1082
:10B82000D20644BF10221A62FFF7C2FD08BD9A6912
:10B8300042F008029A61F9E7008000402DE9F84FD4
:10B840000368B0F86060D3F81CB01F689D68D0F83A
:10B850008C20222A044640F0B980B0F8683043B109
:10B86000DFF87491DFF874A14FF000081BF0200F8F
:10B8700020D1B4F85E309BB2D3B1B4F868209A42BC
:10B8800016D9226802F1080353E8003F23F08053E1
:10B89000083242E8003122680029F2D1504B636738
:10B8A00052E8003F43F0200342E800310029F7D17D
:10B8B000BDE8F88F2368A26D5B6A33401370A36DF7
:10B8C0000133A365B4F85E30013B9BB2A4F85E304F
:10B8D0002368D3F81CB01BF0070F2ED01BF0010F0C
:10B8E00009D0F90507D501221A62D4F8902042F058
:10B8F0000102C4F890201BF0020F09D0EA0707D517
:10B9000002221A62D4F8902042F00402C4F8902077
:10B910001BF0040F09D0E80707D504221A62D4F8F7
:10B92000903043F00203C4F89030D4F8903023B143
:10B930002046FFF70EFDC4F89080B4F85E309BB24D
:10B94000002B93D1226852E8003F23F4807342E831
:10B95000003123680029F5D103F1080252E8002FD5
:10B9600002EA090203F1080040E800210029F3D1AE
:10B9700020225345C4F88C20616721670AD05A6899
:10B98000110207D553E8002F22F0806243E800211E
:10B990000029F7D1E26E012A14D10022E26653E8B1
:10B9A000002F22F0100243E800210029F7D1DA69C4
:10B9B000B4F85C10D20644BF10221A622046FFF78A
:10B9C000F7FC53E72046F8F79FFC4FE79A6942F0EF
:10B9D00008029A616CE700BFFEFFFFEF00800040A5
:10B9E000ADB600082DE9F84F0368B0F86060D3F8F1
:10B9F0001CB01F689D68D0F88C20222A044640F0B5
:10BA0000B780B0F8683043B1DFF87091DFF870A10B
:10BA10004FF000081BF0200F20D1B4F85E309BB22D
:10BA2000D3B1B4F868209A4216D9226802F108030B
:10BA300053E8003F23F08053083242E80031226887
:10BA40000029F2D14F4B636752E8003F43F02003D7
:10BA500042E800310029F7D1BDE8F88F2368A26DD4
:10BA6000596A314022F8021BA265B4F85E20013AFF
:10BA700092B2A4F85E20D3F81CB01BF0070F2ED0B2
:10BA80001BF0010F09D0F90507D501221A62D4F87D
:10BA9000902042F00102C4F890201BF0020F09D060
:10BAA000EA0707D502221A62D4F8902042F0040275
:10BAB000C4F890201BF0040F09D0E80707D5042232
:10BAC0001A62D4F8903043F00203C4F89030D4F8EE
:10BAD000903023B12046FFF73CFCC4F89080B4F8C6
:10BAE0005E309BB2002B95D1226852E8003F23F4D0
:10BAF000807342E8003123680029F5D103F1080280
:10BB000052E8002F02EA090203F1080040E8002190
:10BB10000029F3D120225345C4F88C2061672167A6
:10BB20000AD05A68110207D553E8002F22F080622C
:10BB300043E800210029F7D1E26E012A14D1002246
:10BB4000E26653E8002F22F0100243E800210029AA
:10BB5000F7D1DA69B4F85C10D20644BF10221A6239
:10BB60002046FFF725FC55E72046F8F7CDFB51E7C7
:10BB70009A6942F008029A616EE700BFFEFFFFEF8C
:10BB80000080004079B7000838B504460368216991
:10BB9000A2681D68C0690A4361690A437749024384
:10BBA00029400A431A605A68E16822F440520A4365
:10BBB0005A60734AA16993421CBF226A11439A6872
:10BBC00022F06E4222F430620A439A60DA6A616AB5
:10BBD00022F00F020A43DA626A4A934219D14FF007
:10BBE000B043694AD3F8883003F0030343F4403389
:10BBF000934200F0B480B3F1031F24D0013A934282
:10BC000040F0B580B0F5004F40F08F80FCF780FF2A
:10BC10006EE05E4A93421CD14FF0B0435C49D3F8CA
:10BC2000883003F00C0343F440228A4200F09780EE
:10BC300006D8002B7CD0574B9A42E3D0012026E057
:10BC4000B2F10C1FFAD1B0F5004F53D04FF40040C1
:10BC500075E04B4A9342F1D14FF0B043D3F88830AE
:10BC600003F44063B3F5006F18D006D85BB1B3F5A9
:10BC7000806FE3D1FCF74CFF07E0B3F5406FDDD1F7
:10BC80004FF400400BE0FDF73BFB40B900204FF0C4
:10BC90000113A3660023C4E91D3338BD3E4865681F
:10BCA0003E4B626A05EB450133F81220B0FBF2F31C
:10BCB0009942C3D8B3EB053FC0D800231946F6F725
:10BCC000F3FB090241EA10616B080002C0182A4622
:10BCD0004FF0000341F10001F6F7E6FB304BA0F511
:10BCE00040729A42AAD82368D860CFE7FDF708FBD4
:10BCF0000028CBD06168294B626A33F81220B0FB70
:10BD0000F2F24B0803EB42034FF6EF72B3FBF1F391
:10BD1000A3F11001914291D823F00F02216892B251
:10BD2000C3F342031343CB60B0E7FCF7F1FE04E03A
:10BD3000B0F5004FDAD0FDF7E3FA0028A6D063682B
:10BD4000616A164A32F81120B0FBF2F000EB5300A2
:10BD5000B0FBF3F04FF6EF73A0F11002C1E7B0F5BE
:10BD6000004F0D48EBD1C5E7FDF7DAFAC0E7B0F5B3
:10BD7000004FF9D0FDF7D4FADFE700BFF369FFCF3A
:10BD800000800040003801400200030000440040F1
:10BD900008000C0004000C000024F40020810308BB
:10BDA000FFFC0F00836ADA0710B506D50168C46A84
:10BDB0004A6822F4003222434A609C0706D5016893
:10BDC000046B4A6822F4803222434A60590706D540
:10BDD0000168446B4A6822F4802222434A601A07B1
:10BDE00006D50168846B4A6822F4004222434A6007
:10BDF000DC0606D50168C46B8A6822F480522243AF
:10BE00008A60990606D50168046C8A6822F400529B
:10BE100022438A605A060FD50168446C4A6822F4AE
:10BE200080122243B4F5801F4A6005D14A68846CB1
:10BE300022F4C00222434A601B0606D50268C16C88
:10BE4000536823F400230B43536010BD2DE9F843DE
:10BE5000DDF8209005460F46164698462A68D369B5
:10BE600037EA03030CBF01230023B34201D00020B3
:10BE700029E0B9F1FF3FF2D0F7F76EFEA0EB080022
:10BE800048452C6802D8B9F1000F1ED154E8003F94
:10BE900023F4D07344E80032002AF7D104F10803F8
:10BEA00053E8003F23F0010304F1080141E80032A8
:10BEB000002AF3D12023C5F88830C5F88C30002340
:10BEC00085F884300320BDE8F88323685A07C5D578
:10BED000E3691B05C2D54FF40063236254E8003FB9
:10BEE00023F4D07344E80032002AF7D104F10803A8
:10BEF00053E8003F23F0010304F1080141E8003258
:10BF0000002AF3D12023C5F88830C5F88C30C5F855
:10BF10009030D4E773B504460026C0F89060F7F778
:10BF20001BFE23681B681A07054619D423681B6883
:10BF30005B070AD56FF07E43009300222B464FF437
:10BF400080012046FFF782FFB0B900202023C4F80B
:10BF5000883084F88400C4F88C30E06620670CE0F8
:10BF60006FF07E430093324603464FF400112046A3
:10BF7000FFF76CFF0028D9D0032002B070BD10B5C8
:10BF8000044650B3D0F888301BB980F88430F8F7F5
:10BF9000BBF822682423C4F88830136823F0010317
:10BFA00013602046FFF7F0FD012816D0A36A13B1F5
:10BFB0002046FFF7F7FE23685A6822F490425A6041
:10BFC0009A6822F02A029A601A6842F0010220461A
:10BFD0001A60BDE81040FFF79DBF012010BD0000B2
:10BFE00030B581658168A0F85C200023B1F5805FE1
:10BFF000A0F85E20436735D10369002B40F2FF13A0
:10C0000018BFFF23A0F860300023C0F8903022232F
:10C01000C0F88C30016801F1080353E8003F43F099
:10C020000103083141E800340368002CF2D1456E69
:10C0300084680169B5F1005F32D1B0F8685095426B
:10C040002ED8B4F5805F244A03D1244C002908BFC0
:10C0500022464267B1B153E8002F42F4807243E8B0
:10C060000021F7E729B90369002B14BF7F23FF23C1
:10C07000C8E7B1F1805FC5D10369002B14BF3F232E
:10C080007F23BFE703F1080252E8002F42F08052FD
:10C0900003F1080040E800210029F3D1002030BD61
:10C0A000B4F5805F0E4A03D10E4C002908BF22462A
:10C0B000426741B153E8002F42F4907243E80021F7
:10C0C0000029F7D1EAE753E8002F42F0200243E8C5
:10C0D00000210029F7D1E1E73DB80008E5B90008E3
:10C0E000ADB6000879B70008D0F88C30202B30B4FA
:10C0F00015D1B9B1B2B100230468C3660A4B9C42A2
:10C100000AD063681B0207D554E8003F43F0806300
:10C1100044E80035002DF7D130BCFFF761BF0220A5
:10C1200030BC70470120FBE700800040436E30B513
:10C130002BB90123A0F86A30A0F8683030BD03683D
:10C14000094D9A689968094C490FC2F342626B5CC9
:10C15000615CDB00B3FBF1F3A0F86A30AB5CA25C7E
:10C16000DB00B3FBF2F3E7E7408103083881030803
:10C170007047704770471FB504AB03E9060090F89D
:10C180008430012B04463AD0012380F884302423E4
:10C19000C0F8883003681A6822F001021A609A68B1
:10C1A00022F440120A439A6071B95A68BDF80C0033
:10C1B0009DF80E1022F0100202435A605A6822F0D5
:10C1C0007F4242EA01625A601A6842F001021A6034
:10C1D000F7F7C2FC6FF07E42034600924FF48001F5
:10C1E00000222046FFF732FE38B92023C4F88830F9
:10C1F000002384F8843004B010BD0320F8E7022047
:10C20000F9E790F88430012B0FD0012380F88430B7
:10C21000016851E8002F42F0020241E80023002BA0
:10C22000F6D180F88430184670470220704710B568
:10C2300090F88430012B044617D02423C0F88830AE
:10C2400003681A68196821F00101196042F0005270
:10C250004FF0005141661A60FFF768FF2023C0F8D5
:10C260008830002084F8840010BD0220FCE770B5FF
:10C2700090F88430012B044617D005682423C0F8B9
:10C2800088302E682B6823F001032B60AB6823F005
:10C2900060431943A960FFF749FF20232E60C0F8CF
:10C2A0008830002084F8840070BD0220FCE770B55F
:10C2B00090F88430012B044617D005682423C0F879
:10C2C00088302E682B6823F001032B60AB6823F0C5
:10C2D00060631943A960FFF729FF20232E60C0F88F
:10C2E0008830002084F8840070BD0220FCE7000044
:10C2F00038B5084D052455F8043B2BB9013C14F022
:10C30000FF04F8D1204638BDDB6898470028F5D0F7
:10C31000F9E700BF54230020034BD870034B1B6880
:10C320001B6C03B1184770473C23002038230020C2
:10C33000034B1874034B1B685B6C03B118477047C1
:10C340003C23002038230020F0B5314D314B95F9C6
:10C350000420314E91B00C46012795F905108DF857
:10C36000047002288DF809208DF80A1010D18DF87C
:10C370000800D8711C7203F075FB337803B114B157
:10C3800001A804F0A5F8254B059A1A6011B0F0BD7C
:10C3900059714FF480711A71D9801C7233788DF8FD
:10C3A000087053BB1F2306A88DF81C208DF8183089
:10C3B00003F036FD20238DF8183006A82B798DF870
:10C3C0001C3003F02DFD22238DF8183006A86B7960
:10C3D0008DF81C3003F024FD21238DF8183006A8B9
:10C3E0006B798DF81C3003F01BFD29238DF8183074
:10C3F00006A80B4B079303F013FD03F033FB012357
:10C4000006A88DF818308DF81C3003F009FDB4E74C
:10C410003C230020E0030020182200200C230020F1
:10C42000000400017FB5092301A88DF8043004F051
:10C430004FF80038044B059A1A6018BF012040429B
:10C4400007B05DF804FB00BF0C23002070B5044664
:10C450000B46144962784A700020A2780A7208706C
:10C460001A884A729A788A72DB780B746368CB6098
:10C470000D4B1B68DA6A2AB1237803F0FB030A2B01
:10C4800000D09047094E002556F8043B1BB15B6A6B
:10C490000BB1204698470135EBB2052B6DB2F3D1B5
:10C4A00070BD00BFB00300203823002054230020BB
:10C4B00070B5044611480123037063784370A37874
:10C4C0008372E368C360E378037623694376237954
:10C4D00043720B4B1B689B6A03B19847094E0025BA
:10C4E00056F8043B1BB19B690BB1204698470135B8
:10C4F000EBB2052B6DB2F3D170BD00BFC4030020B9
:10C500003823002054230020014B1868704700BFD7
:10C510000C23002000B58BB0012368468DF8003055
:10C5200003F058FB38B99DF80400003818BF01200B
:10C530000BB05DF804FB0020FAE7000008B502F03C
:10C5400049FC40B9FFF7E6FF012806D0054B197AF0
:10C55000D879FFF7F9FE012008BDBDE80840FFF7D4
:10C56000C7BE00BFE00300202DE9F04186B00546BC
:10C570000E46174602F02EFC002873D102F042FC52
:10C58000044640B9FFF7C6FF01280AD03D4B197A8F
:10C59000D879FFF7D9FE6FF00204204606B0BDE857
:10C5A000F081DFF8E48088F80860003E18BF0126BB
:10C5B0008DF80460354E687833798DF8123069460D
:10C5C00003F0A6FA00283FD08DF804400394ADF89C
:10C5D00010406FF0060495E803002D4B83E803003C
:10C5E000337988F80A30394601A804F075F8294BE8
:10C5F000059A1A6011283FD801A353F820F000BF14
:10C600006BC6000865C6000879C6000879C6000830
:10C6100079C6000879C6000879C6000897C50008E1
:10C6200079C6000879C6000879C600085FC6000808
:10C6300079C6000879C6000865C6000865C6000806
:10C6400065C600087FC600082B788DF808306B7827
:10C65000ADF810306B6803934FF0FF34BBE76FF019
:10C6600005049AE76FF0010497E70B4B00221A705C
:10C67000E31D18BF144690E74FF0FF348DE76FF0CD
:10C6800004048AE7E0030020C40300203C230020C8
:10C69000D40300200C2300200B23002037B502F028
:10C6A000BBFB134D052455F8043B4BB11A693AB155
:10C6B0009B682BB1984718B155F8043C1B69984703
:10C6C000013C14F0FF04EED1FFF712FE68B9094DEA
:10C6D0002B7853B1084BADF80040D978019422462D
:10C6E0006846FFF741FF00B92C7003B030BD00BFB2
:10C6F000542300200B2300203C23002030B58BB0B6
:10C70000044602F067FB0546002835D1FFF702FF1B
:10C71000012834D168468DF8005003F05BFA40BB25
:10C720009DF80430A34204D0012C22D0022C12D058
:10C7300014B100200BB030BD002BFAD068468DF844
:10C74000044003F06DFBA0B90E4B1B681B6B002B64
:10C75000EFD09847EDE763B968468DF8044003F0E1
:10C760005FFB30B9074B1B681B6B002BE1D02046E9
:10C77000EFE74FF0FF30DDE76FF00100DAE76FF031
:10C780000200D7E73823002010B504468AB018B954
:10C790004FF0FF300AB010BD002368468DF800301E
:10C7A00003F018FA0028F3D19DF804302370F1E764
:10C7B0007FB500220B4620498DF8072001220A7020
:10C7C00042784A700446002A33D102790A721A88E4
:10C7D0004A729A788A72DB780B740369CB60C378EB
:10C7E000164D8DF80830037B8DF80930836803936C
:10C7F0002B68DB6A0BB102A898472B689B6B13B1BF
:10C80000227E02B198470E4E052556F8043B1BB117
:10C81000DB690BB120469847013D15F0FF05F4D1C7
:10C820000DF10700FFF7B0FF637913B1054B01224B
:10C830001A7004B070BD00BFB00300203823002080
:10C84000542300200B23002010B504468AB018B9E9
:10C850004FF0FF300AB010BD202368468DF800303D
:10C8600003F0B8F90028F3D1024A9DF9043023708F
:10C870001371EFE73C23002000B58BB02323019018
:10C8800068468DF8003003F0CBFA003818BF01205D
:10C8900040420BB05DF804FB70B5654C01468EB0AC
:10C8A0001822204606F0BCFF624B00221A70FAF7ED
:10C8B0007FFE23784068012202FA03F1014004D18F
:10C8C0005D4B084608F098FFFEE75C495C481A4655
:10C8D00002F00AFF18B14FF0FF300EB070BD2723F1
:10C8E00004A88DF8103003F09BFA564E564D0028E0
:10C8F00070D1012333702B68DB690BB1002098479E
:10C90000272304A88DF8103003F064F9059B93F8F1
:10C910004820227093F8182193F81A316270A3709E
:10C92000464BD3E9020106F06BFE05460028D2D142
:10C93000464E062304A88DF8103003F04BF9059BF2
:10C94000736104A803F06CFA022304A88DF8103078
:10C95000059603F03FF90836032304A88DF810303C
:10C96000059603F037F90F2606F010FF012304A8FF
:10C970008DF814308DF8106003F052FA10230DEB8F
:10C9800003008DF810308DF8145003F049FA042399
:10C990008DF8103004A8A3788DF8143003F040FA15
:10C9A0003A238DF8103004A86369059303F038FA30
:10C9B00002A920788DF8086004F0CCFF003818BF79
:10C9C0000120E0711420FFF757FFE07904F046F8EA
:10C9D000284682E728238DF810302B681B6943B165
:10C9E00004A803F0F7F82B6805981B6940F2C451BE
:10C9F0009847272304A88DF8103003F011FA50B996
:10CA0000012304A88DF8103003F0E4F89DF81430E9
:10CA1000002B7FF46EAF3378002B7FF46CAF0522D0
:10CA200004A88DF81020059303F0FAF978E700BF09
:10CA30003C2300200B230020488103081023002002
:10CA400028230020182200203823002078230020EB
:10CA500037B500230D4601930446D0B900F07CFDA4
:10CA60000190019BD3B10F4A42F824300E4A9A62DA
:10CA70000E4A1268916B1963916C596392690C4963
:10CA8000D9625A6128465B680A49F2229847002019
:10CA900006E001A900F076FD0028E2D04FF0FF305B
:10CAA00003B030BD5423002049C3000838230020C0
:10CAB00025C4000819220020194B07B51860194B2E
:10CAC000194A1A60194A5A60194A9A60194ADA6072
:10CAD000194B02681A6042685A6082689A60C2689C
:10CAE000DA60164A1A6182695A61154BC26B5A6044
:10CAF000144A019119609A601946134ADA600020BD
:10CB0000FFF7A6FF48B901A800F02AFD003818BFBA
:10CB10000120404203B05DF804FB4FF0FF30F9E71D
:10CB20003823002028230020B1C40008B1C7000822
:10CB3000F1CB00084DC4000810230020051901089E
:10CB40006823002019C3000831C3000849B118B197
:10CB5000012804D000207047034B0B60FAE7034B19
:10CB6000FBE74FF0FF3070470004000101000102B5
:10CB700008B503F08FFF002814BF6FF001000020FC
:10CB800008BD08B502F096FF002814BF6FF0010041
:10CB9000002008BD20B1044BDB79037000207047F2
:10CBA0004FF0FF30704700BF3C23002008B5034B17
:10CBB000D87103F053FF002008BD00BF3C230020C4
:10CBC00010B504468AB018B94FF0FF300AB010BD56
:10CBD000212368468DF8003002F0FCFF0028F3D1D5
:10CBE000024A9DF9043023705371EFE73C23002083
:10CBF0002DE9F0412F4D304F00232B7043786B709F
:10CC00003B689B6A8AB004460BB128469847DFF818
:10CC1000AC80002658F8043B1BB11B6A0BB12046C0
:10CC200098470136F3B2052B76B2F3D12378052B62
:10CC30002FD00B2B35D0012B25D1214C0623684654
:10CC40008DF8003002F0C6FF0199E07906F01EFD74
:10CC500010B91C4B019A5A611B48FFF7F5FD1B48A0
:10CC6000FFF7AEFF6B788BB9A371194B5878FFF7BC
:10CC700045FD3B685B6A0BB1114898476B7813B967
:10CC8000E07906F095FD0AB0BDE8F081FF23A371BD
:10CC9000EFE7104B01225A74227A9A74627ADA749E
:10CCA000F1E76378002BEED00AB0BDE8F041FFF762
:10CCB000B9BB00BFC4030020382300205423002048
:10CCC000E003002078230020E4030020E503002097
:10CCD0003C230020B003002030B58BB0FFF751FF9C
:10CCE0000446F0B904F016FE831C1DD0F8B9134DAC
:10CCF0002B685B69DBB1272368468DF8003002F0B2
:10CD000069FF2B6801985B694FF4B961984704F09B
:10CD100013FE78B92CB9094B1B68DB690BB10120F4
:10CD2000984720460BB030BD6FF00704EFE74FF097
:10CD3000FF34ECE74FF0FF34F3E700BF3823002067
:10CD4000014B1878704700BFA8230020014B58788A
:10CD5000704700BFA8230020064B074810B50122EA
:10CD60005A7309F085F9054B5B6913B1BDE81040B2
:10CD7000184710BDA823002090230020EC030020BA
:10CD800013B50A4C79B1A2700123002261602370AF
:10CD90000748084B00924FF0FF3109F0BDF800231F
:10CDA000637002B010BD2170F9E700BFA823002016
:10CDB0009023002059CD00082DE9FF47C378CA2BE6
:10CDC000804600F0BE8004B0BDE8F087D8F8083097
:10CDD0005A5D6E1CF6B2032A0FD8DFE802F0022E6D
:10CDE0006CAB7A6800231355611CA31CDBB2C9B27B
:10CDF000012050540334D054E4B2354698F80C3036
:10CE0000AB42E3D8002CDED0CA238DF80830504B5B
:10CE10008DF809405B6803930DF10700FFF7BAFE38
:10CE20000020FFF7C3FE0122002102A8FFF79CFBB0
:10CE30009DF80700FFF7BAFEC5E700227A7398F85D
:10CE400018204AB96A1DD2B2397A9A5C01F00F01F2
:10CE500002F00F02914202D0AE1DF6B2CDE7AA1C3D
:10CE6000D2B29E5D9A5C06EB0226EA1CD2B20DF1AC
:10CE7000080A9A5C06EB02462A1DD2B250469B5C19
:10CE800006EB036608F022FF029B334402939AE804
:10CE9000030008F0F3FE3B7AC3F30302013262F3AE
:10CEA00003033B722B4B1B6B002BD5D00136022E9C
:10CEB000D2D89847D0E7EE1C0235EDB21E215B5D5B
:10CEC000002003F00F0380259D4006F08DFC7A685A
:10CED0000223135504EB030A631CDBB20021D15477
:10CEE000054402A808F0F2FE029B7A684B4504F163
:10CEF000030188BFA3EB09035FFA8AFAC9B2180AD3
:10CF000002F80A305054611D201DC9B2C0B24FEA68
:10CF1000134C1B0E02F800C053544FF47A7169434E
:10CF20000D4809F0DFF806340B48F6B2E4B209F018
:10CF30009FF862E79B5D023503F007037B73EEB257
:10CF40005BE70024024FDFF81490254656E700BF48
:10CF5000A8230020EC03002090230020803DD51260
:10CF600010B5114C637A8AB0E3B104238DF8003018
:10CF70006846A37A8DF8043002F052FF18238DF82A
:10CF800000306846E37A8DF8043002F049FF202330
:10CF90008DF800306846237B8DF8043002F040FFA6
:10CFA000002363720AB010BDA82300200048704718
:10CFB000EC03002030B58FB0FFF7C0FA002861D134
:10CFC000324C657A4DBB042304A88DF8103002F072
:10CFD00001FE9DF81430A37204A88DF8145002F0DD
:10CFE0001FFF182304A88DF8103002F0F3FD9DF800
:10CFF0001430E37204A801238DF8143002F010FFFE
:10D00000202304A88DF8103002F0E4FD9DF81430C0
:10D0100023731F4BDB6A03B1984702A808F056FE42
:10D02000029A1C4B1C4913448B4288BF1B4B6168FE
:10D0300088BF9B181A0A4B708A701A0C1B0E0B7152
:10D04000237ACA7001256FF304134B710D7023729C
:10D050000DF1070040F2CA63ADF81030059165721A
:10D06000FFF798FD0020FFF7A1FD2A46002104A844
:10D07000FFF77AFA04469DF80700FFF797FD204670
:10D080000FB030BD4FF0FF34F9E700BFA8230020F8
:10D09000EC03002080C22AED803DD512008555DAD0
:10D0A00010B5054C637B2BB1FFF784FF10B9637B90
:10D0B000013B637310BD00BFA8230020014B18780B
:10D0C000704700BFD4230020014B5878704700BF41
:10D0D000D423002070470000044B9A7A0AB1012241
:10D0E0005A70034B5B6903B118477047D423002083
:10D0F0002404002073B5224C6378002B33D008F051
:10D1000025FF66680546FFF7FFF90644AE4214D2D4
:10D11000A37A93B1E0228DF800208DF80130217AB6
:10D12000E368019301226846FFF71EFA08B1073051
:10D1300010D100236370A372656094F83430EBB1B2
:10D14000002384F834300F4B5B6BBBB102B0BDE8F9
:10D150007040184740F2DC510B4808F0C3FF0A4802
:10D1600008F086FFE8E794F83520002AE5D094F827
:10D17000360084F83530FFF7C1FADEE702B070BD43
:10D18000D423002024040020B823002037B5104DFC
:10D19000104CC8B1C1B16272012300222860E16065
:10D1A00023700D480D4B00924FF0FF3108F0B4FE94
:10D1B00000250B4825822022294606F045FB657094
:10D1C000A574A58603B030BD00232B602370EFE764
:10D1D000D0230020D4230020B8230020D9D0000879
:10D1E000E82300202DE9F0478E4C23788CB0002BEB
:10D1F00056D0C2780AB9837B13B1238A01332382C4
:10D20000437B002B4CD0E02A4AD10023A3728768CD
:10D2100097F80080B8F1220F27D8B8F1220F30D844
:10D22000DFE818F04100FB0052005A0061006E0078
:10D2300075008E009D00B400C7002F002F002F0046
:10D240002F002F002F002F002F002F002F002F0066
:10D250002F002F002F002F002F002F002F002F0056
:10D260002F002F00C900D000D400B8F17E0F00F0CD
:10D27000CC80B8F17F0F00F0DF80B8F17D0F00F0B7
:10D28000AB80A57A002D00F05B81674C637A3BB9D7
:10D290004FF47A71204608F025FF204608F0E8FE9A
:10D2A0000CB0BDE8F087E36801220021A27219707A
:10D2B000A37AE1689818A0720620C854A37AE1689E
:10D2C0009818A072CA54DCE7584B9B6A002BD8D040
:10D2D000012102209847D4E77B7884F83630012377
:10D2E00084F83530CDE704238DF804307B78003B9B
:10D2F00018BF012301A88DF8083002F091FDC0E7A6
:10D300007878003818BF012003F0A8FBB9E7484E31
:10D310000FCE01AD0FC50FCE0FC596E8070085E80B
:10D3200007007B780A2BACD8424A12685268002A60
:10D33000A7D00CA901EB830353F82C0C9047A0E76E
:10D340007878431E012B9CD83A4B01381B6818BFD4
:10D35000012020729B68002B93D0984791E7E268E8
:10D3600001230821A3721170627A057BA17AAA4277
:10D3700028BF2A46934284D285685A1CEB5CE56834
:10D3800001334E1CA6726B54D3B2EDE7E368012261
:10D39000A27209221A70A37AE268218A581CA0722C
:10D3A000D154A27A238AE1681B0A501CA0728B54C4
:10D3B00067E7238265E705238DF8043001A803F0B1
:10D3C00087F85EE7194BDB6A98475AE7194B78787C
:10D3D0001B686075DB68BEE7037B072B7FF451AFEA
:10D3E00006238DF80430B7F80130ADF808307B79AA
:10D3F0003A791B0443EA0223FA7813436422534325
:10D400000393BB798DF81030D8E73B2201A88DF843
:10D4100004208DF8083002F003FD012384F8343035
:10D420002FE700BFD4230020B823002024040020CD
:10D43000342C0308D02300202A2301A88DF80430BF
:10D4400002F0C8FB94F80A90E6689DF808009DF881
:10D4500009509DF80A709DF80BC09DF80D309DF89D
:10D460000E209DF80F109DF80CE009F1010A84F8D8
:10D470000AA006F80980354E94F80A903668D4F868
:10D480000C8009F1010A84F80AA096F803A008F8B4
:10D4900009A094F80A90D4F80C8009F1010A84F8E4
:10D4A0000AA096F802A008F809A094F80A90D4F807
:10D4B0000C8009F1010A84F80AA096F801A008F886
:10D4C00009A094F80A9009F1010A84F80AA096F8D4
:10D4D0000080E66806F8098094F80A80E66808F19A
:10D4E000010984F80A9006F808C094F80AC0E668B2
:10D4F0000CF1010884F80A8006F80C70A77AE66837
:10D5000007F1010C84F80AC0F555A57AE6686F1C8E
:10D51000A7727055A07AE568461CA6722954A17AB4
:10D52000E0684D1CA5724254A27AE168501CA072BA
:10D530008B54A37AE268591CA17202F803E0A0E6BA
:10D54000034808F047FD6570AAE600BFD02300201D
:10D55000B8230020704700000048704724040020D2
:10D56000002108B50120FFF773FA014638B90220FF
:10D57000FFF76EFA003818BF0120404208BD4FF097
:10D58000FF30FBE710B50C4661B1012803D002283B
:10D5900005D0002010BDFFF709FD2060F9E700F07D
:10D5A0001FFCFAE74FF0FF30F4E70000014B18785A
:10D5B000704700BF94040020014B5878704700BFAB
:10D5C00094040020F7B500208DF80700EFF31082D7
:10D5D00072B62A4FBB78FD7882F31088012B08D0F1
:10D5E000022B04D1264B93F82030012B3CD103B001
:10D5F000F0BD234E0DF10700FFF7C6F8382303FBFB
:10D60000056393F82C00012806D19DF80730022B02
:10D6100008D10023BB70EAE7022803D19DF8073048
:10D62000012BF5E7FFF76AF805EB4504E400B0B914
:10D63000144BB8701C44382303FB05664FF47A7111
:10D6400096F82830994096F82C30012B00D1C9016A
:10D65000204608F047FD204608F00AFDC7E70A4BC0
:10D660001C444FF47A71F3E7FFF748F80028D0D054
:10D67000044C05EB450504EBC504F2E794040020D7
:10D680003C2400200C2400202424002037B50F4C1B
:10D69000D1B100250123A160227123702A460C4BD1
:10D6A0000C4800954FF0FF3108F036FC0A4B0B4850
:10D6B00000952A464FF0FF3108F02EFC084A00235F
:10D6C0006370137003B030BD2170F7E7940400203D
:10D6D00019D7000824240020E5D600080C240020D7
:10D6E0003C24002010B5084808F074FC074B0022C9
:10D6F00083F82020064B02225A80064B5B6913B147
:10D70000BDE81040184710BD0C2400203C24002028
:10D71000940400205C04002010B5084808F05AFC6E
:10D72000074A012382F82030064A5380064B5B6982
:10D7300013B1BDE81040184710BD00BF24240020DD
:10D740003C240020940400205C0400202DE9F04FCC
:10D75000C378C82B8FB0824600F029830FB0BDE894
:10D76000F08FDAF80820D05C591CC9B2052816D809
:10D77000DFE810F00600AA00F000AE01E1018B0224
:10D78000BA680023601C1355C0B2A31CDBB24FF073
:10D79000020C02F800C001200334D054E4B20B465E
:10D7A0009AF80C209A42DCD8002CD7D0C8238DF8E8
:10D7B0001430B74B8DF815409B6806930DF113009C
:10D7C000FFF7E8F90020FFF7F1F90122002105A891
:10D7D000FEF7CAFE9DF81300FFF7E8F9002DBDD152
:10D7E000AC4CAD4F637803F003032A4629460093FF
:10D7F0000220AA4B08F000F82646636800932A46E8
:10D800002946A74B022007F0F7FF16F8083F0093C0
:10D810002A462946A34B022007F0EEFF012516F801
:10D82000013F009300223B4611460220013507F0DC
:10D83000E3FF102DF3D1002211469B4B022007F08D
:10D84000DBFFA369009300221146984B022007F0EA
:10D85000D3FFE369009300221146954B022007F0A5
:10D86000CBFF636A009300221146924B022007F01F
:10D87000C3FF94F82820012393400022114600930F
:10D8800002208D4B07F0B8FF94F82C300022012BBA
:10D89000236B00931146894B4FF0020040F08D82BC
:10D8A00007F0AAFF94F9343000930022844B11460C
:10D8B000022007F0A1FFE38E0093824B0022114665
:10D8C000022007F099FF49E7BD6812F801C0012264
:10D8D0002A55023300220234DBB2E4B211469646E6
:10D8E0000CF0010C96F80080BEF1000F07D0120179
:10D8F00002F0700211436970054619464FE7B8F10E
:10D90000000FF4D0BCF1000F21D005F804E004F1C1
:10D91000010E5FFA8EFE716805F80E1004F1020E1A
:10D9200071685FFA8EFE090A05F80E1004F1030E05
:10D930005FFA8EFEB6F8068005F80E80211DC9B28A
:10D9400096F807E005F801E00534E4B261460132DB
:10D950008646C7E7555C382105F0030501FB0561E4
:10D9600003F1020B5FFA8BFB4D70002D40F08E80AF
:10D97000D81C12F80B107160C0B203F1050C105CDA
:10D9800001EB0021181DC0B27160105C5FFA8CFCC5
:10D9900001EB0041716012F80CC0981D01EB0C699D
:10D9A00003F11601DFF820C1C6F80490C0B2C9B275
:10D9B00086460130C0B212F80EE00CF801EF884242
:10D9C000F6D1115CB16103F11700C0B203F11E0B77
:10D9D000105C01EB002103F11800C0B2B161105CD2
:10D9E00001EB004103F11900C0B2B161105C01EB21
:10D9F000006803F11A01C9B2C6F8188003F11B00D0
:10DA0000515CF161C0B25FFA8BFB105C01EB00214D
:10DA100003F11C00C0B2F161105C1D3301EB004149
:10DA2000DBB2F161D35C0DF1170001EB036321223E
:10DA30000021F361039321F001FE40F20112ADF8E1
:10DA400014207278039B0A93C2F301028DF816200A
:10DA500005A81E4ACDF818900792CDF8248002F050
:10DA600065FC012390B93370B96802230B55621C21
:10DA70001C44382303FB0563D2B25B78C3F3010374
:10DA800043EA80008854E4B2594688E60120EBE777
:10DA9000940400203C240020E7810308AC810308A3
:10DAA000BF810308D4810308A57E0308ED81030824
:10DAB0000082030813820308268203083B820308BE
:10DAC0004E8203086482030843240020442400207B
:10DAD000555C382005F00305023300FB05FB5FFAB7
:10DAE00083F906EB0B034FF000081846102241465D
:10DAF000083083F80180C3F80480039305F0A4FE86
:10DB0000039BC3E90688BB68032204F101081A5588
:10DB100028465FFA88F802F051FC40B145F0040352
:10DB2000BA68023402F80830E4B2494637E606F82B
:10DB30000B002B46F4E74FF0000B8DF813B0555C4B
:10DB400003F1020815F003055FFA88F840F09680AB
:10DB5000DFF874B24FF002098BF82C90D81C12F841
:10DB60000810CBF82410C0B203F10B08105C01EBD5
:10DB70000021181DC0B2CBF82410105C01EB00414D
:10DB8000581DC0B2CBF82410105C01EB00618F4827
:10DB90000844991DC9B2CBF82400515C01F00F0173
:10DBA0008BF82810D91DC9B203F10800515CCBF8DD
:10DBB0003010C0B25FFA88F8105C41EA002103F12E
:10DBC0000900C0B2CBF83010105C0A3341EA0041C2
:10DBD00064204143DBB2CBF83010D35C8BF8343097
:10DBE0000DF113020BF12C01284602F013FC002862
:10DBF00049D105A808F06AF8DBF82420059BA2EBC0
:10DC0000030BBBF1000F31DD4FF47A7101FB0BF117
:10DC10006F48039108F066FA6D4808F029FA0399F5
:10DC200000916C4B29462A46484607F0E5FD012144
:10DC3000BA6804231355601CC0B29DF813C002F8E3
:10DC400000C0A31CDBB271B102F803B0E31CDBB26D
:10DC50004FEA2B21D154631D0434E4B24FEA2B4B1D
:10DC600002F804B0DBB21C46414698E59DF813303B
:10DC700043F010038DF813302946D9E710238DF8AF
:10DC800013305946D4E7AB46F6E74FF0000B8DF85A
:10DC900013B0555C03F1020815F003055FFA88F82C
:10DCA0007ED1DFF824B14FF001098BF82C90D81CFD
:10DCB00012F80810CBF82410C0B203F10B08105C66
:10DCC00001EB0021181DC0B2CBF82410105C01EB51
:10DCD0000041581DC0B2CBF82410105C01EB00616C
:10DCE0003A480844991DC9B2CBF82400505CC0F3EF
:10DCF0000210ABF83600515C01F00F018BF82810D0
:10DD0000D91DC9B203F10800515CCBF83010C0B284
:10DD10005FFA88F8105C41EA002103F10900C0B203
:10DD2000CBF83010105C0A3341EA004164204143D3
:10DD3000DBB2CBF83010D35C8BF834300DF113022A
:10DD40000BF12C01284602F065FB70BB05A807F01B
:10DD5000BDFFDBF82420059BA2EB030BBBF1000FFA
:10DD600016DD4FF47A7101FB0BF11948039108F0AD
:10DD7000B9F9174808F07CF903990091154B294629
:10DD80002A46022007F038FD4946BA68052351E7C4
:10DD90009DF8133043F010038DF813302946F4E753
:10DDA00010238DF813305946EFE7AB46F6E7002411
:10DDB000094F054EFF252346F2E407F01DFD94F9B7
:10DDC00034300093054B79E53C240020803DD5128A
:10DDD0002424002091810308940400204E8203082B
:10DDE000004870475C040020044B054A93F8183142
:10DDF000022B18BF062382F890347047E02A0020D7
:10DE0000A4300020034BD3F8483313B15B6903B14E
:10DE100018477047A4300020034A137843F00403E6
:10DE20001370FFF7EFBF00BF882400201FB50A4B17
:10DE30008DF8090093F87C208DF80A2093F88C2047
:10DE400093F848000D3202A98DF8082003F082FDF6
:10DE5000C0B205B05DF804FBE02A002008B5074811
:10DE600008F0B8F8064B93F81A2412B1012283F88F
:10DE70001924BDE80840FFF7C5BF00BFA434002047
:10DE8000A430002010B50C4CD4F8403343F080038C
:10DE9000C4F8403394F81A3413B10020FFF7DEFFC2
:10DEA00094F8913423F0120343F0120384F8913470
:10DEB000BDE81040FFF798BFA43000202DE9F041E5
:10DEC000DFF8AC8098F81831022B06460D4602D0D8
:10DED000284BDB6A984702F078FE044628B10220FE
:10DEE00002F069FE002002F06BFE98F81831012B59
:10DEF00017D102F06CFE074630B1002002F05CFE44
:10DF0000002002F05EFE3C4602F063FE48B10020B5
:10DF100002F053FE002002F055FEBDE8F041FFF78D
:10DF200063BF002CF9D1144C94F8902494F81A345F
:10DF3000BAB90BB184F84164304602F0EBFFD8F86F
:10DF40002C0008F00DF8D4F8B4339842E5D30B4810
:10DF500008F040F894F8913443F0100384F89134B9
:10DF6000DBE70BB184F84154284602F0D3FFF1E718
:10DF7000E02A0020A4890308A43000203C340020BB
:10DF8000074A10B5137843F002031370FFF73AFF06
:10DF9000BDE81040034B01220021022007F02CBCF9
:10DFA0008824002077820308074A10B5137843F0CD
:10DFB00008031370FFF726FFBDE81040034B012252
:10DFC0000021022007F018BC882400208782030863
:10DFD0002DE9F0410F4616461D46804607F0B6FF74
:10DFE0000B4A0C4C1378278123F0110343F01103E3
:10DFF000C4E90008137066812573FFF703FFBDE8CD
:10E00000F041054B01220021022007F0F5BB00BFC3
:10E0100088240020742400209782030813B507F099
:10E0200095FF0D4B6C461860204607F04FFE94E8B4
:10E0300003000A4A0A4B83E80300137843F02003E5
:10E040001370FFF7DFFE074B01220021022002B010
:10E05000BDE8104007F0D0BB8424002088240020B5
:10E06000DC330020A48203082DE9F04192B006467B
:10E0700002F0ABFD002840F05881AD4D95F8183105
:10E08000012B09D02B6BAB4C93B194F80431BBB18D
:10E09000042B6FD0032003E002F099FD18B10F208C
:10E0A00012B0BDE8F08102F094FD0028EAD0F6E756
:10E0B000B5F82031D4F81C24013B53432B63E4E72B
:10E0C0009D4803F07EFB002840F0128194F80C314B
:10E0D00023802B6B0C930DF1180895F839308DF8CF
:10E0E0003830404695F81C318DF83A3007F014FE70
:10E0F000D5F82831009302AF98E80600D5F824310E
:10E10000384607F09FFD97E803000FAB83E8030054
:10E11000EB6A0D9300238DF844302388ADF8463028
:10E1200095F8303101228DF839201BB98DF8442043
:10E130008DF83930814B0093814B95F84800A3F15D
:10E1400079020CA903F07BFCC0B10B28A8D1D4F84C
:10E15000941499B1002EA3D0D4F84033794843F0F9
:10E160002003C4F8403307F0BDFF764807F080FF76
:10E17000002095E7704803F058FBA4E795F8487035
:10E1800095F9693095F9392095F87D106E4E38462D
:10E1900003F062FC009641B2EB6C95F850203846D3
:10E1A000183603F0FDFB0096EB6C95F8502095F9BE
:10E1B000701095F8480003F0F3FBD4F8C413AB6D6E
:10E1C000D4F8DC230B44C4F8B033EB6D1344C4F82B
:10E1D000B43394F80431042B07D02B6E0B44C4F8ED
:10E1E000B0336B6E1344C4F8B4330023089395F82E
:10E1F0003031002B40D100238DF8133095F83930A1
:10E200008DF8213095F838308DF82230D5F88030EF
:10E210000993D5F884300A932388ADF82C3095F80B
:10E22000303194F81B648DF82E3095F84800474B38
:10E230008DF820600DF1130208A903F0C5FB01233E
:10E2400084F8413495F8393084F842349DF813301D
:10E2500084F84334D4F81C34C4F85064C4F8483407
:10E26000C4F8583402F0B7FCC8B1D4F81C0402F06A
:10E27000C4FCA0B1102013E708A802F07BFD60B930
:10E2800095F9390094F837629DF82070FFF7CEFDBC
:10E290003E44B042AFD2082002E7132000E795F8D1
:10E2A0001831012B01D102F0AAFC02F097FC0023E7
:10E2B000059394F8043195F9395094F81B649BB197
:10E2C000042B7FF4E7AE05A802F088FF58BB94F852
:10E2D000183413B1059B013B0593174B0598324643
:10E2E000E9B202F0E1FF02E0134802F0B1FF08B129
:10E2F0001120D5E6D4F8403394F80C11218043F076
:10E300000203C4F8403394F8183411480133DBB2E7
:10E3100084F8183484F845340E4B00259B6AC4F801
:10E320009854984724E71220BAE60E20B8E600BFBA
:10E33000E02A0020A4300020AC310020102B002067
:10E34000383500200C3400205C340020C03400201C
:10E35000A6300020A489030873B5134D134E009610
:10E36000EB6C95F8502095F9781095F8480003F07B
:10E3700017FB95F83031337595F8480040F20123CA
:10E3800006F13C023146738203F016FB50B196F859
:10E390003C3086F88230064B00205B6B9847F37C5C
:10E3A00086F8A83002B070BDE02A00208C3400202E
:10E3B000A4890308F8B5324C94F81831012B0546AE
:10E3C0000ED0022B4ED0002B57D138B9D4E91B0107
:10E3D00004F1740383E803000020F8BD012806D18E
:10E3E00002F0FEFB0028F8D184F81851F5E7022866
:10E3F00043D1244E84F8180106F5747CBCE80F0064
:10E4000006F57A770FC79CE8030094F8E92094F8A2
:10E41000003187E8030086F8FB53D2B1022B18D1F4
:10E42000D4F804316367C6F8EC3394F87D3094F87F
:10E43000082186F8F83394F88C3084F8782086F830
:10E44000F93396F81B2486F8E82340F20133A6F846
:10E45000FA33002386F81A340B4BDB6A9847FFF730
:10E460007BFFB9E748B9074B84F81801062283F807
:10E470009024054BDB6A9847AEE70320ADE700BF69
:10E48000E02A0020A4300020A4890308F0B5504CF5
:10E49000504EB4F8DC202287D4E92D0194F8B12045
:10E4A00084F8692004F16C0282E80300D4E92F01AA
:10E4B00004F1740282E80300B4F8C420A4F87C20BC
:10E4C00091B0D4F8CC20D4F8C810C4F8842000252A
:10E4D000D4F8D020C4F888200123A4F82031C4F84F
:10E4E000801084F83051A56284F81B5184F83A50AA
:10E4F00084F81D5184F81E51C4F83451C6F898545C
:10E50000A6F8185486F81A54A4F838518DF8183023
:10E5100004F50973039304F50A7394F8480004930F
:10E5200003A92D4B84F84551C4E94F55A4F8465131
:10E53000059303F01DFAE36EC6F8D43394F87D30EA
:10E5400086F8E03394F88C3086F8E1334FF480732A
:10E55000A6F8E23386F8D05394F8303186F8E433E5
:10E5600006F574770FCF06F57A740FC497E80300A9
:10E5700040F2012384E80300A6F8FA33D6F84833C2
:10E5800086F81B54CDE901551BB15A685B690192AD
:10E590000293124B0793A3F148020892A3F11402CD
:10E5A00009920F4A0B9229330A93A2F19C030C9310
:10E5B000A2F198030D93131D0E9301A902F14C03D0
:10E5C00007A802F599620F9302F0F4FA11B0F0BDBA
:10E5D000E02A0020A43000208C2400200C350020EC
:10E5E000C42B0020F8B50D4F0D4E0C4607F0F2FC81
:10E5F0003B6B98470B4A96F84800214603F0DCF93C
:10E6000050B1094D706D95F8243485F86A347B6BF0
:10E610009847E37C85F89034F8BD00BFA4890308CF
:10E62000E02A0020C8340020A43000200F4890F8D1
:10E630001B3480F8B8330E4B93F8692080F8BB2365
:10E6400093F87D2080F8C82393F88C2080F8C923A4
:10E6500093F8303180F8CC330022A0F8CA2300F5BB
:10E660006E7100F56070FFF7BDBF00BFA4300020E1
:10E67000E02A0020114890F89034EBB190F81B3458
:10E6800080F8D0330E4BDA6EC0F8D42393F87D2097
:10E6900080F8E02393F88C2080F8E12393F8303160
:10E6A00080F8E4334FF48072A0F8E22300F574712F
:10E6B00000F56670FFF796BF704700BFA4300020DA
:10E6C000E02A002070B5344C2421204605F0BEF825
:10E6D000636A984218BF60624FF01C012F4814BF54
:10E6E0000125002505F0B2F8636C984218BF6064FC
:10E6F0004FF480712A4818BF45F0020505F0A6F8CE
:10E70000D4F84831984218BFC4F848014FF0D401FA
:10E71000244818BF45F0040505F098F8D4F82032D5
:10E72000984218BFC4F820024FF000011E4818BFDD
:10E7300045F0080505F08AF8D4F82432984218BF4D
:10E74000C4F824024FF46071184818BF45F0100552
:10E7500005F07CF8D4F8A835984218BFC4F8A8058D
:10E760004FF01401124818BF45F0200505F06EF86F
:10E77000D4F8C03598420F4B18BFC4F8C005D3F881
:10E78000483318BF45F040052BB11B691BB1284623
:10E79000BDE87040184770BDE02A0020082B00201B
:10E7A000282B00202C2C0020042D0020082D0020D8
:10E7B0008C300020A43000202DE9F04F8FB04FF0B6
:10E7C0000009012B06460F4690468DF80D90ADF8D6
:10E7D000109002D84C46BC4202D30FB0BDE8F08F77
:10E7E000305D02F007FB2044B842F6DC335D651C67
:10E7F000023BEDB2112BF0D801A252F823F000BF7A
:10E8000049E8000873E8000871E9000899E9000880
:10E8100017EA00083DEA0008A3EA0008CBEA00086E
:10E8200051EB0008DBE70008DBE70008A5EB000878
:10E83000DBE70008DBE700084DEC000875EC00089A
:10E84000ADEC0008E1EC0008052002F07BFB70B1A4
:10E850000521002002F03CFB725DBA4BE51C02343E
:10E86000E4B283F85C24325D83F85D24EDB22C467B
:10E87000B1E700238DF80E308DF80F308DF814308D
:10E880008DF81830B9F1000F6DD1AF4C4FF005097C
:10E8900094F87C208DF831206B1E94F839208DF887
:10E8A0003320334494F838200B938DF8342094F8B7
:10E8B0001A3194F868208DF83520D4F82C218DF881
:10E8C00032300A9273B37B1C5B1BDBB28DF83030A5
:10E8D00006AB019305AB009394F848000DF10F03CC
:10E8E0000DF10E020AA903F07BF88DF80D0000F07F
:10E8F0000700072813D194F939209DF90E3084F8C8
:10E9000039309A429DF80F3084F83830B8BF012270
:10E910009DF81430B8BF84F81D2184F868304FF09A
:10E92000000A09E00523D1E701220DF10D010320C2
:10E9300002F078F90AF1010A5FFA8AF29DF81830BC
:10E94000B3FBF9F19142EFD82B44DDB26B1EDBB281
:10E950009F420BD9F25C032A9AD0AF4288BF1D4672
:10E960004FF0010983E70534E5B2F9E71D46F7E703
:10E97000735D754903F00F03012281F81B310234E6
:10E9800002FA03F3A1F82031E4B2002204A9042022
:10E9900002F048F925466AE707238DF80D30735DCC
:10E9A000C3F3021203F00F038DF82830E31CDBB22F
:10E9B0008DF82920F25C231DDBB2651DF35C023467
:10E9C000E4B21B0443EA0223325D5F4C134364222A
:10E9D000534394F848000B930AA903F010F800F091
:10E9E0000703072BEDB28DF80D000CD19DF82830F0
:10E9F00084F8703084F878300B9BE36663679DF889
:10EA0000293084F869308DF81000012204A905200E
:10EA100002F008F92BE74B4BD3F8483363B11B687E
:10EA200053B1984708F03F038DF810008DF811306E
:10EA3000022204A90620EBE7FF20F3E703238DF869
:10EA40000D30735D8DF81C300AAB0693E31CDBB20E
:10EA5000A51DF25C231DDBB206A9F35C1B0443EA8F
:10EA60000223A21CD2B20534B25C13436422534386
:10EA7000E4B20A9300230B93335D8DF83030324BB0
:10EA800093F8480002F0C1FFC3B20028EDB28DF840
:10EA90000D30FFF6ECAE8DF81030012204A90720EE
:10EAA000B6E7735D03F00F03012B4FF47A7238BFA2
:10EAB00001235343244A0234936503F57A73D365E3
:10EAC000E4B2002204A9082062E7735D1E4DC3F37F
:10EAD00040128DF8152095F84800C3F3001205A9DF
:10EAE00003F00F038DF814208DF8163002F093FF19
:10EAF00002340130E4B23FF44DAFBDF81430134A94
:10EB0000A5F87C309DF816309DF814A0D05CF3F782
:10EB100051FA0223C5F880000AA995F848008DF83B
:10EB200028308DF82AA002F015FF95F939300690AB
:10EB300040B29842B8BF184685F83900002204A9AF
:10EB4000092025E7A4300020E02A0020B182030834
:10EB500003238DF80D30735D8DF82830E31CDBB294
:10EB6000651DF25C231DDBB20234F35CE4B21B04CE
:10EB700043EA0223325D1343642253430B93644BF5
:10EB80000AA993F8480002F04CFFC3B20028EDB286
:10EB90008DF80D30FFF66BAE8DF81030012204A910
:10EBA0000A2035E7092002F0CDF9DFF868B1002826
:10EBB00049D00921002002F08BF90023ADF81E3066
:10EBC000A31CDBB2F25CE31CDBB216F803A0735D9E
:10EBD0004FEA0A4A4AEA022A4AEA030A231DDBB23A
:10EBE000A51D0534F35CE4B24AEA036A335D4FF4D1
:10EBF0007A7253430AAC1B122046ADF81C3007F062
:10EC000065F8454B53440693DBF83C3300930DF114
:10EC1000180A9AE80600DBF8383308A807F012F85B
:10EC2000099B009394E80600089B504606F0EFFF0E
:10EC30009AE8030007F022F801F0DCFF0123EDB2AF
:10EC40008BF8383413E68BF8380410E60C2002F009
:10EC500079F900283FF40BAE0C21002002F038F9BE
:10EC60002C4B93F89034043B012B7FF600AE01F05F
:10EC7000BDFFFCE5A31CDBB2725DF15CE31CDBB203
:10EC8000651DF35C0434E4B21B04305D43EA0123E8
:10EC900013436421594300F00F0001F0A8FFEDB2C7
:10ECA0008DF81000012204A91120B1E60D2002F018
:10ECB00049F900283FF4DBAD0D21002002F008F9EE
:10ECC000A31CDBB2154AF05C735D1268251D03348A
:10ECD000E4B243EA0020315DEDB201F08AFFC6E5FF
:10ECE000725DA31C251D0334DBB2E4B2F15C335D1D
:10ECF0001B0443EA012313436420584301F07BFFC4
:10ED0000EDB28DF81000012204A9132080E600BFA7
:10ED1000E02A0020A4300020803DD5127424002079
:10ED20000E4B93F89124920703D593F88F24012A70
:10ED300008D90B4991F81A2122B18A6A501C18BFD0
:10ED400001328A620022A3F8182483F81A24D3F827
:10ED5000402322F00202C3F840237047A430002071
:10ED6000E02A002070B5184C1848194D07F032F908
:10ED7000D4F84033D4F89804D5F8906023F02003F9
:10ED8000C4F8403338B107F0EBF8864203D20023D1
:10ED900085F83A3070BD0120FFF766F90028F9D0F8
:10EDA0000B28F7D095F8393084F84234092094F8CC
:10EDB000183484F8453484F8410402F0ABF8BDE817
:10EDC0007040FFF7ADBF00BFA43000200C3400201E
:10EDD000E02A0020094BD3F84023012A0AD0084931
:10EDE0000978C90708D43AB993F89204013818BFD2
:10EDF000012070470020704701207047A430002098
:10EE000088240020034BD3F84003431E5842584146
:10EE1000704700BFA43000202DE9F04FA9B0EFF3F8
:10EE2000108272B6DFF8F0B20021DBF80030CBF8C8
:10EE3000001082F31088B94C002B00F0E180DAB2A8
:10EE40009B06039264D5B64D95F81831022B02D07B
:10EE5000B44BDB6A9847EFF3108872B6B24F07F0F5
:10EE600075F83E68D4F8B013361A3144AF4807F04D
:10EE700039F9AE4807F0FCF8D4F8B413AC48314483
:10EE800007F030F9AA4807F0F3F888F3108894F8EF
:10EE90001A34002B00F06B81152312A995F8480055
:10EEA0008DF8483002F056FDD4F8B4130F900144A9
:10EEB000A04807F017F99F4807F0DAF83B6894F884
:10EEC0001B24EB620DAF38468DF870201D9306F0C1
:10EED00023FFD5F82831009306AE97E80600D5F851
:10EEE0002431304606F0AEFE96E803001FAB83E8FF
:10EEF0000300D4F81C341E9395F8303195F848007F
:10EF0000003B18BF01231CA98DF8713002F02BFDC6
:10EF1000039BDF0648D5824DDFF81CA2D5F8E4201C
:10EF200004929BF80020BAF90A809AF90C90A4F890
:10EF30008C84002363F300020A9384F84434A4F819
:10EF4000223484F82534C4F82834A4F82C3484F806
:10EF50002E34C4F8303484F82034C4F8343484F8BF
:10EF60003834C4F83C346F4B8BF8002094F890246C
:10EF7000DB6A84F88E9484F88F24DAF80470BAF887
:10EF80000860984794F88F3413B9694807F022F85D
:10EF90003146384601F017FE8346002800F0EA802B
:10EFA000A4F87E8484F88094039B19071AD55C4BDF
:10EFB00093F81831022B02D05A4BDB6A9847022093
:10EFC000FEF712FF84F8410401F0A4FF94F81A340C
:10EFD00013B1012384F8193494F8913443F01003E9
:10EFE00084F89134039B5A0703D506210520FEF7C8
:10EFF00065FF039B9B0703D504210320FEF75EFFFB
:10F0000001F000FE94F89124D7065FD5002384F820
:10F010009234D4F840331E0644BF23F08203C4F870
:10F02000403312F0050F00F0FB820B2001F08AFF45
:10F03000002800F0F58294F89134DD0700F1F082A9
:10F04000580740F10783D4F8403323F00203C4F893
:10F050004033D4F8402382BB94F8915415F0010159
:10F060001EBF2B4662F3000384F8913494F8913468
:10F070005E0744BF6FF3820384F89134012384F860
:10F08000923421B1D4F844332C481B6898476D075B
:10F090000BD52B4801F062FF01F090FF28B194F8E6
:10F0A000913443F0040384F8913401F098FD94F80E
:10F0B00091346FF3041384F89134012384F892346B
:10F0C00094F8913443F0200384F8913494F8913407
:10F0D00018070AD56FF3C3031A4984F89134D4F89A
:10F0E0004433A1F12400DB68984794F891349907E0
:10F0F0000AD56FF34103134984F89134D4F84433AB
:10F10000A1F16C005B68984794F89034022B1BD1F6
:10F11000FFF722F918E000BF88240020A430002067
:10F12000E02A0020A489030884240020243400203D
:10F130003C340020A434002074240020E434002057
:10F14000F83400203035002094F891349A0640F1CC
:10F15000C4826FF3451384F89134D4F84033002B04
:10F1600040F0BB8229B0BDE8F04FFFF7ABBA84F89E
:10F170004134A3E695F81831012B0CD101F027FD9D
:10F18000804668B1584601F017FD584601F019FD58
:10F19000042384F88F347EB9012384F821344FE1AD
:10F1A00001F017FD0028F6D0404601F006FD40466C
:10F1B00001F008FD0523ECE73B7805935B09013B73
:10F1C000062B00F21782DFE813F007001502950006
:10F1D0001502920015020602102EDDD995F8303185
:10F1E0001297F6B28DF84C60002BD5D11CA804F014
:10F1F0003FFA12AA1CA9FF2002F072F99DF85830BC
:10F20000C3F3030307468DF82C3095F8480095F8B2
:10F210007D308DF82D3007220BA902F0AEFB002FB8
:10F220005DD100285BD09DF853309DF85220159990
:10F23000C5F8E4101B0443EA02239DF85120022084
:10F240001343C5F8E03004F021FA9DF8583095F8E2
:10F25000480085F82E71C3F30212C3F3030385F847
:10F26000703085F878309DF8593085F86920012B89
:10F2700038BF01234FF47A725343AB651344EB65F7
:10F280000DF15A034FF001081093113E94F81B340E
:10F290008DF83C300FA985F868808DF8446002F045
:10F2A00074FB0223404685F8303101F04BFE18B163
:10F2B0004146384601F00CFE94F88F34012B00F2E1
:10F2C000A78194F81A34002B40F09A8194F8913475
:10F2D00043F0100384F89134FEF786FD64E60120C4
:10F2E00001F030FE0028E7D001210720E2E70123EA
:10F2F00084F8203495F87D308DF82E3094F824343D
:10F300008DF82D3095F88C3095F848000D330BA909
:10F310008DF82C3002F01EFBA6F10D031BB20990F4
:10F3200023EAE37300B283423FF736AF0B2E7FF63A
:10F3300033AFBA4B25931CA8FF231C978DF874603C
:10F340008DF8983002F0E2F9074600287FF424AFE8
:10F3500095F81831012B13D101F039FC002872D037
:10F36000384601F029FC384601F02BFC04239DF8B7
:10F370007C101E9884F88F34C1F3001101F041FC19
:10F380009DF87C301E99C4F8341413F00F0203D09A
:10F390009DF89000002862D19DF89800002861D067
:10F3A000002A7FF4F9AE9DF89020002A14BF4FF098
:10F3B00003084FF0020800220A92D5F8EC2095F8D5
:10F3C000E900914251D100284FD0D5F80C1195F8A1
:10F3D000EAB009680A9195F81811022902D10321AF
:10F3E00084F88F14B8F1030F7FF4D6AE13F0600FDA
:10F3F0007FF4D2AE0492012795F82E31BBF1000FB5
:10F4000036D0BBF1010F13D1012B33D16FF00906B8
:10F4100046FA08F606F00106C6F10206F6B2BDF895
:10F420007E100AAA304601F0E5FE38B3072823D043
:10F43000012384F821340A9BC4F83034C4F86C34B6
:10F44000FEF720FDB0E501F0C4FB002898D0384657
:10F4500001F0B3FB384601F0B5FB052387E74FF019
:10F460000008A8E74FF00108A5E74FF0010BC3E73C
:10F470000426D4E70326D2E70823DAE71CAB00937F
:10F4800004990A9B3246584601F076FF20B10228C3
:10F4900014BF0B230A2380E60A9BC4F83034C4F857
:10F4A0006C349DF87C3084F82104C3F3401384F855
:10F4B0002E3484F8443494F88F3484F82274012B69
:10F4C0009EBF0122A86285F81E21012FC4F82804DE
:10F4D00084F82C0484F8410438D1022284F82024D2
:10F4E00095F83A20002A4AD19DF87C20D60646D4C9
:10F4F000012B94F840149DF87C2005D8012901D1F6
:10F50000900601D501F020FCB8F1020F94F88F3479
:10F5100043D0B8F1030F0AD09DF87C10B8F1010F69
:10F520004A4601F00F0120A83BD0FFF745F99DF8AE
:10F53000903084F82334259BC4F828349DF8983003
:10F5400084F82C34012384F82D3430E0059A02F03D
:10F55000E002A02A1BD195F82E11012285F83A204D
:10F5600009B927996963012B84F8202407D9D5F8B4
:10F570009020C4F83C24DAF80020C4F8982495F8C8
:10F580001821002AB4D1012284F82524B0E70022F2
:10F5900085F83A2084F82024A6E79DF8981025984D
:10F5A0004A46FFF709F99DF8903084F823349DF816
:10F5B0009020E02A08D195F81F312BB984F8232434
:10F5C000C4F82834A4F82C3494F8913443F002039E
:10F5D00084F8913470E6114D013EB2B2791C284690
:10F5E00004F01EF90323A4F82034C4F8285484F846
:10F5F0002C64E9E7012384F82134FEF743FC5BE641
:10F6000094F84434002B3FF461AE0020FEF726FC52
:10F6100094F88F34022B3FF45FAE57E6DC320020C3
:10F6200094F89134590715D5012001F08BFC60B195
:10F63000012001F05FFC08B984F81804D4F84033C5
:10F6400023F00203C4F8403304E0062001F07AFC02
:10F650000028F3D194F89134DA077FF5FAAC94F8E6
:10F6600040240AB1032A18D11D4A94F8181492F8BC
:10F670006820914205D29B0723D594F88F34012B43
:10F680001FD8184806F0A6FCD4F8403323F0200316
:10F69000C4F84033FFF744FBDBE4012A11D194F8AE
:10F6A0001924002A3FF4D5AC0D4A94F8181492F8A6
:10F6B00068209142E5D29F0703D594F84434002B8B
:10F6C000DFD194F8913400206FF3041384F891345F
:10F6D00084F81904FFF746FBBBE429B0BDE8F08FBE
:10F6E000E02A00200C3400202DE9F04F89468DB02F
:10F6F00090460746002800F08F81002900F08C8199
:10F700000368002B00F088814368002B00F084819F
:10F710008368002B00F08081C368002B00F07C819F
:10F72000104602F013F9002800F07881BD4CBE4D60
:10F73000384601F083FB40F2C4520021204604F019
:10F7400083F840F21C520021284604F07DF8B74BA4
:10F75000C4F82C3104F50973089304F50A730026E4
:10F760004046099308A9B24B84F848800A9384F86C
:10F77000186184F88C608DF82C6002F0F9F80F2382
:10F7800006A994F848008DF8183002F0E3F8801BC1
:10F7900018BF01204FF00A0B84F81C0106A994F849
:10F7A00048008DF818B002F0D5F84FF0060A84F83A
:10F7B000DC0006A994F848008DF818A002F0CAF8F9
:10F7C000102384F8DD0006A994F848008DF818305D
:10F7D00002F0C0F81123C4F89C0006A994F8480070
:10F7E0008DF8183002F0B6F81223C4F8A00006A96C
:10F7F00094F848008DF8183002F0ACF81323C4F8E0
:10F80000A40006A994F848008DF8183002F0A2F878
:10F810001423C4F8A80006A994F848008DF81830FD
:10F8200002F098F81623C4F8AC0006A994F8480032
:10F830008DF8183002F08EF8172384F8B10006A96D
:10F8400094F848008DF8183002F084F818230DEB76
:10F850000301C4F8B400C4F8BC0094F848008DF863
:10F86000183002F077F8C0B21D2384F8B80084F88D
:10F87000C00006A994F848008DF8183002F06AF824
:10F880001E2384F8C40006A994F848008DF81830A7
:10F8900002F060F81F2384F8C50006A994F8480018
:10F8A0008DF8183002F056F82023C4F8C80006A9D5
:10F8B00094F848008DF8183002F04CF80B23C4F887
:10F8C000CC0006A994F848008DF8183002F042F8F0
:10F8D0000C2306A9A4F8D00094F848008DF818303D
:10F8E00002F038F8D4F89C306365D4F8A030A365F2
:10F8F000D4F8A430E365D4F8A83023664FF00108AB
:10F90000D4F8AC300590A4F8D200636684F8B080D7
:10F91000C4F894B084F898A0C4F84CB084F850A00F
:10F9200084F8688084F81F81C5F84893FEF7AEFD1F
:10F93000C5F84473C4E90B663E4B84F8198185F819
:10F940009164C5F8408332464FF0FF31009605F5CB
:10F950005A7006F0E1FA384B009632464FF0FF310C
:10F9600005F5607006F0D8FA344B009632464FF039
:10F97000FF3105F5667006F0CFFA02AF304B009606
:10F9800032464FF0FF3105F5806006F0C5FA384683
:10F9900006F0C2F997E8030004F5927383E80300C8
:10F9A000284B294F1E60294BC5F84C33284BC5F80E
:10F9B0005433284BC5F85C33274BC5F85033274BDD
:10F9C000C5F8583305F553703B68984704F5A670A1
:10F9D00003F06AFC20B1112630460DB0BDE8F08F6F
:10F9E000204601F0D7FB0028F5D101F00DF9B8B998
:10F9F0001B4801F021FC06460028ECD17B699847A2
:10FA000003F0ECFEBB6D94F819019847FB6A984728
:10FA1000012385F89234DFE70326DDE70926DBE7DB
:10FA20001326D9E7E02A0020A430002000040001BA
:10FA30008C24002065ED00082DE6000875E600081E
:10FA40005DDE000888240020A48903081DE000086A
:10FA5000D1DF000819DE0008A9DF000881DF0008F7
:10FA6000C82B002008B5034B0020C3F84003FEF765
:10FA7000BBF908BDA430002010B5FFF7ABF90A4C64
:10FA800060B90A4B93F81831022B02D1084BDB6A9C
:10FA900098470123C4F84033002010BDD4F8400338
:10FAA000013818BF0120F8E7A4300020E02A002028
:10FAB000A489030838B5124C204606F08BFA04F1ED
:10FAC000180006F087FA04F1300006F083FA04F11A
:10FAD000980006F07FFA01F081F80A4B0025DB6AF6
:10FAE000984744F8285CFEF7EDFD0749074840F2C7
:10FAF000C45203F095FE012344F8283C284638BD43
:10FB00000C340020A4890308E02A00201C250020D2
:10FB100070B52E4B8AB0054693F8DD008DF80900CC
:10FB200093F8DC008DF80A0029489A6A90F81804C6
:10FB3000039200268DF80B0004960C46002940D055
:10FB40000692D3F8882007921A8F93F81A118DF82D
:10FB5000151052BAADF8202093F87C2093F8483065
:10FB60008DF8243003AB8DF822008DF8232000930C
:10FB70000DF10A020DF10B030DF1090105A88DF835
:10FB8000146000F0A9FF9DF90900FEF74FF96070BD
:10FB900004A801F0EFF8B0B9049A0F2A0DD86378E1
:10FBA0009A420AD81544AB42A3EB02012CBF0020B5
:10FBB00001202170C0000AB070BD0023237008200E
:10FBC000F9E70320F7E71320F5E700BFE02A00205C
:10FBD000A43000201FB50446002800F010810378EF
:10FBE000412B00F20781DFE813F0420049004D008D
:10FBF0005100550059005E00050105010501050190
:10FC00000501050105010501650069006D00780029
:10FC10007F00820085008A0088008C00900093009D
:10FC2000960099009C009F00AE00B200BA00B6009A
:10FC3000BE00C100C500CE00CA00CC000501D20044
:10FC40000501050105010501050105010501050184
:10FC50000501050105010501050105010501DA00A0
:10FC6000DE00E200E700EB00EF00F300FC00664B73
:10FC700093F818312371002004B010BD624B93F843
:10FC80003031F7E7406803F0ADFCF4E7406803F07B
:10FC9000EFFCF0E75C4B93F81A31EBE75A4BD3F8E3
:10FCA000E0306360E7E7584B011D93F8300103F043
:10FCB000F7FCE0E7544B93F81931DBE7524B93F82C
:10FCC0008C30D7E71C238DF808304F4B02A993F8EE
:10FCD000480001F03FFE6060CDE74C4B043493E8F0
:10FCE000030084E80300C6E7494B0434F7E7494BB7
:10FCF0000434F4E7484B0434F1E71A23E3E719230B
:10FD0000E1E7414B93F86830B4E73F4B5B6DC8E7E0
:10FD10003D4B9B6DC5E73C4BDB6DC2E73A4B1B6E21
:10FD2000BFE7394B5B6EBCE702238DF80830364BDA
:10FD300002A993F87C2093F848008DF80A2001F07E
:10FD400009FE207197E7304B93F8DD3092E72E4B98
:10FD500093F839308EE72C4B93F8DC308AE72A4B46
:10FD600093F8383086E7284BDB6C9AE7264B93F8FC
:10FD700050307FE7244BD3F8843063607BE7224B1D
:10FD80008FE7264B8DE7204BD3F8CC30F5E71E4BA1
:10FD9000D3F82C31436001F06BFEA0606BE71A4B87
:10FDA000D3F890307DE7184B93F81F3162E7164B7C
:10FDB000B3F88830A3805EE7134BB3F88A30F9E7D5
:10FDC000114BB3F8D030F5E70F4BB3F8D230F1E771
:10FDD0000D4B93F848200AB1062A12D1B3F8A0358A
:10FDE000E8E7094B93F848200AB1062A09D1D3F86D
:10FDF000A43556E704B0BDE8104000F0F3BE032080
:10FE00003AE7182038E700BFE02A00204C2B0020FA
:10FE1000942B0020542B00209C2B00201C2500201C
:10FE20007FB5044610B9032004B070BDA34DD5F8CA
:10FE300040339A0700F16F820278412A00F268820B
:10FE4000DFE812F04200470055005B005F006400ED
:10FE500069007600810087008D00930099009F0063
:10FE6000A500AB00B5006602BA00DC00EF00160189
:10FE70003801290142014B014F01530157015B0138
:10FE800066025F01710199018701AB01B101B801FF
:10FE9000BD01C201660228026602660266026602AF
:10FEA0006602660266026602660266026602660212
:10FEB0006602660266026602340239023E024302AC
:10FEC00048024D0252025C020079FEF773FA30B12B
:10FED000AAE70379022BA6D0794A82F8303195F847
:10FEE000913443F0200385F8913400209CE740686A
:10FEF00003F06AFB0028F2D095E7406803F0A8FB06
:10FF0000F8E76F4B027983F81A21E8E76C4B4268F7
:10FF1000C3F8E020E3E76A4E416896F8300103F049
:10FF2000B5FB00287FF47FAF6368C6F8E430D6E7FE
:10FF3000416800293FF477AF002001F0B1FA0028B2
:10FF4000CDD0112070E7416800293FF46CAF01204B
:10FF5000F3E7416800293FF466AF0820EDE7416808
:10FF600000293FF460AF0920E7E7416800293FF42A
:10FF70005AAF0C20E1E7416800293FF454AF0D204F
:10FF8000DBE7416800293FF44EAF0E20D5E741681A
:10FF900000293FF448AF0F20CFE74A4C484B007987
:10FFA00083F81901A36D9847E36A984797E7444B94
:10FFB000027983F88C2092E7414E037A8DF8043061
:10FFC00096F8480096F87D308DF80530072201A993
:10FFD00001F0D3FC00283FF426AF636896F8480090
:10FFE0000193002201A901F0C8FC00283FF41BAFD7
:10FFF0006C36D4E9010186E8030070E7304E037ADD
:020000040801F1
:100000008DF8043096F8480096F87D308DF805306C
:10001000072201A901F0B1FC00283FF404AFB43677
:10002000E7E7274E037A8DF8043096F8480096F8F3
:100030007D308DF80530072201A901F09EFC0028D3
:100040003FF4F1AED4E9010106F1740383E8030043
:1000500096F81831022B7FF442AF96F83031002B1E
:100060003FF43DAF174BDB6A9847FEF775F936E76B
:10007000134E037A8DF8043096F8480096F87D30D8
:100080008DF80530072201A901F077FC00283FF424
:10009000CAAEBC36ADE74368029301238DF80C303D
:1000A000074B02A993F8480001F074FC00287FF484
:1000B00016AFB8E6436802930023EFE7A4300020B0
:1000C000E02A0020A489030803795A1E0E2A3FF66D
:1000D000AAAE934A82F8683001E7914B42685A65AC
:1000E000FDE68F4B42689A65F9E68D4B4268DA650A
:1000F000F5E68B4B42681A66F1E6894B42685A6610
:10010000EDE6874C037994F848008DF80430062218
:1001100001A901F032FC00283FF485AE9DF80430BF
:1001200084F8DD30DBE67E4C03798DF8043094F8FA
:10013000480094F87C308DF80630052201A901F0C2
:100140001CFC00283FF46FAE9DF8043084F8393071
:10015000C5E6734C037994F848008DF804300A2200
:1001600001A901F00AFC00283FF45DAE9DF80430BF
:1001700084F8DC30B3E66A4C037994F848008DF8D3
:100180000430092201A901F0F8FB00283FF44BAE2E
:100190009DF8043084F83830A1E6614B4268C3F81A
:1001A0009420DA649BE65E4B027983F8982083F80A
:1001B000502094E65A4B4268C3F884208FE6584B8F
:1001C0004268C3F8CC208AE6012B40F0A480554C4D
:1001D0002421204603F03AFB636A984201D017209D
:1001E00022E61C2104F1280003F030FB636C9842E6
:1001F000F5D14FF4807104F1480003F027FBD4F8E7
:1002000048319842EBD1D42104F5A67003F01EFBCF
:10021000D4F820329842E2D1002104F5097003F0AD
:1002200015FBD4F824329842D9D14FF4607104F50B
:100230000A7003F00BFBD4F8A8359842CFD11421F3
:1002400004F2AC5003F002FBD4F8C0359842C6D19A
:10025000334E2146304640F2C45203F0E1FA2046C4
:1002600040F2C452002103F0EFFA95F81B3485F8F0
:10027000E833736FC5F8EC3396F87D3085F8F833C2
:1002800040F20123A5F8FA33274B96F819019B6D2C
:10029000984724E68379012B3FF6C5AD204B426891
:1002A0004068C3F82C2100F091FF48E61C4B4268DF
:1002B000C3F8902013E61A4B027983F81F210EE64B
:1002C000174B8288A3F8882009E6154B8288A3F88B
:1002D0008A2004E6124B8288A3F8D020FFE5104B59
:1002E0008288A3F8D220FAE50D4B93F848200AB192
:1002F000062A12D1A288A3F8A025F0E5084B93F8AE
:1003000048200AB1062A08D16268C3F8A425E6E5A8
:1003100000F06AFCDBE5012086E5182084E500BFDB
:10032000E02A00201C250020A4890308DFF880C0F3
:10033000F8B5DCF840339B07064635D48778002FA4
:1003400034D105460FCD1B4C0FC40FCD0FC42B6805
:1003500023609CF89134B16843F020038CF8913409
:100360003378BBB10D2001F09BF810B1112738464E
:10037000F8BD7168B07801F031F90028F6D1B27893
:100380000D4B302101FB02334FF0FF32D3F80C311B
:100390001A60ECE70E2001F083F80028E6D1F1683E
:1003A0000F2001F07DF8E8E70127E0E71627DEE7F8
:1003B000A4300020C82B0020E02A0020F0B5134F05
:1003C000D7F840339B078BB006461AD4D8B9104CE7
:1003D00094F8E930BBB10146242201A801AD03F035
:1003E00033FA0FCDE8340FC40FCD0FC42B68236050
:1003F00097F8913443F0200387F8913430460BB0DE
:10040000F0BD0126FAE71626F8E700BFA430002069
:10041000E02A002000F00303F7B51C33294F1370C6
:100420001546D7F8402392070C4647D40A78013A7C
:10043000012A03D90325284603B0F0BD00283FD187
:10044000214E96F8E920002A3AD003F00F032B70D2
:1004500091F908308DF8043096F8480096F87D3010
:100460008DF80530072201A901F087FA18B12B7821
:1004700023F004032B70636896F848000193002270
:1004800001A901F07AFA18B12B7823F008032B7038
:100490002D78002DCED194E807000C4B83E807009F
:1004A00097F8912442F0200287F891242278012ABB
:1004B000C1D1A3F1180000F0A3FBBCE70125BAE706
:1004C0001625B8E7A4300020E02A0020E02B002009
:1004D0002DE9F04387B00023ADF800300646002830
:1004E00000F0EE800361FEF775FC20B10124204688
:1004F00007B0BDE8F08300F067FD0028F6D100F0FA
:100500005DFD014618B96F48142203F09DF96E4D48
:1005100095F89134012243F0040385F8552485F8B9
:10052000913433788DF804300021013B8DF805209B
:10053000ADF806100C2B00F2BB80DFE803F007B922
:10054000B9B97982B9B990B9AD9AA900D5F8407313
:1005500017F02007CAD196F80480B8F1020F46D1EF
:10056000DFF868815A4CFDF791FF96F9051098F86D
:1005700048003A4601F05BFA88F83900B37988F808
:100580003830384607238DF80530FDF713FFFF2379
:1005900004F58670A5F80C31C5F8084185F804719A
:1005A00003F066F804F58A7003F01CF83846FDF78E
:1005B0005BFD0446002839D096F9051098F84800EC
:1005C000012201F034FA88F83900D5F89434336107
:1005D000002C71D000F0F2FC002888D195F89134FD
:1005E00085F81A0460F3820385F891347FE7B8F147
:1005F000010F4FF00204E8D1DFF8D0908DF81440DD
:1006000099F8480089F81D7102A901F0B1F9337910
:1006100089F830318DF805708DF80680FDF7F2FB12
:1006200095F8913443F0100385F891340024CCE719
:1006300000226946022000F0F5FA0028F6D01324C3
:10064000C3E7244BB288DB6B96F90C10B06898476F
:10065000D5F8403343F00203C5F84033E6E702A97A
:100660000D2000F055FB0028E0D0002269460D2047
:10067000E1E7164B93F81831D3B9347904F0070049
:1006800000F0ABFA8DF80040012269461020D2E755
:10069000002269461220CEE78DF8072000F08EFA7E
:1006A000044638B900F087FA204600F089FABDE721
:1006B00002248AE7012488E701A800F0D3FB16E7AB
:1006C000032414E7F8340020A4300020E02A00209E
:1006D000A6300020A48903082DE9F04F99B0804688
:1006E000059118B9032019B0BDE8F08F002303610C
:1006F000FEF770FB0446002840F0A58046460FCE6A
:100700000EAD0FC51422524898F800A0B8F80C702E
:1007100098F90EB04F4E214603F096F84E4B012249
:1007200083F8412496F83021022A25460BD196F809
:100730001821022A07D196F81E2122B9BAF1010F19
:1007400038BF4FF0010ABAF1010F2BD0BAF1030FF5
:100750002AD0BAF1000F33D102229DF83C30DDF8E7
:100760004090029362F34715012496F87C108DF8AF
:10077000321002220CA996F848008DF8302001F0C2
:10078000E9F896F81A3196F830C196F81D1140B282
:10079000002B63D0BCF1010F57D1002955D1002C9B
:1007A00061D153E00422D8E70023DDF83C90BDF886
:1007B00040709DF942B0029365F01F050124D4E713
:1007C0004FF0000BD946CDF808B0CEE74FF001004E
:1007D00084F81A04D2E005F29A420BA900F0D6FA86
:1007E000002800F015811320049B33871A4B002248
:1007F00083F81A2423E105F29A452A460BA900F052
:10080000C5FA0028EFD10B9B84F82801C4F82C51BD
:1008100084F83031FCE0B9F1000F00F0F980002AD3
:1008200000F0F6804946E01C02F0FAFF94F83732F7
:1008300001332380ECE01220D6E70220D4E7072022
:10084000D4E71320D2E701204DE7FCB90220F6E0FF
:10085000E4340020E02A0020A4300020002CF5D051
:100860005845B8BF584696F87C308DF820000522D0
:1008700096F848008DF8223008A901F07EF800288B
:100880003FF430AF9DF8203086F839306F4A704B16
:10089000D2F89804D3F8904038B105F061FB6C4B66
:1008A00084423CBF002283F83A20198F1A8F93F8B4
:1008B00030010491996A099152BA0028BFD093F887
:1008C0001B0100B9186393F81801ADF858200138DE
:1008D00093F87C2093F81A411491D0F1000BD3F8CF
:1008E00088108DF85B204BEB000B93F8482093F8B1
:1008F0003A0093F868308DF85A3009AB0093554BA5
:1009000003904FF001008DF84C0015918DF85C209C
:10091000A3F12F01A3F1300213A88DF84D4000F090
:10092000DBF8039B4FEA0B1B4BEA431B00264BEA09
:10093000801B4BEAC413B145444C039308BF3746B0
:100940003A46494604F59C70CDE90A669B462680E6
:1009500084F81A6402F064FFE9B2A570C5F3421589
:10096000FAB2042D3A4E039B84F837223FF42EAF9F
:10097000072D3FF450AF022D7FF45FAF364D84F862
:100980000D110420029984F80401FF2084F80C0161
:1009900084F8281184F81431D6F8E410C4F808510A
:1009A00005F59B730AA8C4F8101184F83021C4F827
:1009B0002C3100F013FC00287FF43DAF0A9BA4F813
:1009C00044040BA8A4F81631C4F84C3400F0D2F952
:1009D00000287FF408AF0B9BD3B196F93900FDF7DF
:1009E00025FA94F83732002B3FF405AF0B9B0F2B01
:1009F0003FF6F1AE05F58B720BA90F2000F0C6F99A
:100A000000287FF4F0AE0B9B63F3030B84F814B162
:100A10000598FDF729FB00287FF4E6AE099B86F8D0
:100A20003A00B36200F082F900287FF40AAF94F82C
:100A3000913484F840A443F0010384F89134034BCB
:100A4000D3F89434C8F810304DE600BFA43000202D
:100A5000E02A0020482B0020A630002037B50B4D9F
:100A60008DF8040004460F2295F8480001A900F013
:100A700084FF40B1064A85F81C4192F8913443F056
:100A8000200382F8913403B030BD00BFE02A00207B
:100A9000A430002010B5FEF7EFFF044688B90A48DD
:100AA00005F098FA094805F095FA094805F092FA18
:100AB00000F094F8FDF7EAFC064BDB6A9847204605
:100AC00010BD0124FBE700BF0C34002024340020BB
:100AD0003C340020A48903082DE9F04F8BB04778FF
:100AE0000093149B90F90C8090F90D6090F80EB073
:100AF0008A464168196004469146002F58D0022367
:100B00008DF8103004A9C37B007C8DF8123000F002
:100B100021FFB4F808C0618943B260689845454632
:100B20006144B8BF1D46604534BF00270127884295
:100B300009D30A218DF81010207C019304A900F03C
:100B400009FF019B46B2B4F808C0608961680CEBEC
:100B5000400E714519D3A1EB0C01B1FBF0FC00FB79
:100B60001C1191B9984503DC2378CBB94FF0010BE8
:100B700021238DF81030207CE37B8DF8115004A9DF
:100B80008DF8123000F0E6FE45B2009B8AF8005066
:100B9000384689F8006083F800B00BB0BDE8F08FEC
:100BA0000223207C8DF8243006A900F0E1FEDDE769
:100BB0004546EAE770477047704770470020704726
:100BC0007047704770470020704700207047002032
:100BD000704700207047002070477047704770478B
:100BE00002207047022070470220704770470020A3
:100BF000704770477047002070470020704770476B
:100C0000704770477047000010B5054C4FF40372F1
:100C10002046002102F018FE0020C4E9000010BDAB
:100C2000C03500202DE9F8438146904600293CD08C
:100C30001F4C2023224604F1100012F8017F6FBBE5
:100C40008242FAD11B4E3368013403B934607368B1
:100C500003B11C6000252560C4F8088074601FFA89
:100C600088F284F80490601D02F0DAFDB9F1110FEA
:100C70004FF0000398BF104D6373D6F8083298BF49
:100C800025FA09F503F1010398BF05F00105434476
:100C90002573C6F808323846BDE8F883013B13F0E7
:100CA000FF030446C6D10227F5E70127F3E700BF9B
:100CB000C7350020C03500202007020010B518B34A
:100CC000124A1368984204D103681360002305E0B8
:100CD0000B46002BFAD019688842F9D15168884236
:100CE00008BF53600BB101681960D2F808328168FF
:100CF000013B00245B1A04602146C2F8083210222E
:100D000002F0A2FD204610BD0120FCE7C035002006
:100D1000054B1B6813B11A798242FAD1002B0B6084
:100D20000CBF032000207047C035002010B5054BD4
:100D3000186800B910BD037B04680BB9FFF7BEFF4C
:100D40002046F6E7C035002038B5084B084C186837
:100D500000B938BD03790568112B05D824FA03F3CF
:100D6000DB0701D5FFF7AAFF2846F1E7C0350020D1
:100D70002007020028B1044BD3F80832036000209A
:100D800070470120704700BFC03500202DE9F041B9
:100D900007460E46154642B339B3154B1C6800236F
:100DA0002CB93046FFF7E6FF0020BDE8F081A268CD
:100DB000F91A0132914215D32279EA54581C22893A
:100DC0005FFA80F8611D55FA80F002F029FDA368F2
:100DD000246898445FFA88F3E2E720462568FFF725
:100DE0006DFF2C46002CF8D1DBE70120DDE700BFCA
:100DF000C03500200238C0B211289ABF014B185CE0
:100E000000207047C182030830B50B4B93F82020B7
:100E10000446084672B100211C330578A54208D06B
:100E200001319842CDB214BF04301038AA42F4D830
:100E3000002030BD1046FCE7CC37002010B5084C30
:100E400000232060142204F10C00FF2184F82030DC
:100E5000C4E9010002F0F8FC012384F8213010BD40
:100E6000CC37002010B50E4A92F82010042915D86E
:100E7000936804781C7044785C70C47880789870AB
:100E80000131DC7082F8201002F11C018B4214BF8A
:100E9000043302F10C039360012010BD0020FCE735
:100EA000CC370020094B93F8200068B15A6803F151
:100EB0001C018A4200F1FF3014BF043203F10C021E
:100EC00083F820005A600120704700BFCC37002013
:100ED00010B5074B93F820200446084632B15968F4
:100EE000FFF792FF10B101234470837010BD00BF63
:100EF000CC37002008B5064B93F820202AB159685A
:100F0000FFF782FF08B1407808BD0120FCE700BF71
:100F1000CC37002030B50A4A92F82010536882F886
:100F2000210061B1916801241C32DD78587005B947
:100F30009C70934214BF0433103B9942F5D130BDED
:100F4000CC37002008B5044B5968FFF75DFF003827
:100F500018BF012008BD00BFCC370020F7B5042220
:100F6000154E044600210DEB020096F8207002F0A9
:100F70006BFC0025EBB29F4201D803B0F0BD736853
:100F8000197821705A786270987838B133682046A1
:100F90009B689847FFF786FF0135EBE7DB788DF814
:100FA00004108DF805208DF80730FFF77BFF01A8AE
:100FB000FFF758FFF0E700BFCC370020014B93F854
:100FC00020007047CC370020034B93F82000042802
:100FD00094BF002001207047CC3700201FB50024AB
:100FE000CDE90244C41F8DF800408DF801100C0AB1
:100FF000ADF80420090C120C8DF803108DF80620B2
:101000008DF8073002461B0A012168468DF8024020
:101010008DF8083002F073FA002818BF0E2004B0D3
:1010200010BD2DE9F04188B090460D460F9A074655
:10103000002847D000240121CDE904448DF8101088
:101040009DF838108DF81510ADF81630190CCDE953
:1010500000441B0ECDE902448DF81930ADF81A207A
:10106000130C120E07948DF818108DF81C308DF8A3
:101070001D20E3B21E01002DF6B203DC002008B0F3
:10108000BDE8F081013310218DF81F3042466B46D8
:101090000DEB010002F0C9F90346A8B9102D28464E
:1010A0003E44A8BF10206946327811F801CB0133C5
:1010B00082EA0C02984206F8012BF5DC103D2DB2B5
:1010C0000134D6E70920DAE70E20D8E701380328F3
:1010D00015D8DFE800F002080C100A4B1B681B69EA
:1010E0000B6000207047074B1B685B69F8E7054BF6
:1010F0001B689B69F4E7034B1B68DB69F0E705207D
:10110000704700BFF03700202DE9F041C4B00C4615
:101110004A9E17461D468046B8B3B1F5807F36D843
:101120004FF488720021684602F08EFB4923009339
:101130004FF48073ADF804302B0C8DF80830330C6D
:10114000ADF80650ADF80A608DF80C302246002349
:10115000414604A82D0E360E8DF80E308DF809503C
:101160008DF80D608DF80F4002F05AFB04F110016C
:101170004B9A3B4689B2684602F041F910B101280A
:1011800018BF0E2044B0BDE8F0810920FAE70D2019
:10119000F8E7000010B590B10A4C28220021206029
:1011A00002F052FB2368084A1A6000204FF0FF3219
:1011B000C3E90302C3E90522C3E9072210BD0820E1
:1011C000FCE700BFF037002000010101024B1B6863
:1011D00018600020704700BFF037002030B1044B8A
:1011E0001B68DB68013303600020704709207047EB
:1011F000F037002013B500230C460193CAB101A9B2
:10120000FFF764FF18B9019B591C02D1146002B0AA
:1012100010BD99B2611A002901DD5C18F6E702D110
:1012200013600720F3E71B0C1B0403F580331C44F9
:10123000ECE70920EBE7000028B1044B1B681C33E6
:101240004362002070470920704700BFF03700203C
:101250001FB5044600B3002303A8039302F0A6F9C8
:10126000104ABDF80C30126820469380E38200F0EB
:10127000A8FA98B904F118030093216801231322F6
:1012800002F0B2F860B9204600F09BFA003818BFAF
:101290000120000104B010BD0920FBE71020F9E790
:1012A0000E20F7E7F0370020F0B5054687B01C4662
:1012B00013B9092007B0F0BD2E4E3368DB688342B6
:1012C00055D894F82020002A0CBF08220922834216
:1012D00005D3204600F0A9FA68B11020EAE7002300
:1012E00001900093A36894F82810606AFFF799FEB4
:1012F0000028EED0DEE723792168B4F808C0A7689B
:10130000043B9AB20029D4D0B2F5807F2DD8ADF835
:101310000EC08DF817304FEA174C04F12C033F0E26
:101320008DF8117000932F0C08234FF0490EADF883
:101330000C008DF814708DF816002F0E0DEB0300C5
:10134000CDF808E08DF810C0ADF812508DF815708A
:1013500002F04AF808B10E20ACE7204600F065FA2A
:101360000028BAD13368DD60A4E70D20A2E706208B
:10137000A0E700BFF03700202DE9FF410A9D80461D
:101380000F4616461C46002D5AD0002303A91046CE
:101390000393FFF79BFE18B1062004B0BDE8F0816F
:1013A000039B9C4201D80133F6D1284600F0AEF9E8
:1013B000002847D1264B1A78424503D01A79424576
:1013C00042D10120AA68BA4240D103EB8002EB6A05
:1013D00092F801802979CDE9004304399278286890
:1013E0003B4689B2FFF790FE0028D6D195F8203011
:1013F0000194002B4FF00103009314BF42460822D2
:1014000095F82810686A3B46FFF70BFE0028C4D108
:10141000013E032EC1D8DFE806F002070B0F0D4B8B
:101420001B681C611C62B8E70A4B1B685C61F9E72A
:10143000084B1B689C61F5E7064B1B68DC61ACE759
:101440000920AAE70F20A8E70B20A6E70220A4E7BF
:10145000A0040020F03700201FB50B294FF0000337
:10146000CDE90033CDE902330A4607D00C2914D068
:101470000A2910D00A2005B05DF804FB012802D12A
:1014800020238DF800300021684602F038F800284B
:1014900018BF0E20EFE73023F3E70B21F4E700003D
:1014A00038B5054602F026F8044610B10E24204651
:1014B00038BD002DFBD1094B1B680B219878FFF735
:1014C000CBFF0028F2D10C21FFF7C6FF0028EDD199
:1014D0000A21FFF7C1FF0028E9D0E7E7F037002035
:1014E0002DE9F04380468FB00C461746002A6BD09A
:1014F000002969D0002529461D2206A805951EF061
:101500009DF88DF81350344D2B680DF114099E8809
:10151000CDF804900DF1130302933B7900933B68DF
:1015200032462146404602F006F800284ED138687F
:101530003A79494602F074F9384600F099F80028E3
:1015400046D13C7AFA79BB79240444EA02241C434C
:101550002B689A6894423DD99C609DF813000B213A
:10156000FFF77AFF034658BB0C21FFF775FF0346D0
:1015700030BB0A21FFF770FF034608BB7B7ABA7ABB
:10158000FF7A3F0447EA02271F433A463346214683
:101590000920FFF723FD034690B933463A4621461A
:1015A0000820FFF71BFD034650B92A689DF8131069
:1015B00091700021D1604FF0FF31C2E904119161B7
:1015C00018460FB0BDE8F0830923F9E70E23F7E7CB
:1015D0000F23F5E70323F3E7F037002070B588B059
:1015E00000293FD0214C2378834231D02379834294
:1015F0003AD101220023CDE90133CDE9053304EBD3
:101600008204039307930123C1F30720CDB28DF821
:101610000030C1F30743090E8DF802008DF8041065
:1016200002268DF812008DF814106278E1788DF89A
:10163000015068468DF803308DF810608DF8115018
:101640008DF8133001F05BFF20B10E2008B070BDA3
:101650000022CFE7A278E17804A801F050FF00282B
:10166000F4D0F2E70920F1E70B20EFE7A004002017
:1016700010B50446002845D00168002942D011F871
:10168000013B43710322063002F0CAF820460322D0
:1016900050F8091B043102F0C3F82168CB79E360EC
:1016A0000A7A43EA0223E3604A7A43EA0243E360A8
:1016B0008A7A43EA0263E360CB7A23740B7B637418
:1016C0002379212B1AD110220D3104F1120002F0DE
:1016D000A7F81D222168501C8B5C6362085C43EAFA
:1016E0000023901C6362085C033243EA0043636298
:1016F0008A5C43EA02636362002010BD112B03DCA5
:101700000D22E7E70220F8E70120F6E710B50446CE
:10171000002854D00168002951D00B7843714B78D0
:1017200083608A7843EA02238360CA7843EA0243EB
:1017300083600A7943EA026383604B7903738B7990
:10174000C381CA7943EA0223027BC38102F00F02FC
:101750000831103002F064F8237B002203F00F03FD
:1017600084F8202084F82820227903F10800111A37
:1017700004290DDD21680933043AD21A085C84F883
:101780002000D2B2606A84F82820194402F048F898
:10179000237922681A44002012F8043CE36212F80C
:1017A000031C43EA0123E36212F8021C43EA0143EB
:1017B000E36212F8012C43EA0263E36210BD0220E7
:1017C000FCE710B5044660B3036853B30279162AE8
:1017D00029D942791A700146082251F8060B0130C6
:1017E00002F028F82146082251F80E0B093002F0C9
:1017F00021F82368E28A5A74E38A22681B0A9374E8
:101800002368A269DA74A36922681B0A1375236826
:10181000628B5A752368E27E9A7517232371002024
:1018200010BD0120FCE70220FAE738B50446002885
:1018300063D00168002960D0037B90F8282003F072
:101840000F03002A57D108332079043213449842F9
:1018500055D363790B702368A2685A70A368226815
:101860001B0A937023686289DA702368E27A1A711E
:101870002368227B5A712368E2899A71E38922687E
:101880001B0A2146D371227B51F8100B02F00F0284
:10189000083001F0C5FF237B94F8282003F00F03E4
:1018A00003F108052AB1226894F82010515503F17C
:1018B0000905206894F82820616A284401F0B0FFE7
:1018C00094F828302268E16A2B44D1545A1CE16A0A
:1018D000206892B2090A81549A1C2168E08D92B264
:1018E0008854DA1C216894F82F0092B2043388548B
:1018F0002371002038BD0933A6E70120FAE7022052
:10190000F8E70000024B1A8810431880704700BFA8
:10191000F437002008B5074B1B883BB1FEF7ACF845
:10192000002814BF6FF00200002008BD6FF0010016
:10193000FBE700BFF437002010B5034B00241C80E8
:10194000FEF790F8204610BDF4370020B0FA80F082
:101950004009704782B018B9084602B000F0CAB812
:10196000002002B0704710B9084600F079B97047FE
:1019700010B9084600F090B9704703460846114672
:101980000BB900F0DDB90020704710B9084600F02F
:1019900039BD704710B9084600F0FEB90020704705
:1019A00010B40446084611461A46019B14B910BCEF
:1019B00000F00CBA10BC70470346084611460BB93C
:1019C00000F036BA0020704710B4044608461146AD
:1019D0001A4614B910BC00F0A3BA002010BC70471E
:1019E00030B40546084611461A46DDE902341DB9F1
:1019F000029430BC00F022BB002030BC704710B90C
:101A0000084600F0D3BB0020704710B9084600F02C
:101A100037BD0020704710B9084600F0E2BB002037
:101A2000704710B9084600F0DFBB0020704703463E
:101A3000084611460BB900F0F9BB0020704710B4FE
:101A40000446084611461A46019B14B910BC00F022
:101A5000EFBB092010BC704710B40446084611467D
:101A60001A4614B910BC00F02DBDC8B210BC7047A6
:101A70000048704701000102064B10B51B6A04467E
:101A8000984730B10448054B204498428CBF002051
:101A9000012010BDA4890308403576C9405DC60009
:101AA000F0B5114B85B00C4610491F56054601F0A4
:101AB00017F80F4BE4B25E6A072D4FF00103CDE932
:101AC000024301460AD105220023CDE900234FF449
:101AD0007A727A431846B04705B0F0BD082200205C
:101AE000CDE900203A46F5E78C8303086C830308B0
:101AF000A48903081FB5002300930378013B372B0B
:101B000021D8DFE803F01C242020201E20202020E4
:101B10004143454E2055585B5E6164206C1E6E73D8
:101B2000787A7D207F8326202020202020202020DE
:101B30002020202085878C2020858C208E92C378C1
:101B40000BB102230093009805B05DF804FB837885
:101B5000F6E743788DF8043007238DF80530837855
:101B6000003B18BF01235B008DF8063010238DF871
:101B70000730314B1B6801A803F55872CDE90223E9
:101B800000F08EFF0090DEE74023DBE72023D9E75B
:101B9000827890F9013012B9284AD35CD2E7284AFA
:101BA000FBE7827890F90130002AF8D1254AF4E762
:101BB00040F6B833C6E74FF47A73C3E74FF4FA63DD
:101BC000C0E741F28833BDE741F27073BAE71E48BF
:101BD0004FF47A7101F008FE00F5FA60D2E71B4B72
:101BE000B0E7154B1B6803F55873ABE7124B1B6846
:101BF00003F55B73A6E71023A4E70F4B1B68A1E76F
:101C000001239FE74FF0834300939CE7104BFBE7D2
